:100000000C9467420C9410430C9410430C941043CE
:100010000C9410430C9410430C9410430C94104314
:100020000C9410430C9410430C9410430C94104304
:100030000C9410430C943A440C9410430C941043C9
:100040000C9410430C9410430C9410430C941043E4
:100050000C9410430C9410430C9410430C941043D4
:100060000C9410430C9410430C9410430C941043C4
:100070004656495650565356565649565656565653
:100080005956495656565956595653565956595611
:100090005C565956000000000000000000000000FF
:1000A0000000000000000000000000000000000050
:1000B0000000000000000000000000000000000040
:1000C0000000000000000000000000000000000030
:1000D0000000000000000000000000000000000020
:1000E0000000000000000000000000000000000010
:1000F0000000004900000000004952520000004981
:1001000052531C25004952522425251B52525C2D66
:100110002D1C121200000000000000000000000072
:100120004049494900404949525B5B5B4A52525B36
:100130001C1C13125B1C241C12090909241B120924
:100140000909090A0A0A0A0A0A0A0A130A0A120A01
:100150000A12130A000000000000000092525252DE
:100160005252524913121309001C1B130A12124057
:100170001B65641C090A0009241B1C65120000256C
:100180001C1C1C1C010025241C1C1C1C00242524D8
:1001900024241C1C00000000000000004940000056
:1001A0000000000052494900000000001C5B4A4862
:1001B000000000001C25524900000000652464492D
:1001C0000000000065256449000000006D2E5C49B8
:1001D000000000000000000000004052000000008D
:1001E0000049525C000000005352242500000053D7
:1001F0005225252500004A5225251B0000005B25BD
:100200001300001B005B53000A1C3737095B1C6599
:100210007F372E2E522E2E1C131312002E251B1349
:10022000120000121C1C12000012251C12000012E9
:100230002E371C1300132E37361C131B37372E2E68
:1002400025131C1C2E2E2E2E1B1C1C1C6E6E6E1CB1
:100250001C1C1C1C09131312121313001313131369
:10026000131C0009131313131C0100371313131C61
:1002700013002E2E1B1B1C1C001C772E1B1B250085
:10028000137F251C1C1C010A37241C1C1C130A2E5E
:1002900025250900132E2425252525252E25252550
:1002A0002525252525252D2E251B1C1C2E2E251C00
:1002B00013251B13251C1C1C1C0109521C1C13009C
:1002C000011C5B5C0A000165775C1B00016E7F6EA0
:1002D000521B00006D1C5249000000001C1353000B
:1002E000000000001C524A00000000005B5B0000A0
:1002F000000000005C0000000000000000000000A2
:1003000000000000000000000000000000000000ED
:1003100000000000135B7F776E6E6E6E136577765C
:100320006E6E6E6E1B65777676766E771B5BBF762C
:10033000B676767609136DBFB7B6B765001B125C4B
:1003400076BF766D0000121B125B5B5C0000000044
:10035000090A12136E77241C1C1C1C1C77251C1CFC
:100360001C1C24256E1C1C1C2425251B1C1C242540
:1003700025130000646D6D1B00096EBF6D5B0912D3
:100380006EBF6D5B5B125B645B121312131B121268
:10039000090100001C242E1C0900096E25240100FF
:1003A00009767F7F000012777F7F641264BFBF777A
:1003B0005B121B09BF6D5B121B09000012131B09A6
:1003C0000000000009000000000000000000000024
:1003D000000000007F7F53131300000064121B0114
:1003E000000000001B1200000000000000000000E0
:1003F00000000000000000000000000000000000FD
:1004000000000000000000000000000000000000EC
:1004100000000000000000000000000026000000B6
:10042000260026262F0000002F00000037000000C5
:1004300037000000FF000000FF000000BF000000C8
:10044000BF0000BF3700003700003700002626003D
:1004500000002626000000000000000026262600DE
:100460002626262600002F002F000000003700005F
:1004700037000000FF000000FFFFFFFF000000004A
:10048000BF00000000000000370000002626260004
:100490002626262600000000000000002600262652
:1004A0002626000000002F0000002F00000037006B
:1004B000000037000000FFFFFFFF00000000BF004A
:1004C0000000BF000000370000003700260026268D
:1004D0002626000000000000000000000000262684
:1004E00026002600002F00002F002F0037000000FC
:1004F00037000037FF000000FF000000BF000000D1
:10050000BF0000BF37000037000037002626260056
:10051000000026000000000000000000000026008F
:100520000000000000002F00000000000037000065
:1005300000000000FF0000000000000000BF0000FD
:10054000000000000000370000000000000026004E
:10055000000000000000000000000000000000009B
:10056000000000000000000000000000000000008B
:10057000000000E400000000099BEDF60000009B75
:10058000A4ADBFBF00529BA4767F7FB75B9B6D7706
:100590007F766EB700000000000000000000000041
:1005A0005BB6F6F6005BF6FFFFFFFFBFF6FFFFFF4F
:1005B000FFBFBFAEFFBFFFFFFFB7AD65BFBFFFFF10
:1005C000B7B6AD65B7BFFFFFBFB7AE6EB7BFFFFF32
:1005D000BFB7B7650000000000000000F6F6EDEDC3
:1005E000ADA4A49BB66D6D5C526E65646565655285
:1005F00065766D255C5C52536E24656E6552526E55
:10060000252524255B52772D25252524526E6E2D18
:100610002525252500000000000000009B49000062
:1006200000000000A49B9200000000002564934994
:1006300000000000652E9B52000000006D256552F1
:10064000000000006D2D6552000000006E2E645207
:1006500000000000000000000000495B00000000F6
:10066000004A5B65000000005B9B6D2D0000005B95
:100670005B2D2E250000525B2E2E1C0900015B2DE8
:100680001C01091C005C5B014A65777F4A5B1C6E9C
:100690007F7777769B77776D656E6EA4776E6565ED
:1006A000655BA4B725255C52526DBFBF1309496431
:1006B0007FBFBFBF095C7F7FBFBFB7BF7F7F777F33
:1006C0007FB7BFBF77777F7F6EB7BFBF777F7F6E04
:1006D00077BFBFBFB6FFFFFFBFBFB75BBFFFFFFF67
:1006E000BFBFA464BFFFFFFFBFADA47FBFFFFFFF7D
:1006F000BFA4BF7FFFFFFFBFADBFBFBFFFFFFFB600
:10070000BFBFBF77FFFFF7BFBFBF7777FFFFFFBF59
:10071000BFBF64526D7F6E2E2D2D256E7F766E6E5F
:100720006E2E2565777777762E1C25247F776E25AC
:100730001C251C1B776525251C090A5B6E6E1C0990
:10074000492564645B494A6E7F645C005377BF77D8
:100750005B5C00006E255B4A000000001C1B5B0018
:1007600000000000245B5300000000005B5C000000
:100770000000000064000000000000000000000015
:100780000000000000000000000000000000000069
:10079000000000005B5C7FBF777677775C6D7FB78A
:1007A000777777775C6D7FBF777777BF5C64BFBF04
:1007B000BFBFBF7F0A5C6EBFBFBFBF760065646D01
:1007C000BFBFBFBF00005B6D646DADB60000000031
:1007D000125B646D777F6E6E77BFBFBF7F766D767D
:1007E00077BFBFBF776D6E767FBFBFBF6D6E767F01
:1007F000BFB7ADF676BFBF76A4ADFFFFBFB664ADA1
:10080000FFFFFFFFB6ADBFFFFFFFFFF6ADB6AD6464
:100810005B520000FFFFBFBFAD5B64BFFFFFB6AD23
:10082000ADBFFFBFFFF6FFFFFFFFBF64FFFFFFFF8E
:10083000BFB6765BFFFFFFBFBF5B0000FFFFFF5C43
:1008400000000000A4000000000000000000000004
:1008500000000000BFBF645C5C0000006E5C654986
:10086000000000006D5B00000000000000000000C0
:100870000000000000000000000000000000000078
:100880000000000000000000000000000000000068
:100890000000000005040001020304050607080922
:1008A0000A0B0C0D000E0F10111205030013141586
:1008B000161718191A1B1C1D1E1F0000020800081D
:1008C0005504085A0000F8000990000A1E3205007D
:1008D00000FF000000BB0800000000334F414F1430
:1008E00050EF53D953444F534F624FBF53704F7E15
:1008F0004F000000000000000000000000000000A9
:1009000000000000000000000000000000000000E7
:1009100000000000000000000000000000000000D7
:1009200000000000000000000000000000000000C7
:1009300000EBEBEBEBEBEBEBEBEB00000000000074
:1009400000EB00EBEBEBEBEBEBEB00EB0000000064
:1009500000EB00EB0000000000EB00EB0000EBEB15
:10096000EBEB00EB0000EB0000EB00EB0000EB001A
:10097000EBEBEBEBEBEBEBEBEB0000000000000034
:10098000EBEBEBEBEBEBEB00EB0000000000EB0024
:10099000EB0000000000EB00EBEBEBEBEBEBEB0014
:1009A000EB00000000000000EBEBEBEBEBEBEBEB04
:1009B000EB0000000000000000000000000000004C
:1009C0000000000000000000000000000000000027
:1009D0000000000000000000000000000000000017
:1009E0000000000000000000000000000000000007
:1009F00000000000000000000000000000000000F7
:100A000000000000000000000000000000000000E6
:100A1000000000000000000000000000000000C90D
:100A2000C90000000000C900000000000000C9006B
:100A3000C9000000000000000000000000000000ED
:100A400000000000000000000000000000000000A6
:100A500000C9C9C9C9C9C9C9C9000000000000004E
:100A6000000000000000000000C9C9C9C9C9C9C907
:100A7000C9000000000000000000000000000000AD
:100A80000000000000000000000000000000000066
:100A900000C9C9C9C9C9C9C9C9000000000000000E
:100AA000000000000000000000C90000000000007D
:100AB000C90000000000000000000000000000006D
:100AC0000000000000000000000000000000000026
:100AD000000000000000000000C9C9000000000084
:100AE000000000C90000000000C900C900000000AB
:100AF00000EBEBEBEBEBEBEBEBEB000000000000B3
:100B000000EB00EBEBEBEBEBEBEB00EB00000000A2
:100B100000EB00EB0000000000EB00EBEBEBEBEB7D
:100B2000EBEB00000000000000EBEBEBEBEBEBEB82
:100B3000EBEBEBEBEBEBEBEBEB0000000000000072
:100B4000EBEBEBEBEBEBEB00EB0000000000EB0062
:100B5000EB0000000000EB00EBEBEBEB0000EB0028
:100B6000EB0000EB0000EB00EBEB00EB0000EB0018
:100B7000EBEB00EB0000EB00EBEB00EB0000EB001D
:100B8000EBEB00EB0000EB00EBEB00EB0000EB000D
:100B9000EBEB00EB0000EB00EBEB00EB0000EB00FD
:100BA000EBEB00EB0000EB00EBEB00EB0000EB00ED
:100BB000EB0000000000000000000000000000004A
:100BC000000000EBEBEBEBEBEB0000EB00000000B8
:100BD000000000EB00EBEBEBEB0000EB00EB0000A8
:100BE000000000EB00EB0000000000EB00EB000059
:100BF00000000000000000000000000000000000F5
:100C000000EBEBEBEBEBEB00000000000000EB0077
:100C100000EBEBEBEB00EB0000000000EB00EB0067
:100C200000000000EB00EB0000000000EB00EB0018
:100C30000000000000C90000C900000000C9000059
:100C4000C900000000C90000C900000000C9000080
:100C5000C900000000C90000C900000000C9000070
:100C6000C900000000C90000C900000000C9000060
:100C7000C9000000000000000000000000000000AB
:100C8000000000000000000000000000B7B70000F6
:100C900000000000B7B700000000000000000000E6
:100CA0000000000000000000000000000000000044
:100CB00000C9000000000000C9C9000000000000D9
:100CC000C9C9000000000000C9C900000000000000
:100CD000C9C9000000000000C9C9000000000000F0
:100CE000C9C9000000000000C9C9000000000000E0
:100CF000C9C90000C900000000C90000C900000007
:100D000000C90000C900000000C90000C9000000BF
:100D100000C90000C900000000C90000C9000000AF
:100D200000C90000C900000000C90000C90000009F
:100D300000EB00EB0000EB00EBEB00EB0000EB0046
:100D4000EBEB00EB0000EB00EBEB00EB0000EB004B
:100D5000EBEB00EB0000EB00EBEB00EBEBEBEB0065
:100D6000EBEB000000000000EBEBEBEBEBEBEBEB55
:100D7000EB0000EB00EB0000000000EB00EB0000DC
:100D8000000000EB00EB0000000000EB00EB0000B7
:100D9000000000EB00EB0000000000EB00EB0000A7
:100DA000000000EB00EB0000000000EB00EB000097
:100DB00000000000EB00EB0000000000EB00EB0087
:100DC00000000000EB00EB0000000000EB00EB0077
:100DD00000000000EB00EB0000000000EB00EB0067
:100DE00000000000EB00EB0000000000EB00EB0057
:100DF000000000C9C9C9C9C9C900C9000000000074
:100E000000C900000000000000C900000000000050
:100E100000C900000000000000C900000000000040
:100E200000C900000000000000C900000000000030
:100E300000C9C9C9C9C9C90000000000000000C933
:100E40000000000000000000C900000000000000D9
:100E5000C900000000000000C90000000000000000
:100E6000C900000000000000C900000000000000F0
:100E7000C9C9C9C9C9C9C9C9C90000000000000061
:100E80000000000000000000000000000000000062
:100E90000000000000000000000000000000000052
:100EA0000000000000000000000000000000000042
:100EB000000000EB00EB0000000000EB00EB000086
:100EC000000000EB00EB0000000000EB00EBEBEBA0
:100ED000EB0000EB00000000000000EBEBEBEBEBA5
:100EE000EB00000000000000000000000000000017
:100EF00000000000EB00EB0000000000EB00EB0046
:100F000000000000EB00EB0000EBEBEBEB00EB0074
:100F1000000000000000EB0000EBEBEBEBEBEB0064
:100F200000000000000000000000000000000000C1
:100F3000000000000000000000000000B7B7000043
:100F4000000000B7B7B7B7000000B7B7B7B7B7B77B
:100F50000000B7B7B7B7B7B7000000B7B7B7B7006B
:100F600000000000B7B70000000000000000000013
:100F700000C900000000000000C9000000000000DF
:100F800000C900000000000000C9000000000000CF
:100F900000C900000000000000C9000000000000BF
:100FA0000000C90000000000000000C9C9C9C9C98B
:100FB000C900000000000000C9000000000000009F
:100FC000C900000000000000C9000000000000008F
:100FD000C900000000000000C9000000000000007F
:100FE000C9000000000000C900C9C9C9C9C9C900B9
:100FF00000000000000000000000000000000000F1
:1010000000000000000000000000000000000000E0
:1010100000000000000000000000000000000000D0
:10102000000000000000000000C9C9C9C9C9C9C941
:10103000C9C9000000000000C9C90000000000008C
:10104000C9C9000000000000C9C90000000000007C
:10105000C9C9000000000000C9C90000000000006C
:10106000C900C900000000C9000000C9C9C9C90001
:101070000000000000000000000000000000000070
:101080000000000000000000000000000000000060
:101090004900000000000051A3000000000000A271
:1010A0009A000000000000A3E300000000005AEBDB
:1010B000EB000000004952A2A30000499A9AE3EB1A
:1010C000EB009AA39A9AE3EBEBA39A9AE3EBEBEB90
:1010D000EB9A9AE3EBEBEBEBEB9AEBEBEBEBEBA3A3
:1010E00051E3EBEBEBEBA3519AEBEBEBE3E39A9AD7
:1010F000EBA39A510000000000EBEBEBA3510000C2
:1011000000EBEBEBEBEB9A0000EBEBEBEBEBEB9A92
:1011100000A3EBEBEBEBEBE349099AEBEBEBEBEB2F
:101120009AA349A3A351525A49EBA39A5A5249513F
:10113000000000C9C9C9C9C9C900C9000000000030
:1011400000C900000000000000C90000000000000D
:1011500000C900000000000000C9000000000000FD
:101160000000C90000000000000000C9C9C9C9C9C9
:10117000C9C9C9C9C9C9C90000000000000000C927
:101180000000000000000000C90000000000000096
:10119000C900000000000000C900000000000000BD
:1011A000C9000000000000C900C9C9C9C9C9C900F7
:1011B000000000C9C9C9C9000000C900000000C979
:1011C00000C9000000000000C9C9000000000000C4
:1011D000C9C9000000000000C9C9000000000000EB
:1011E000C9C9000000000000C9C9000000000000DB
:1011F000C9C9C9C9C9C9C9C9C900000000000000DE
:1012000000000000000000000000000000000000DE
:1012100000000000000000000000000000000000CE
:10122000000000000000000000C9C9C9C9C9C9C93F
:10123000C9C9C9C9C9C9C9C9C9000000000000009D
:10124000000000000000000000000000000000009E
:10125000000000000000000000000000000000008E
:10126000000000000000000000C9000000000000B5
:10127000C9000000000000000000000000000000A5
:10128000000000000000000000000000000000005E
:10129000000000000000000009000000000000083D
:1012A000A2000000000000115A00000000000936F2
:1012B0002E0000495AA3A3A39A009AE3EBEBEBEBB1
:1012C000EB08A2EBEBEBEBEBEB49525AA3EBEBEBAE
:1012D000EB5151499AEBA3A3E39AEB9A9A9A5109DD
:1012E00051A2EB9A51A2EBE30812A39A9AE3EBEB1B
:1012F000515A49000000000000EBE39A0900000089
:1013000000EBEBEBA349000000EBEBEBEBE3080099
:1013100000EBEBEBE39A9A0000E3EBEBEB9AA349CB
:10132000009AEBEBEBE3A29A009AEBEBEBE39AA3C8
:10133000080000000049E3EBEB00000008A3EBA36A
:101340009A000000A3EBE39A9A0000A2EBEB9A51FB
:101350009A51A3EBEBA3519A4B9AEBEBEB9A49050D
:101360000749E3EBEB51030707009AEB9A4905079E
:1013700007EBEBEBE3529AEBA3A3EBEBEB51A309E7
:1013800012A2EBEBEBE3521B37519AEBEBEB092D7F
:10139000374B099AEBEB09362D070509A3EB112E04
:1013A000360707059AEB522D3F07070703A3511B8A
:1013B00025EBEB499AEB5A510012A351E3EBA39AA8
:1013C000002D52A35A1252520012095224373609E4
:1013D000001BBF133F372409000900363724BF0024
:1013E000002D123F36000000001B253F2D525100FA
:1013F00000000000000000253F0000000000BF13B7
:101400003F0000000051002D3F0000005AA31B3F89
:1014100037000052A29A12372E00495A529AA25B04
:1014200052009A04060B5252A3514A0707070707B6
:1014300004249AA3521152E39A2449082D37129A90
:101440009A1BBF092D3F129A510A001B372E09A380
:10145000E31B3F3F36099AEBEB1B3636129AEBEB58
:10146000A3A35B115AEBE35A09539AA39A520305BB
:1014700007A3EBEBEBEB9AA3519AE3EBEBEB9AA30D
:101480009A9AEBEBEBEBA29AA2EBEBEBEBEBEBA379
:1014900008EBEBA3A3EBEBA300A3A3A39AA3EB9A04
:1014A00000495A519A9AEB9A00060BA351E3EB9A22
:1014B000000009A3524A070707000051A30B0707C2
:1014C000070000005103070707000000514A060704
:1014D0000700000008A39A530B0000000000095108
:1014E0005A000000000000000000000000000000A2
:1014F0000007070706529BA3A30707070707054B2B
:101500005207070707070707070707070707070720
:101510000704040B05070707079A9AA29A04060610
:10152000040000009A9B525A9A000000005149089A
:10153000009A5A1B52A3510000529AA39A9A5A0039
:101540000007054B0B529A000007070707035A00D4
:1015500000070707070B5100004B520B059A0000CC
:10156000005A51529B9A00000000000051090000EF
:10157000000000000000C900C90000000000C90010
:1015800000000000000000C9C900000000000000C9
:10159000000000000000000000000000000000004B
:1015A000000000000000000000000000000000003B
:1015B00000C9C9C9C9C9C9C9C900000000000000E3
:1015C000000000000000000000C9C9C9C9C9C9C99C
:1015D000C900000000000000000000000000000042
:1015E00000000000000000000000000000000000FB
:1015F00000C9C9C9C9C9C90000000000000000C96C
:101600000000000000000000C9C9C9C9C9000000ED
:10161000C900000000C90000C900000000C90000A6
:10162000C900000000C90000C900000000C9000096
:10163000C9C9000000000000C9C900000000000086
:1016400000C900000000000000C900000000000008
:1016500000C900000000000000C9000000000000F8
:1016600000C900000000000000C9000000000000E8
:10167000C9C9000000000000C9000000000000000F
:10168000C900000000000000C900000000000000C8
:10169000C900000000000000C900000000000000B8
:1016A000C900000000000000C9C9000000000000DF
:1016B000C90000C9C9C9C9C9C900C90000000000E2
:1016C00000C900000000000000C9000000C9C9C92D
:1016D000C9C90000C900000000C90000C90000001D
:1016E00000C90000C900000000C90000C9000000D6
:1016F00000C900C900000000000000C9000000008F
:1017000000C9C90000000000000000000000000047
:1017100000000000000000000000000000000000C9
:1017200000000000000000000000000000000000B9
:10173000009A0B050507070707A39A529A040707A3
:1017400007000000525A050707000000005252052A
:101750000700000000005A9A5300000000000051EA
:101760005A0000000000000000000000000000001F
:101770000006060505060707070707070707070707
:1017800007070707070707070706060707070707EB
:10179000075B9A04070707070749519A4A05070795
:1017A00007000000529A530B0B0000000008519AEA
:1017B000A207075251A3EBA20007070A51EBEBA3C4
:1017C000000707089AEBEBA308070451A3EBEBEB28
:1017D00051075251E3EBE3520004A3A2A2520000CE
:1017E0000052490000000000000800000000000056
:1017F00000000000000000000000000000000000E9
:1018000000000000000000000000000000000000D8
:1018100005000000000000020700000000000003B7
:1018200007000000000000030700000000000001A6
:101830000600000000122D373F0000001B373F3F1D
:101840003F0204040A2E3F3F3F070707070A362DD1
:101850000B070707040012030707070702BF020769
:10186000070707070400030707070707070203071F
:1018700007372E1B00000000003F3F3F2E120000E4
:10188000003F3F3F3F370A000002031C373F360945
:101890000007070513372E1B0007070400252D2D11
:1018A00000070702BF1B2E3609070703001B363649
:1018B0000A0000000000000000000000000000001E
:1018C0000000000000000000000000000000000018
:1018D0000000000000C9C9C9C900000000000000E4
:1018E00000000000000000000000000000C9C9C99D
:1018F000C900000000C90000C900000000C90000C4
:10190000C900000000C90000C900000000C90000B3
:10191000C9C9C9C9C9000000C90000000000000011
:10192000C9000000000000C900C9C9C9C9C9C9006F
:1019300000C9C9C9C9C9C9C9C9C900000000000096
:1019400000C900000000000000C90000C9C9C9C9E1
:10195000C9C90000C900000000C90000C90000009A
:1019600000C90000C900000000C90000C900000053
:1019700000C9C9C9C900000000000000C9F7F7F795
:10198000F7000000C9F7F7F7F7C9C9C9C900000097
:101990000000000000000000000000000000000047
:1019A0000000000000000000000000000000000037
:1019B000000000000000000000F7F7F7F7F7F7F766
:1019C000F7F7F7F7F7F7F7F7F70000000000000068
:1019D0000000000000000000000000000000000007
:1019E00000000000000000000000000000000000F7
:1019F0000000000000C9C9C9C9F7F7F7F7C900001E
:101A000000F7F7F7F7C900000000000000C9C9C9D6
:101A1000C9000000000000000000000000000000FD
:101A200000000000000000000000000000000000B6
:101A300000C9C9C9C9C9C9C9C9000000000000005E
:101A4000C900000000000000C9C9C9C9C9C9000017
:101A5000C900000000C90000C900000000C9000062
:101A6000C900000000C90000C900000000C9000052
:101A7000C9C90000C900000000C90000C900000079
:101A800000C90000C900000000C90000C900000032
:101A900000C9000000C9C9C9C9C900000000000090
:101AA0000000C90000000000000000C9C9C9C9C980
:101AB000C90000000000000000000000000000005D
:101AC0000000000000000000000000000000000016
:101AD00000C9C9C9C90000000000000000000000E2
:101AE000000000000000000000C9C9C9C9000000D2
:101AF0000000000000000000090000000000001BC2
:101B00002E000000000013362E0000000009362EC3
:101B10002D00000000253736120000000936362D52
:101B2000000000001237362D030000001B3F3F3736
:101B30000B1C363F3F362512003F3F3F3F3F3F37AC
:101B40002D37241B1B363F3F3F0903070603243F65
:101B50003FBF03070707042E2D00060707070609E6
:101B600001070707070706BF010707070707030065
:101B7000020000000000000000090000000000005A
:101B8000002D000000000000003F240000000000C5
:101B900000130B0000000000000507060200000013
:101BA00000050707070200000007070707030000FA
:101BB0000000000000000000020000000000000023
:101BC000001B0000000000000936090000000000B2
:101BD0000924240000000000092436090000000048
:101BE000121B361B0000000012092E2E0000000000
:101BF0001B06070704130307071B1313253F2404C1
:101C0000073F373F3F3F37240B3F3F3F3F3F3F3F7B
:101C10003737252425373F3F3F3737372D1B2D37A3
:101C20003F3F3F3F3F37251B243F3F3F3F3F3F3F25
:101C30002E070706012436370907070613373636FD
:101C400009040313363F372E002E36372E3F3F242C
:101C5000003F3F3612363709003F371B253F24002F
:101C6000002513243F370000002D363F37120000B7
:101C7000000000001B3F362E250000001B3F1B2DDF
:101C80003F09000012372D243F3612000936371362
:101C9000372E2D00002D3F2D1B1C3609001B3F3F0A
:101CA000360936240009363F3F001B3F09001B3F21
:101CB0003F03070707040A04072E1313132D2E03EF
:101CC000073F3F373F3F3F24043F3F3F3F3F3F3FBA
:101CD0002D2D2E2E2E2E363F3F2D2D2D2D2D252414
:101CE000373F3F3F3F3F3F37363F3F3F3F3F3F3F1D
:101CF0002507070707030000000707070601000084
:101D00000006060602000000001C0A000000000099
:101D1000003709000000000000250000000000005E
:101D200000090000000000000000000000000000AA
:101D30000900253F000000002D001B3712000000A5
:101D4000360009372500001B3F0000242E00003616
:101D50002E000000361C2D2D090000001237360021
:101D6000000000000013120000000000000000004E
:101D7000003F3F3F3F3F3F3F3F3F3F3F3F3F3F3FB2
:101D80003F37241B243F3F3F3F0A0000002D3F3FC9
:101D90002D000000002D3F250000000000373F36D9
:101DA0002D000000243F3F3F37000009363736241E
:101DB000123F3F371B00000A243F3F1B0000123632
:101DC000253612000012372E090900001B372E0994
:101DD00000000A2D372D000000373F2E12000000B2
:101DE000002E1B00000000000000000000000000AA
:101DF0000000000000C9C9C9C900000000000000BF
:101E000000000000000000000000000000C9C9C977
:101E1000C9000000000000000000000000000000F9
:101E200000000000000000000000000000000000B2
:101E300000C90000C900000000C90000C90000007E
:101E400000C90000C900000000C90000C90000006E
:101E500000C90000C9C9C9C9C9C900000000000003
:101E600000C900000000000000C9C9C9C9C9C9C92A
:101E7000C900000000C90000C900000000C900003E
:101E8000C900000000C90000C900000000C900002E
:101E9000C9C9C9C9C9C90000C900000000000000C3
:101EA000C900000000000000C9C9C9C9C9C9C9C921
:101EB000C9C9C9C9C9000000000000000000000035
:101EC000000000000000000000C9C9C9C9000000EE
:101ED0000000000000000000000000000000000002
:101EE00000000000000000000000000000000000F2
:101EF0000000002D2D0000363F0000093F25001B8B
:101F00003F000000133736243F000000001B3F3F16
:101F10003F00000000001B3F3F00000000000012D7
:101F20002D00000000000000000000000000000084
:101F3000003F3F3F3F3F3F3F123F362D373F3F3F40
:101F40000037000009363F2E002D00000012372D0B
:101F5000002D00000000252D0036000000000A378B
:101F600000090000000001362D00000000000025DF
:101F700024000000000009242400000000092D2591
:101F80000900000012362D0A00000012362E120041
:101F90000000093736120000001237360900000031
:101FA000002E250900000000000A000000000000CB
:101FB00000EBEBEBEBEBEBEBEBEB000000000000DE
:101FC000EBEB00EBEBEBEB00EBEB00EB0000EB00E3
:101FD000EBEB00EB0000EB00EBEB00EB0000EB00A9
:101FE000EBEB00EB0000EB00EBEB00EB0000EB0099
:101FF000EBC9C9C9C9C9C90000000000000000C977
:102000000000000000000000C90000000000000007
:10201000C900000000000000C9000000000000002E
:10202000C900000000000000C9C900000000000055
:10203000C90000C9C9C9C9C9C900C9000000000058
:1020400000C900000000000000C9000000000000FE
:1020500000C900000000000000C9000000000000EE
:1020600000C900000000000000C9000000000000DE
:10207000C9EB00EB0000EB00EB0000EB0000EB0015
:10208000EBEBEBEB0000EB00EB0000000000EB00E3
:10209000EB0000000000EB00EBEBEBEBEBEBEB00FD
:1020A000EB00000000000000EBEBEBEBEBEBEBEBED
:1020B000EBEB00EB0000EB00EBEB00EB0000EB00C8
:1020C00000EB00EB0000EBEBEBEB00EB00000000A3
:1020D00000EB00EB0000000000EB00EBEBEBEBEBA8
:1020E000EBEB00000000000000EBEBEBEBEBEBEBAD
:1020F000EB00000000C90000C900000000C900009A
:102100000000000000C900000000000000C900003D
:102110000000000000C900000000000000C900002D
:102120000000000000C900000000000000C900001D
:10213000C9C90000C900000000000000C90000007B
:1021400000000000C900000000000000C9000000FD
:1021500000000000C900000000000000C9000000ED
:1021600000000000C900000000C90000C900000014
:1021700000EBEBEBEBEBEBEBEBEB252E2E2E2E2E11
:102180002EEB2E373737373737EB2E373737373792
:1021900037EB2E373737373737EB2E373737373779
:1021A00037EB2E373737373737EB2E373737373769
:1021B00037EBEBEBEBEBEBEBEB2E2E2E2E2E2E2E4E
:1021C0002E37373737373737370000000000000029
:1021D000000000000000000000373737373737377E
:1021E000373737373737373737373737373737377F
:1021F00037EBEBEBEBEBEBEBEB2E2E2E2E2E2E2517
:10220000EB3737373737372EEB3737373737372E08
:10221000EB3737373737372EEB3737373737372EF8
:10222000EB3737373737372EEB3737373737372EE8
:10223000EBEB2E373737370037EB2E37373737375B
:1022400037EB2E373737370037EB2E3737373737FF
:1022500037EB2E373737373737EB2E3737373737B8
:1022600037EB2E373737373737EB2E3737373737A8
:1022700037000000000000000037373737373737A6
:1022800037000000003737373737373737373737BA
:10229000370000000000000037373737373737374F
:1022A0003700000000000000003737373737373776
:1022B000373737373737372EEB3737373737372E0C
:1022C000EB3737373737372EEB3737373737372E48
:1022D000EB3737373737372EEB3737373737372E38
:1022E000EB3737373737372EEB3737373737372E28
:1022F000EBC9000000000000C90000000000000061
:1023000000000000000000000000000000000000CD
:1023100000000000000000000000000000000000BD
:10232000000000000000000000C9C9C9C9C9C9C92E
:10233000C93737373737376F6F373737376F6F6F83
:10234000373707076F37376F3707076F07376F372D
:1023500037070707FF076F073707FF070707070755
:102360000737070737FF0707073737373707FF07ED
:1023700037373737373737393737373737273939F7
:1023800039376F6F2727276F376F6F6F6F276F6F23
:102390006F6F6F6F6F6F6F6F6F6F6F6F6F6F6F6F4D
:1023A0006F376F6F6F6F6F6F3737376F6F6F6F3755
:1023B0003737EFEF37372F2F37F7EFEFF7B72F2FED
:1023C000B7EFEFEFEF2F2F2F2F373737373737375D
:1023D0003737373737373737373707073737F2F277
:1023E000371F07071FACF2F2AC07070707F2F2F23C
:1023F000F237373737371F1F373737371F1F1F1F42
:102400003737371FFFFF1F1F3737371FFF1F1F1FAC
:1024100037371F1F1F1F1F1F371F1D1D1D1F1F1F8A
:102420001F371F1D1F1D1D1F1F3737371F1F1D1F64
:1024300037EB2E373737373737EB2E3737373737D6
:1024400037EB2E373737373737EB2E3737373737C6
:1024500037EB2E373737373737EB2E3737373737B6
:1024600037EB252E2E2E2E2E2EEBEBEBEBEBEBEBA4
:10247000EB37373737373737373737373737373738
:1024800037373737373737373737373737373737DC
:1024900037373737373737373737373737373737CC
:1024A000372E2E2E2E2E2E2E2EEBEBEBEBEBEBEB18
:1024B000EB3737373737372EEB3737373737372E56
:1024C000EB3737373737372EEB3737373737372E46
:1024D000EB3737373737372EEB3737373737372E36
:1024E000EB2E2E2E2E2E2E25EBEBEBEBEBEBEBEB70
:1024F000EB00000000EBEBEBEB00000000EB00005A
:102500000000000000EB00EBEB00000000EB00EB34
:102510000000000000EB00EB0000000000EB00EB0F
:102520000000000000EB00EB0000000000EB00EBFF
:1025300000EBEBEBEBEBEBEBEB0000000000000043
:1025400000EBEBEBEBEBEBEBEB0000000000000033
:10255000000000000000000000000000000000007B
:10256000000000000000000000000000000000006B
:1025700000EBEBEBEB0000000000000000000000AF
:1025800000EBEBEBEB00000000000000000000009F
:10259000000000000000000000000000000000003B
:1025A0000700000000000007070000000000070708
:1025B0000700000000000000000000000707000006
:1025C00000000007070707000000070707070707C5
:1025D0000007070707070707070707070707070792
:1025E000070707070707070707070707070707077B
:1025F0000700000000EBEBEBEB0000000000000028
:102600000000000000EBEBEBEB000000000000001E
:1026100000000000000000000007000000000000B3
:102620000007070000000000000707070000000087
:1026300000EBEBEBEB00000000000000EB00000003
:1026400000EBEB00EB0000000000EB00EB000000F3
:102650000000EB00EB0000000000EB00EB000000CE
:102660000000EB00EB0000000000EB00EB000000BE
:1026700000EBEBEBE3529AEBA3A3EBEBEB51A309DB
:102680003FA2EBEBEBE3521B2D519AEBEBEB093F37
:102690003F4B099AEBEB093F3F070509A3EB113FBD
:1026A0003F0707059AEB522D3F07070703A3511B6E
:1026B00025EBEB499AEB5A5100120951E3EBA39A2F
:1026C0000009BFA35A1252520009005224120009F5
:1026D000000909133F00BF09003F253637120000EB
:1026E000002D123F3F3F0900001B253F2D52510096
:1026F00000EBEBEBE3529AEBA3A3EBEBEB51A3095B
:102700002DA2EBEBEBE3521B2D519AEBEBEB093FC8
:102710003F4B099AEBEB093F3F070509A3EB113F3C
:10272000090707059AEB522D0907070703A3511B59
:1027300025EBEB499AEB5A5100120951E3EBA39AAE
:10274000003F2DA35A125252003F3F52241200095B
:10275000000912133F37130900BF25363700130055
:102760000000123F00BF0900001B253F120051006E
:102770000000000000000000000000000000000059
:102780000000000000000000000000000000000049
:102790000000000000000000090000000000000828
:1027A000A20000000000000025000000000000BFA3
:1027B00013000000000051002D0000000051002D0A
:1027C0003F0000000051003F3F0000005AA31B3FA4
:1027D0003F000052A29A122D2E00495A529AA25B33
:1027E00052009A04060B5252A3514A0707070707E3
:1027F000042424009A1152E39A241BBF0037129A32
:102800009A1B0A001B3F129A510A2D3F3F3F09A312
:10281000E31B3F3F3F099AEBEB1B3636129AEBEB7B
:10282000A3A35B115AEBE35A09539AA39A520305E7
:10283000070000000000253F3F0000000000133F9C
:102840003F000000000000253F0000005A00BF09C3
:102850003F000052A25100132E00495A529AA25B27
:1028600052009A04060B5252A3514A070707070762
:1028700004249AA3521152E39A24491B2D37129A29
:102880009A1B1B3F3F3F129A5124001B3F3F09A355
:10289000E31BBF093F099AEBEB0A001B129AEBEB13
:1028A000A3A35B115AEBE35A09539AA39A52030567
:1028B0000700000000122D373F0000001B373F3F8C
:1028C0003F02040400123F3F3F070702F702362D84
:1028D0000B07070400041203070707070703020793
:1028E000070707070702030707070707070203078A
:1028F00007372E1B00000000003F3F3F2E12000054
:10290000003F3F3F3F370A00000204001B3F3609EB
:10291000000702F71B372E1B0007030001252D2D92
:1029200000070702031B2E3609070707041B36366C
:102930000A00000000122D373F0000001B373F3F08
:102940003F0204040A2E3F3F3F070707070A362DC0
:102950000B070707070A1203070707070403020705
:10296000070707040012030707070702F702030718
:1029700007372E1B00000000003F3F3F2E120000D3
:10298000003F3F3F3F370A000002031C373F360934
:102990000007070513372E1B0007070700252D2DFD
:1029A000000707040A252E36090704001B253636C2
:1029B0000A06070400030307071B1313253F24041B
:1029C000073F373F3F3F37240B3F3F3F3F3F3F3FAE
:1029D0003737252425373F3F3F3737372D1B2D37D6
:1029E0003F3F3F3F3F37251B243F3F3F3F3F3F3F58
:1029F0002E0702F71B243637090703001B3736362C
:102A000009040313363F372E002E36372E3F3F245E
:102A1000003F3F3612363709003F371B253F240061
:102A2000002513243F370000002D363F37120000E9
:102A3000001C363F3F362512001B1B3F3F3F3F37F0
:102A40002D09031B1B363F3F3FF703070603243FB7
:102A50003F0006070707042E0905070707070609B1
:102A60000907070707070609040707070707030001
:102A70000700000000000000000900000000000046
:102A8000002D0000000000000024240000000000D1
:102A9000000105000000000000F70206020000002F
:102AA00000020707070200000007070707030000EE
:102AB00000070707070300000007070706010000DB
:102AC0000006060602000000001C0A0000000000CC
:102AD0000037090000000000002500000000000091
:102AE00000090000000000000000000000000000DD
:102AF000001C363F3F362512003F3F3F3F3F3F37E8
:102B00002D37241B1B363F3F3F1306070603243F88
:102B10003F0907070707042E2D06070707070609C1
:102B2000010506070707060905090307070703004C
:102B3000020000000000000000090000000000008A
:102B4000002D000000000000003F240000000000F5
:102B500000360B0000000000000507060200000020
:102B60000007070707020000000707070703000028
:102B700000F7030507040A0901000313132D2E09AA
:102B8000F73F3F373F3F3F00023F3F3F3F3F3F3F21
:102B90002D2D2E2E2E2E363F3F2D2D2D2D2D252445
:102BA000373F3F3F3F3F3F37363F3F3F3F3F3F3F4E
:102BB00025030707070300000002070706010000BE
:102BC0000003060602000000001C0A0000000000CE
:102BD0000037090000000000002500000000000090
:102BE00000090000000000000000000000000000DC
:102BF00000003F3F3F3F0000003F3F3F3F3F3F3F20
:102C00000000003F3F3F3F3F00000000003F3F3FCC
:102C10003F000000003F3F3F3F00003F3F3F3F3F3E
:102C2000003F3F3F3F3F3F3F00003F3F3F3F0000EF
:102C3000000000000000000000003F3F3F3F2E006A
:102C400000003F2E00003F2E00003F2E00003F2ED0
:102C500000003F3F3F3F3F2E00003F3F3F3F2E00E1
:102C600000003F2E003F3F2E00000000000000004B
:102C70000000000000000000003F3F3F3F3F2E00EB
:102C80003F3F2E000000003F3F3F3F3F3F2E003FB1
:102C90002E3F3F3F3F2E003F3F3F2E000000003FB2
:102CA0002E3F3F3F3F3F2E3F2E0000000000000020
:102CB0000000000000000000003F3F2E00003F3FEA
:102CC0003F2E3F3F2E003F2E0000003F2E003F2EA4
:102CD000003F3F3F2E003F2E0000003F2E003F2EC2
:102CE0000000003F2E003F3F3F00000000000000BA
:102CF0000000000000000000002E0000003F2E0930
:102D00003F3F2E00003F2E093F003F2E003F2E2E5A
:102D10003F003F2E00003F3F2E3F2E0000003F3F70
:102D20002E2E000000003F3F2E000000000000009B
:102D30000000000000000000002E0000003F3F2EB9
:102D4000002E0000003F3F2E002E00003F3F2E00CF
:102D5000000000003F2E0000000000002E000000D8
:102D60000000003F00000000000000000000000024
:102D70000000000000000000000000070707075FD8
:102D80000000075F000000000700075F0000000070
:102D90000700075F0007075F070007075F00075F7F
:102DA0000700000707075F000700000000000000A1
:102DB0000000000000000000000707075F00000798
:102DC00007075F07075F0707075F0000075F075FE9
:102DD00007070707075F075F005F0000075F075FE0
:102DE000005F0000075F075F0000000000000000B8
:102DF0000000000000000000005F07075F000707F9
:102E0000075F0707075F075F0007075F075F0707A1
:102E100007075F00075F070707000000075F075FFE
:102E200000000000075F0707070000000000000027
:102E3000000000000000000000075F00000000002C
:102E400007000000000000075F5F000000000007AF
:102E50005F5F0000000000075F0000000000000747
:102E60005F075F0000000000070000000000000096
:102E700000000000000000000007075F00075F007F
:102E8000000000075F00075F000000075F00070702
:102E9000000000075F0000075F0000075F000007F9
:102EA0000707075F000000000700000000000000A7
:102EB0000000000000000000000000075F07070797
:102EC0000700075F00075F000000075F00070707B4
:102ED0005F075F00000707075F075F0000075F00ED
:102EE000005F000000070707070000000000000067
:102EF0000000000000000000005F070707075F00F8
:102F00000000075F0000075F0000075F0000075F29
:102F1000000007070707075F0000070707075F00B4
:102F2000005F075F0000075F000000000000000076
:102F300000000000000000000000FAFAFAFAEB00BE
:102F4000FA00FAEB0000FAEBFA00FAEB0000FAEBF9
:102F5000FA00FAFAFAFAEB00FA00FAEB00000000C5
:102F6000FA00FAEB00000000FA0000000000000088
:102F7000000000000000000000EB00000000FAFA72
:102F8000FAEB000000FAFAEBFAEB000000FAEB00B3
:102F900000EB000000FAFAFAFAEB000000FAEB008E
:102FA00000FAFAFAEBFAEB00000000000000000063
:102FB000000000000000000000EB00FAEB00FAEB5C
:102FC000FAFAEBFAEB00FAEBFAFAEBFAEBEBFAEBC4
:102FD000FAFAEB00FAFAEB00FAFAEB00FAFAEB0075
:102FE000FAFAEB00FAFAEB00FA0000000000000029
:102FF000000000000000000000FAFAFAEBFAFAFA0A
:10300000FAEB000000FAEB0000FAFAEB00FAEB0032
:1030100000FAFAEB00FAFAFAFAEB000000FAFAFA10
:10302000FAFAFAFAEBFAEB000000000000000000E8
:10303000000000000000000000EB000000000000A5
:10304000FAFAEB00000000FAEBFAEB00000000FADD
:10305000EBFAEB00000000FAEBEB0000000000FAD6
:10306000EBFAEB0000000000FA0000000000000096
:10307000000000000000000000FAFAEB00FAFAEB92
:10308000000000FAEBFAFAFAEB0000FAEBFAEBFABE
:10309000FA0000FAEBFAEB00FA0000FAEBFAEB00A8
:1030A000FAFAFAEB00FAEB00000000000000000062
:1030B000000000000000000000FAEBFAFAFAFAEB58
:1030C00000FAEBFAEB00000000FAEBFAFAFAEB0078
:1030D00000FAEBFAFAFAEB0000FAEBFAF300000060
:1030E00000FAEBFAFAFAFAEB000000000000000028
:1030F00000000000000000000000000000000000D0
:1031000000000000000000000000000000000000BF
:10311000000000000000000000000000000000A40B
:10312000A40000000000A400000000000000A400B3
:10313000A4000000000000000000000000000000EB
:10314000000000000000000000000000000000007F
:1031500000A4A4A4A4A4A4A4A4000000000000004F
:10316000000000000000000000A4A4A4A4A4A4A4E3
:10317000A4000000000000000000000000000000AB
:10318000000000000000000000000000000000003F
:1031900000A4A4A4A4A4A4A4A4000000000000000F
:1031A000000000000000000000A40000000000007B
:1031B000A40000000000000000000000000000006B
:1031C00000000000000000000000000000000000FF
:1031D000000000000000000000A4A40000000000A7
:1031E000000000A40000000000A400A400000000F3
:1031F0000000000000A40000A400000000A40000E3
:10320000A400000000A40000A400000000A400002E
:10321000A400000000A40000A400000000A400001E
:10322000A400000000A40000A400000000A400000E
:10323000A4A4000000000000A4A4000000000000FE
:10324000A4A4000000000000A4A4000000000000EE
:10325000A4A4000000000000A4A4000000000000DE
:10326000A4A4000000000000A4A4000000000000CE
:10327000A4A40000A400000000A40000A40000001A
:1032800000A40000A400000000A40000A4000000AE
:1032900000A40000A400000000A40000A40000009E
:1032A00000A40000A400000000A40000A40000008E
:1032B000000000A4A4A4A4A4A400A4000000000092
:1032C00000A400000000000000A4000000000000B6
:1032D00000A400000000000000A4000000000000A6
:1032E00000A400000000000000A400000000000096
:1032F00000A4A4A4A4A4A40000000000000000A452
:103300000000000000000000A40000000000000019
:10331000A400000000000000A40000000000000065
:10332000A400000000000000A40000000000000055
:10333000A4A4A4A4A4A4A4A4A400000000000000C9
:10334000000000000000000000000000000000007D
:10335000000000000000000000000000000000006D
:10336000000000000000000000000000000000005D
:1033700000A400000000000000A400000000000005
:1033800000A400000000000000A4000000000000F5
:1033900000A400000000000000A4000000000000E5
:1033A0000000A40000000000000000A4A4A4A4A445
:1033B000A400000000000000A400000000000000C5
:1033C000A400000000000000A400000000000000B5
:1033D000A400000000000000A400000000000000A5
:1033E000A4000000000000A400A4A4A4A4A4A400BD
:1033F00000000000000000000000000000000000CD
:1034000000000000000000000000000000000000BC
:1034100000000000000000000000000000000000AC
:10342000000000000000000000A4A4A4A4A4A4A420
:10343000A4A4000000000000A4A4000000000000FC
:10344000A4A4000000000000A4A4000000000000EC
:10345000A4A4000000000000A4A4000000000000DC
:10346000A400A400000000A4000000A4A4A4A400E0
:10347000000000A4A4A4A4A4A400A40000000000D0
:1034800000A400000000000000A4000000000000F4
:1034900000A400000000000000A4000000000000E4
:1034A0000000A40000000000000000A4A4A4A4A444
:1034B000A4A4A4A4A4A4A40000000000000000A4EC
:1034C0000000000000000000A40000000000000058
:1034D000A400000000000000A400000000000000A4
:1034E000A4000000000000A400A4A4A4A4A4A400BC
:1034F000000000A4A4A4A4000000A400000000A4F4
:1035000000A4000000000000A4A4000000000000CF
:10351000A4A4000000000000A4A40000000000001B
:10352000A4A4000000000000A4A40000000000000B
:10353000A4A4A4A4A4A4A4A4A400000000000000C7
:10354000000000000000000000000000000000007B
:10355000000000000000000000000000000000006B
:10356000000000000000000000A4A4A4A4A4A4A4DF
:10357000A4A4A4A4A4A4A4A4A40000000000000087
:10358000000000000000000000000000000000003B
:10359000000000000000000000000000000000002B
:1035A000000000000000000000A400000000000077
:1035B000A40000000000A400A40000000000A4007B
:1035C00000000000000000A4A400000000000000B3
:1035D00000000000000000000000000000000000EB
:1035E00000000000000000000000000000000000DB
:1035F00000A4A4A4A4A4A4A4A400000000000000AB
:10360000000000000000000000A4A4A4A4A4A4A43E
:10361000A400000000000000000000000000000006
:10362000000000000000000000000000000000009A
:1036300000A4A4A4A4A4A40000000000000000A40E
:103640000000000000000000A4A4A4A4A400000046
:10365000A400000000A40000A400000000A40000DA
:10366000A400000000A40000A400000000A40000CA
:10367000A4A4000000000000A4A4000000000000BA
:1036800000A400000000000000A4000000000000F2
:1036900000A400000000000000A4000000000000E2
:1036A00000A400000000000000A4000000000000D2
:1036B000A4A4000000000000A4000000000000001E
:1036C000A400000000000000A400000000000000B2
:1036D000A400000000000000A400000000000000A2
:1036E000A400000000000000A4A4000000000000EE
:1036F000A40000A4A4A4A4A4A400A40000000000AA
:1037000000A400000000000000A4000000A4A4A485
:10371000A4A40000A400000000A40000A400000075
:1037200000A40000A400000000A40000A400000009
:1037300000A400A400000000000000A4000000009D
:1037400000A4A40000000000000000000000000031
:103750000000000000000000000000000000000069
:103760000000000000000000000000000000000059
:103770000000000000000000000000000000000049
:103780000000000000000000000000000000000039
:103790000000000000A4A4A4A40000000000000099
:1037A00000000000000000000000000000A4A4A42D
:1037B000A400000000A40000A400000000A4000079
:1037C000A400000000A40000A400000000A4000069
:1037D000A4A4A4A4A4000000A40000000000000011
:1037E000A4000000000000A400A4A4A4A4A4A400B9
:1037F00000A40000A400000000A40000A400000039
:1038000000A40000A400000000A40000A400000028
:1038100000A4000000A4A4A4A4A4000000000000D0
:103820000000A40000000000000000A4A4A4A4A4C0
:10383000A4000000000000000000000000000000E4
:103840000000000000000000000000000000000078
:1038500000A4A4A4A40000000000000000000000D8
:10386000000000000000000000A4A4A4A4000000C8
:103870000000000000A4A4A4A400000000000000B8
:1038800000000000000000000000000000A4A4A44C
:10389000A400000000000000000000000000000084
:1038A0000000000000000000000000000000000018
:1038B00000A4A4A4A4000000000000000000000078
:1038C000000000000000000000A4A4A4A400000068
:1038D00000000000000000000000000000000000E8
:1038E00000000000000000000000000000000000D8
:1038F00000A4A4A4A4A4A40000000000000000A44C
:103900000000000000000000A40000000000000013
:10391000A400000000000000A4000000000000005F
:10392000A400000000000000A4A4000000000000AB
:10393000A40000A4A4A4A4A4A400A4000000000067
:1039400000A400000000000000A40000000000002F
:1039500000A400000000000000A40000000000001F
:1039600000A400000000000000A40000000000000F
:10397000A400000000A40000A400000000A40000B7
:103980000000000000A400000000000000A40000EF
:103990000000000000A400000000000000A40000DF
:1039A0000000000000A400000000000000A40000CF
:1039B000A4A40000A400000000000000A400000077
:1039C00000000000A400000000000000A4000000AF
:1039D00000000000A400000000000000A40000009F
:1039E00000000000A400000000A40000A4000000EB
:1039F00000A4000000000000A4000000000000007F
:103A000000000000000000000000000000000000B6
:103A100000000000000000000000000000000000A6
:103A2000000000000000000000A4A4A4A4A4A4A41A
:103A3000A4000000000000000000000000000000E2
:103A40000000000000000000000000000000000076
:103A50000000000000000000000000000000000066
:103A60000000000000000000000000000000000056
:103A7000000000000000006F6F000000006F6F6F1B
:103A8000000007076F00006F0007076F07006F0057
:103A900000070707FF076F070007FF07070707076C
:103AA0000700070700FF07070700000000070707D8
:103AB0000000000000FF00000000393939FF3939EB
:103AC00000070707393907070707FF07070707FF39
:103AD0000707070707FF0707070007FF070707078D
:103AE0000000000707FF07000000000007070000B4
:103AF00000000000000000390000000000273939F4
:103B000039006F6F2727276F006F6F6F6F276F6FF9
:103B10006F6F6F6F6F6F6F6F6F6F6F6F6F6F6F6FB5
:103B20006F006F6F6F6F6F6F0000006F6F6F6F00D0
:103B300000000000006F0000000707006F0007078B
:103B4000000707076F0707070707070707070707A4
:103B500007070707070707FF070707070707FF0705
:103B6000070007070707070700000007000707000F
:103B7000000000B1B1B1B10000000000B1000000D0
:103B800000000039FF39390000003939B1393939BD
:103B9000003939393939FFB13939FFB13939393952
:103BA0003900393939FFB139000000B139393900EC
:103BB000000000001F1F0000001F00001F1F00006A
:103BC0001F1F001F1F1F1F001F1F1F1F1F1F1F1F43
:103BD0001F1F1F001F1F001F1F001F001F1F001F90
:103BE000000000001F1F0000000000001F1F000059
:103BF0000000000000001F1F000000001F1F1F1F0B
:103C00000000001FFFFF1F1F0000001FFF1F1F1FDE
:103C100000001F1F1F1F1F1F001F1D1D1D1F1F1F17
:103C20001F001F1D1F1D1D1F1F0000001F1F1D1F28
:103C3000000000CACACA00000000CACA00CACA00FE
:103C40000000CACACACACA00000000CA00CA0000EE
:103C50000000CACA00CA0000000000CA00CA000072
:103C60000000CACA00CA000000000000CA0000002C
:103C70000000000707070700000007FF0707FF070E
:103C80000000FFFFFFFFFFFF0000FFFFC9FFFFC9AC
:103C9000000707FFC907FFC9070707070707070747
:103CA000EF0707070707EFEFEF000700070700EF31
:103CB0000000000707070700000007FF0707FF07CE
:103CC0000000FFC9FFFFC9FF0000FFC9FFFFC9FFD8
:103CD000000707FF0707FF0707070707070707078B
:103CE000EF0707070707EFEFEF000700070700EFF1
:103CF00000000000000000000000000000000000C4
:103D000000000000000000000000000000000000B3
:103D10000000000000000000000000000707070787
:103D20000700000000070707070000000000000070
:103D3000070000000000000000000000000000007C
:103D40000000000000000000000000000000000073
:103D50000000000000000000000000000000000063
:103D60000007070000000000000707070000000030
:103D70000000000000000000000000000000000043
:103D80000000000000000000000000000000000033
:103D90000000000000000000000000000000000023
:103DA00000000707000000000007070707070000E2
:103DB0000000000707070700000007FF0707FF07CD
:103DC0000000FFFFC9FFFFC90000FFFFC9FFFFC9D7
:103DD000000707FF0707FF0707070707070707078A
:103DE000070707070707070707070007000007007F
:103DF000070000EFEFEFEF000000EFFFEFEFFFEF46
:103E00000000FFFFC9FFFFC90000FFFFC9FFFFC996
:103E100000EFEFFFEFEFFFEFEFEFEFEFEFEFEFEF81
:103E2000EFEFEFEFEFEFEFEFEFEF00EF0000EF005E
:103E3000EF0000F2F2F2F2000000F2FFF2F2FFF205
:103E40000000FFFFC9FFFFC90000FFFFC9FFFFC956
:103E500000F2F2FFF2F2FFF2F2F2F2F2F2F2F2F21A
:103E6000F2F2F2F2F2F2F2F2F2F200F20000F200FA
:103E7000F200002F2F2F2F0000002FFF2F2FFF2FDA
:103E80000000FFFFC9FFFFC90000FFFFC9FFFFC916
:103E9000002F2FFF2F2FFF2F2F2F2F2F2F2F2F2FC1
:103EA0002F2F2F2F2F2F2F2F2F2F002F00002F00DE
:103EB0002F0000FFFFFF00000000FF0000FFFF00D9
:103EC00000FFFF000000FFFF00FFFF000000FFFFFA
:103ED00000FFFF000000FFFF0000FFFF0000FF00E9
:103EE000000000FFFFFF00000000000000000000D5
:103EF00000000000FFFF0000000000FFFFFF0000C7
:103F000000000000FFFF000000000000FFFF0000B5
:103F100000000000FFFF000000000000FFFF0000A5
:103F20000000FFFFFFFFFFFF000000000000000097
:103F30000000FFFFFFFFFF0000FFFF000000FFFF8A
:103F40000000000000FFFFFF000000FFFFFFFF0078
:103F50000000FFFFFFFF000000FFFFFF0000000068
:103F600000FFFFFFFFFFFFFF000000000000000058
:103F70000000FFFFFFFFFFFF0000000000FFFF0049
:103F800000000000FFFF0000000000FFFFFFFF0037
:103F9000000000000000FFFF00FFFF000000FFFF27
:103FA0000000FFFFFFFFFF00000000000000000016
:103FB00000000000FFFFFF00000000FFFFFFFF0008
:103FC0000000FFFF00FFFF0000FFFF0000FFFF00F9
:103FD00000FFFFFFFFFFFFFF0000000000FFFF00EA
:103FE0000000000000FFFF000000000000000000D3
:103FF00000FFFFFFFFFFFF0000FFFF0000000000C9
:1040000000FFFFFFFFFFFF00000000000000FFFFB8
:10401000000000000000FFFF00FFFF000000FFFFA6
:104020000000FFFFFFFFFF00000000000000000095
:10403000000000FFFFFFFF000000FFFF0000000086
:1040400000FFFF000000000000FFFFFFFFFFFF0078
:1040500000FFFF000000FFFF00FFFF000000FFFF68
:104060000000FFFFFFFFFF00000000000000000055
:1040700000FFFFFFFFFFFFFF00FFFF000000FFFF4B
:104080000000000000FFFF0000000000FFFF000034
:10409000000000FFFF000000000000FFFF00000024
:1040A000000000FFFF000000000000000000000012
:1040B0000000FFFFFFFF000000FFFF000000FF0007
:1040C00000FFFFFF0000FF000000FFFFFFFF0000F8
:1040D00000FF0000FFFFFFFF00FF00000000FFFFE8
:1040E0000000FFFFFFFFFF000000000000000000D5
:1040F0000000FFFFFFFFFF0000FFFF000000FFFFC9
:1041000000FFFF000000FFFF0000FFFFFFFFFFFFB9
:10411000000000000000FFFF0000000000FFFF00A3
:104120000000FFFFFFFF0000000000000000000093
:10413000000000FFFFFFFF000000FFFF0000FFFF87
:1041400000FFFF000000000000FFFF000000000073
:1041500000FFFF00000000000000FFFF0000FFFF65
:10416000000000FFFFFFFF00000000000000000053
:1041700000FFFFFFFFFFFFFF00FFFF000000000048
:1041800000FFFF000000000000FFFFFFFFFFFF0037
:1041900000FFFF000000000000FFFF000000000023
:1041A00000FFFFFFFFFFFFFF000000000000000016
:1041B000000000FFFFFFFFFF0000FFFF0000000006
:1041C00000FFFF000000000000FFFF0000FFFFFFF6
:1041D00000FFFF000000FFFF0000FFFF0000FFFFE7
:1041E000000000FFFFFFFFFF0000000000000000D4
:1041F00000FFFF000000FFFF00FFFF000000FFFFC7
:1042000000FFFF000000FFFF00FFFFFFFFFFFFFFB9
:1042100000FFFF000000FFFF00FFFF000000FFFFA6
:1042200000FFFF000000FFFF000000000000000092
:104230000000FFFFFFFFFFFF00000000FFFF000086
:1042400000000000FFFF000000000000FFFF000072
:1042500000000000FFFF000000000000FFFF000062
:104260000000FFFFFFFFFFFF000000000000000054
:104270000000FFFFFFFFFF0000FFFF000000FFFF47
:1042800000FFFF000000FFFF00FFFF000000FFFF36
:1042900000FFFF000000FFFF00FFFF000000FFFF26
:1042A0000000FFFFFFFFFF00000000000000000013
:1042B00000FFFFFFFFFFFF0000FFFF000000FFFF08
:1042C00000FFFF000000FFFF00FFFF000000FFFFF6
:1042D00000FFFFFFFFFFFF0000FFFF0000000000E6
:1042E00000FFFF00000000000000000000000000D0
:1042F00000FFFFFFFFFFFF0000FFFF000000FFFFC8
:1043000000FFFF000000FFFF00FFFF0000FFFFFFB6
:1043100000FFFFFFFFFF000000FFFF00FFFFFF00A7
:1043200000FFFF0000FFFFFF000000000000000092
:104330000000FFFFFFFF000000FFFF0000FFFF0085
:1043400000FFFF00000000000000FFFFFFFFFF0074
:10435000000000000000FFFF00FFFF000000FFFF63
:104360000000FFFFFFFFFF00000000000000000052
:1043700000FFFF000000FFFF00FFFF000000FFFF45
:1043800000FFFF000000FFFF00FFFF000000FFFF35
:1043900000FFFF000000FFFF00FFFF000000FFFF25
:1043A0000000FFFFFFFFFF00000000000000000012
:1043B000000000FFFFFF00000000FFFF00FFFF0004
:1043C00000FFFF000000FFFF00FFFF000000FFFFF5
:1043D00000FFFFFFFFFFFFFF00FFFF000000FFFFE8
:1043E00000FFFF000000FFFF0000000000000000D1
:1043F00000FFFFFFFFFF000000FFFF0000FFFF00C6
:1044000000FFFF000000FFFF00FFFF000000FFFFB4
:1044100000FFFF000000FFFF00FFFF0000FFFF00A4
:1044200000FFFFFFFFFF0000000000000000000091
:1044300000FFFF000000FFFF00FFFF0000FFFF0084
:1044400000FFFF00FFFF000000FFFFFFFF00000074
:1044500000FFFFFFFFFF000000FFFF00FFFFFF0066
:1044600000FFFF0000FFFFFF000000000000000051
:1044700000FFFF000000FFFF00FFFFFF00FFFFFF46
:1044800000FFFFFFFFFFFFFF00FFFFFFFFFFFFFF3A
:1044900000FFFF00FF00FFFF00FFFF000000FFFF25
:1044A00000FFFF000000FFFF000000000000000010
:1044B00000FFFF000000FFFF00FFFFFF0000FFFF05
:1044C00000FFFFFFFF00FFFF00FFFFFFFFFFFFFFF9
:1044D00000FFFF00FFFFFFFF00FFFF0000FFFFFFE7
:1044E00000FFFF000000FFFF0000000000000000D0
:1044F0000000FFFFFFFFFFFF00000000FFFF0000C4
:1045000000000000FFFF000000000000FFFF0000AF
:1045100000000000FFFF000000000000FFFF00009F
:1045200000000000FFFF000000000000000000008D
:10453000000000070007000000000007000700005F
:10454000000000070007000000000000000000005D
:10455000000000000000000000000000000000005B
:10456000000000000000000000000000000000004B
:10457000000000000000000000000000000000003B
:104580000000000000000000000007070707070008
:10459000000000000000000000000000000000001B
:1045A000000000000000000000000000000000000B
:1045B00000000007070700000000070700070700CA
:1045C00000070700000007070007070000000707B3
:1045D000000707070707070700070700000007078E
:1045E00000070700000007070000000000000000AF
:1045F0000007070707070700000707000000070775
:104600000007070000000707000707070707070064
:104610000007070000000707000707000000070762
:104620000007070707070700000000000000000060
:10463000000707070707000000070700000707003B
:104640000007070000000707000707000000070732
:104650000007070000000707000707000007070022
:104660000007070707070000000000000000000027
:104670000007070000000707000707000000070702
:1046800000070700000007070007070707070707DD
:1046900000070700000007070007070000000707E2
:1046A00000070700000007070000000000000000EE
:1046B00000000707070707070000000007070000C2
:1046C00000000000070700000000000007070000CE
:1046D00000000000070700000000000007070000BE
:1046E00000000707070707070000000000000000A0
:1046F0000007070000000707000707000007070082
:104700000007070007070000000707070700000071
:104710000007070707070000000707000707070053
:104720000007070000070707000000000000000066
:10473000000007070000000000000707000000005D
:10474000000007070000000000000707000000004D
:10475000000007070000000000000707000000003D
:10476000000007070707070700000000000000001F
:1047700000070700000007070007070700000707FA
:1047800000070707070007070007070707070707CE
:1047900000070700070707070007070000070707CC
:1047A00000070700000007070000000000000000ED
:1047B00000000707070707000007070000000707BA
:1047C00000070700000007070007070000000707B1
:1047D00000070700000007070007070000000707A1
:1047E00000000707070707000000000000000000A6
:1047F0000000070707070000000707000007070081
:104800000007070000000000000007070707070077
:10481000000000000000070700070700000007076E
:104820000000070707070700000000000000000065
:104830000007070000000707000707000000070740
:104840000007070007000707000707070707070714
:1048500000070707070707070007070700070707FD
:10486000000707000000070700000000000000002C
:104870000000070700000707000007070000070700
:1048800000000707000007070000000707070700F0
:1048900000000000070700000000000007070000FC
:1048A00000000000070700000000000000000000FA
:1048B000000000EF00EF0000000000EF00EF00003C
:1048C000000000EF00EF000000000000000000000A
:1048D00000000000000000000000000000000000D8
:1048E00000000000000000000000000000000000C8
:1048F00000000000000000000000000000000000B8
:1049000000000000000000000000EFEFEFEFEF00FC
:104910000000000000000000000000000000000097
:104920000000000000000000000000000000000087
:104930000000000000000000000000000000000077
:104940000000000000000000000000000000000067
:104950000000000000000000000000EFEF00000079
:10496000000000EFEF000000000000000000000069
:10497000000000EFEFEFEF000000EF00000000EF9D
:1049800000EF0000EFEF0000EFEF00EF000000008D
:10499000EFEF00EF00000000EFEF0000EFEF00008E
:1049A000EF00EF00000000EF000000EFEFEFEF007E
:1049B000000000EFEFEF00000000EF0000EFEF005D
:1049C00000EFEF000000EFEF00EFEF000000EFEF6F
:1049D00000EFEF000000EFEF0000EFEF0000EF004E
:1049E000000000EFEFEF00000000000000000000FA
:1049F00000000000EFEF0000000000EFEFEF00000C
:104A000000000000EFEF000000000000EFEF0000EA
:104A100000000000EFEF000000000000EFEF0000DA
:104A20000000EFEFEFEFEFEF0000000000000000EC
:104A30000000EFEFEFEF000000EFEF000000EF00ED
:104A400000EFEFEF0000EF000000EFEFEFEF0000EE
:104A500000EF0000EFEFEFEF00EF00000000EFEFDE
:104A60000000EFEFEFEFEF0000000000000000009B
:104A70000000EFEFEFEFEF0000EFEF000000EFEFCF
:104A800000EFEF000000EFEF0000EFEFEFEFEFEFD0
:104A9000000000000000EFEF0000000000EFEF005A
:104AA0000000EFEFEFEF000000000000000000004A
:104AB000000000EFEFEF00000000EFEF00EFEF006D
:104AC00000EFEF000000EFEF00EFEF000000EFEF6E
:104AD00000EFEFEFEFEFEFEF00EFEF000000EFEF91
:104AE00000EFEF000000EFEF00000000000000000A
:104AF000000000EFEFEFEF000000EFEF0000EFEF3E
:104B000000EFEF000000000000EFEF0000000000E9
:104B100000EFEF00000000000000EFEF0000EFEFFB
:104B2000000000EFEFEFEF000000000000000000C9
:104B300000EFEFEFEFEF000000EFEF0000EFEF000E
:104B400000EFEF000000EFEF00EFEF000000EFEFED
:104B500000EFEF000000EFEF00EFEF0000EFEF00DD
:104B600000EFEFEFEFEF000000000000000000009A
:104B700000EFEFEFEFEFEFEF00EFEF0000000000CE
:104B800000EFEF000000000000EFEFEFEFEFEF00AD
:104B900000EFEF000000000000EFEF000000000059
:104BA00000EFEFEFEFEFEFEF00000000000000007C
:104BB00000EFEFEFEFEFEFEF00EFEF00000000008E
:104BC00000EFEF000000000000EFEFEFEFEFEF006D
:104BD00000EFEF000000000000EFEF000000000019
:104BE00000EFEF00000000000000000000000000E7
:104BF000000000EFEFEFEFEF0000EFEF000000002C
:104C000000EFEF000000000000EFEF0000EFEFEF1B
:104C100000EFEF000000EFEF0000EFEF0000EFEF1C
:104C2000000000EFEFEFEFEF0000000000000000D9
:104C30000000EFEFEFEFEFEF00000000EFEF0000FC
:104C400000000000EFEF000000000000EFEF0000A8
:104C500000000000EFEF000000000000EFEF000098
:104C60000000EFEFEFEFEFEF0000000000000000AA
:104C700000EFEF000000EFEF00EFEF0000EFEF00BC
:104C800000EFEF00EFEF000000EFEFEFEF000000AC
:104C900000EFEFEFEFEF000000EFEF00EFEFEF00BE
:104CA00000EFEF0000EFEFEF000000000000000059
:104CB00000EFEF000000EFEF00EFEFEF00EFEFEF9E
:104CC00000EFEFEFEFEFEFEF00EFEFEFEFEFEFEFD2
:104CD00000EFEF00EF00EFEF00EFEF000000EFEF6D
:104CE00000EFEF000000EFEF000000000000000008
:104CF00000EFEF000000EFEF00EFEFEF0000EFEF4D
:104D000000EFEFEFEF00EFEF00EFEFEFEFEFEFEF80
:104D100000EFEF00EFEFEFEF00EFEF0000EFEFEF4E
:104D200000EFEF000000EFEF0000000000000000C7
:104D30000000EFEFEFEFEF0000EFEF000000EFEF0C
:104D400000EFEF000000EFEF00EFEF000000EFEFEB
:104D500000EFEF000000EFEF00EFEF000000EFEFDB
:104D60000000EFEFEFEFEF00000000000000000098
:104D700000EFEFEFEFEFEF0000EFEF000000EFEFDD
:104D800000EFEF000000EFEF00EFEF000000EFEFAB
:104D900000EFEFEFEFEFEF0000EFEF00000000009B
:104DA00000EFEF0000000000000000000000000025
:104DB0000000EFEFEFEF000000EFEF0000EFEF007B
:104DC00000EFEF00000000000000EFEFEFEFEF005A
:104DD000000000000000EFEF00EFEF000000EFEF39
:104DE0000000EFEFEFEFEF00000000000000000018
:104DF00000EFEF000000EFEF00EFEF000000EFEF3B
:104E000000EFEF00EF00EFEF00EFEFEFEFEFEFEF6E
:104E100000EFEFEFEFEFEFEF00EFEFEF00EFEFEF6F
:104E200000EFEF000000EFEF0000000000000000C6
:104E30000000EFEF0000EFEF0000EFEF0000EFEFFA
:104E40000000EFEF0000EFEF000000EFEFEFEF00EA
:104E500000000000EFEF000000000000EFEF000096
:104E600000000000EFEF0000000000000000000064
:104E7000000000F200F20000000000F200F200006A
:104E8000000000F200F2000000000000000000003E
:104E90000000000000000000000000000000000012
:104EA0000000000000000000000000000000000002
:104EB00000000000000000000000000000000000F2
:104EC00000000000000000000000F2F2F2F2F20028
:104ED00000000000000000000000000000000000D2
:104EE00000000000000000000000000000000000C2
:104EF00000000000F2F20000000000F2F2F20000F8
:104F000000000000F2F2000000000000F2F20000D9
:104F100000000000F2F2000000000000F2F20000C9
:104F20000000F2F2F2F2F2F20000000000000000D5
:104F3000000000F2F2F200000000F2F200F2F200D3
:104F400000F2F2000000F2F200F2F2000000F2F2D1
:104F500000F2F2F2F2F2F2F200F2F2000000F2F2EB
:104F600000F2F2000000F2F2000000000000000079
:104F700000F2F2F2F2F2F20000F2F2000000F2F2BD
:104F800000F2F2000000F2F200F2F2F2F2F2F200AD
:104F900000F2F2000000F2F200F2F2000000F2F281
:104FA00000F2F2F2F2F2F200000000000000000055
:104FB00000F2F2F2F2F2F2F200F2F200000000006F
:104FC00000F2F2000000000000F2F2F2F2F2F20051
:104FD00000F2F2000000000000F2F2000000000009
:104FE00000F2F2F2F2F2F2F2000000000000000023
:104FF00000F2F2F2F2F2F2F200F2F200000000002F
:1050000000F2F2000000000000F2F2F2F2F2F20010
:1050100000F2F2000000000000F2F20000000000C8
:1050200000F2F2000000000000000000000000009C
:1050300000F2F2000000F2F200F2F2000000F2F2E0
:1050400000F2F2000000F2F200F2F2F2F2F2F2F2FA
:1050500000F2F2000000F2F200F2F2000000F2F2C0
:1050600000F2F2000000F2F2000000000000000078
:105070000000F2F2F2F2F2F200000000F2F20000A0
:1050800000000000F2F2000000000000F2F2000058
:1050900000000000F2F2000000000000F2F2000048
:1050A0000000F2F2F2F2F2F2000000000000000054
:1050B00000F2F2000000F2F200F2F20000F2F20060
:1050C00000F2F200F2F2000000F2F2F2F200000050
:1050D00000F2F2F2F2F2000000F2F200F2F2F2005C
:1050E00000F2F20000F2F2F2000000000000000006
:1050F0000000F2F2000000000000F2F200000000E8
:105100000000F2F2000000000000F2F200000000D7
:105110000000F2F2000000000000F2F200000000C7
:105120000000F2F2F2F2F2F20000000000000000D3
:1051300000F2F2000000F2F200F2F2F20000F2F2ED
:1051400000F2F2F2F200F2F200F2F2F2F2F2F2F215
:1051500000F2F200F2F2F2F200F2F20000F2F2F2E9
:1051600000F2F2000000F2F2000000000000000077
:105170000000F2F2F2F2F20000F2F2000000F2F2AD
:1051800000F2F2000000F2F200F2F2000000F2F28F
:1051900000F2F2000000F2F200F2F2000000F2F27F
:1051A0000000F2F2F2F2F200000000000000000045
:1051B00000F2F2F2F2F2F20000F2F2000000F2F27B
:1051C00000F2F2000000F2F200F2F2000000F2F24F
:1051D00000F2F2F2F2F2F20000F2F200000000003F
:1051E00000F2F200000000000000000000000000DB
:1051F00000F2F2F2F2F2F20000F2F2000000F2F23B
:1052000000F2F2000000F2F200F2F20000F2F2F21C
:1052100000F2F2F2F2F2000000F2F200F2F2F2001A
:1052200000F2F20000F2F2F20000000000000000C4
:105230000000F2F2F2F2000000F2F20000F2F200DE
:1052400000F2F200000000000000F2F2F2F2F200C0
:10525000000000000000F2F200F2F2000000F2F2A2
:105260000000F2F2F2F2F200000000000000000084
:1052700000F2F2000000F2F200F2F2000000F2F29E
:1052800000F2F2000000F2F200F2F2000000F2F28E
:1052900000F2F2000000F2F200F2F2000000F2F27E
:1052A0000000F2F2F2F2F200000000000000000044
:1052B0000000F2F20000F2F20000F2F20000F2F25E
:1052C0000000F2F20000F2F2000000F2F2F2F2004E
:1052D00000000000F2F2000000000000F2F2000006
:1052E00000000000F2F200000000000000000000DA
:1052F0000000002F002F00000000002F002F0000F2
:105300000000002F002F000000000000000000003F
:10531000000000000000000000000000000000008D
:10532000000000000000000000000000000000007D
:10533000000000000000000000000000000000006D
:10534000000000000000000000002F2F2F2F2F0072
:10535000000000000000000000000000000000004D
:10536000000000000000000000000000000000003D
:105370000000002F2F2F000000002F2F002F2F00E4
:10538000002F2F0000002F2F002F2F0000002F2FA5
:10539000002F2F2F2F2F2F2F002F2F0000002F2F08
:1053A000002F2F0000002F2F000000000000000041
:1053B000002F2F2F2F2F2F00002F2F0000002F2F17
:1053C000002F2F0000002F2F002F2F2F2F2F2F0007
:1053D000002F2F0000002F2F002F2F0000002F2F55
:1053E000002F2F2F2F2F2F000000000000000000A3
:1053F0000000002F2F2F2F0000002F2F00002F2F35
:10540000002F2F0000000000002F2F0000000000E0
:10541000002F2F000000000000002F2F00002F2F72
:105420000000002F2F2F2F000000000000000000C0
:10543000002F2F2F2F2F0000002F2F00002F2F00C5
:10544000002F2F0000002F2F002F2F0000002F2FE4
:10545000002F2F0000002F2F002F2F00002F2F00D4
:10546000002F2F2F2F2F0000000000000000000051
:10547000002F2F2F2F2F2F2F002F2F000000000085
:10548000002F2F0000000000002F2F2F2F2F2F00A4
:10549000002F2F0000000000002F2F000000000050
:1054A000002F2F2F2F2F2F2F0000000000000000B3
:1054B000002F2F0000002F2F002F2F0000002F2F74
:1054C000002F2F0000002F2F002F2F2F2F2F2F2FD7
:1054D000002F2F0000002F2F002F2F0000002F2F54
:1054E000002F2F0000002F2F000000000000000000
:1054F000002F2F0000002F2F002F2F00002F2F0034
:10550000002F2F002F2F0000002F2F2F2F00000023
:10551000002F2F2F2F2F0000002F2F002F2F2F00B5
:10552000002F2F00002F2F2F000000000000000090
:1055300000002F2F0000000000002F2F00000000AF
:1055400000002F2F0000000000002F2F000000009F
:1055500000002F2F0000000000002F2F000000008F
:1055600000002F2F2F2F2F2F000000000000000021
:10557000002F2F0000002F2F002F2F2F00002F2F84
:10558000002F2F2F2F002F2F002F2F2F2F2F2F2FB8
:10559000002F2F002F2F2F2F002F2F00002F2F2F06
:1055A000002F2F0000002F2F00000000000000003F
:1055B00000002F2F2F2F2F00002F2F0000002F2F44
:1055C000002F2F0000002F2F002F2F0000002F2F63
:1055D000002F2F0000002F2F002F2F0000002F2F53
:1055E00000002F2F2F2F2F000000000000000000D0
:1055F000002F2F2F2F2F2F00002F2F0000002F2FD5
:10560000002F2F0000002F2F002F2F0000002F2F22
:10561000002F2F2F2F2F2F00002F2F000000000012
:10562000002F2F000000000000000000000000001C
:10563000002F2F2F2F2F2F00002F2F0000002F2F94
:10564000002F2F0000002F2F002F2F00002F2F2FB3
:10565000002F2F2F2F2F0000002F2F002F2F2F0074
:10566000002F2F00002F2F2F00000000000000004F
:1056700000002F2F2F2F0000002F2F00002F2F00B2
:10568000002F2F000000000000002F2F2F2F2F00D1
:105690000000000000002F2F002F2F0000002F2FF0
:1056A00000002F2F2F2F2F0000000000000000000F
:1056B00000002F2F2F2F2F2F000000002F2F000072
:1056C000000000002F2F0000000000002F2F00001E
:1056D000000000002F2F0000000000002F2F00000E
:1056E000000000002F2F000000000000000000005C
:1056F000002F2F0000002F2F002F2F0000002F2F32
:10570000002F2F0000002F2F002F2F0000002F2F21
:10571000002F2F0000002F2F002F2F0000002F2F11
:1057200000002F2F2F2F2F0000000000000000008E
:1057300000002F2F00002F2F00002F2F00002F2FF1
:1057400000002F2F00002F2F0000002F2F2F2F00E1
:10575000000000002F2F0000000000002F2F00008D
:10576000000000002F2F00000000000000000000DB
:105770000000000000000000000000000000000029
:1057800000000000000000000000AFAFAFAFAF00AE
:105790000000000000000000000000000000000009
:1057A00000000000000000000000000000000000F9
:1057B000000000AFAFAF00000000AF0000AFAF00CF
:1057C00000AFAF000000AFAF00AFAF000000AFAF61
:1057D00000AFAF000000AFAF0000AFAF0000AF0000
:1057E000000000AFAFAF00000000000000000000AC
:1057F00000000000AFAF0000000000AFAFAF00003E
:1058000000000000AFAF000000000000AFAF0000DC
:1058100000000000AFAF000000000000AFAF0000CC
:105820000000AFAFAFAFAFAF00000000000000005E
:10583000000000AFAFAF00000000AFAF00AFAF009F
:1058400000AFAF000000AFAF00AFAF000000AFAFE0
:1058500000AFAFAFAFAFAFAF00AFAF000000AFAFC3
:1058600000AFAF000000AFAF00000000000000007C
:1058700000AFAFAFAFAFAF0000AFAF000000AFAF52
:1058800000AFAF000000AFAF00AFAFAFAFAFAF0042
:1058900000AFAF000000AFAF00AFAF000000AFAF90
:1058A00000AFAFAFAFAFAF000000000000000000DE
:1058B000000000AFAFAFAF000000AFAF0000AFAF70
:1058C00000AFAF000000000000AFAF00000000001C
:1058D00000AFAF00000000000000AFAF0000AFAFAE
:1058E000000000AFAFAFAF000000000000000000FC
:1058F00000AFAFAFAFAFAFAF00AFAF000000000081
:1059000000AFAF000000000000AFAFAFAFAFAF001F
:1059100000AFAF000000000000AFAF0000000000CB
:1059200000AFAF0000000000000000000000000019
:1059300000AFAF000000AFAF00AFAFAF00AFAFAF91
:1059400000AFAFAFAFAFAFAF00AFAFAFAFAFAFAFC5
:1059500000AFAF00AF00AFAF00AFAF000000AFAF20
:1059600000AFAF000000AFAF00000000000000007B
:1059700000AFAF000000AFAF00AFAFAF0000AFAF00
:1059800000AFAFAFAF00AFAF00AFAFAFAFAFAFAF34
:1059900000AFAF00AFAFAFAF00AFAF0000AFAFAF82
:1059A00000AFAF000000AFAF00000000000000003B
:1059B0000000AFAFAFAFAF0000AFAF000000AFAFC0
:1059C00000AFAF000000AFAF00AFAF000000AFAF5F
:1059D00000AFAF000000AFAF00AFAF000000AFAF4F
:1059E0000000AFAFAFAFAF0000000000000000004C
:1059F00000AFAFAFAFAFAF0000AFAF000000AFAFD1
:105A000000AFAF000000AFAF00AFAF000000AFAF1E
:105A100000AFAFAFAFAFAF0000AFAF00000000000E
:105A200000AFAF0000000000000000000000000018
:105A300000AFAFAFAFAFAF0000AFAF000000AFAF90
:105A400000AFAF000000AFAF00AFAF0000AFAFAF2F
:105A500000AFAFAFAFAF000000AFAF00AFAFAF0070
:105A600000AFAF0000AFAFAF0000000000000000CB
:105A70000000AFAFAFAF000000AFAF0000AFAF00AE
:105A800000AFAF00000000000000AFAFAFAFAF004D
:105A9000000000000000AFAF00AFAF000000AFAFEC
:105AA0000000AFAFAFAFAF0000000000000000008B
:105AB0000000AFAFAFAFAFAF00000000AFAF00006E
:105AC00000000000AFAF000000000000AFAF00001A
:105AD00000000000AFAF000000000000AFAF00000A
:105AE00000000000AFAF0000000000000000000058
:105AF00000AFAF000000AFAF00AFAF000000AFAF2E
:105B000000AFAF000000AFAF00AFAF000000AFAF1D
:105B100000AFAF000000AFAF00AFAF000000AFAF0D
:105B20000000AFAFAFAFAF0000000000000000000A
:105B30000000000000000000000000000000000065
:105B4000000000000000000000000000B7B70000E7
:105B500000000000B7B700000000000000000000D7
:105B60000000000000000000000000000000000035
:105B7000000000000000000000000000B7B70000B7
:105B8000000000B7B7B7B7000000B7B7B7B7B7B7EF
:105B90000000B7B7B7B7B7B7000000B7B7B7B700DF
:105BA00000000000B7B70000000000000000000087
:105BB000001B19010203030405050505050505057C
:105BC00006050505050505050507030308090A0B74
:105BD0000C030D0E0E0E0E0E0E0E0E0F0E0E0E0EF2
:105BE0000E0E0E0E10030B0C0A111213030D0E14E1
:105BF000150E1416150E0F0E1416150E14150E1084
:105C000003121311031718030D191A1B0E1A1C1B6C
:105C10000E1D0E1A1C1B0E1A1B1910031718030356
:105C20000303030D0E0E0E0E0E0E0E0E0E0E0E0EB6
:105C30000E0E0E0E0E10030303031E1F20030D0E87
:105C400021220E230E21242524220E230E21220E92
:105C50001003262728292A2B030D0E0E0E0E0F0ED9
:105C60000E0E0F0E0E0E0F0E0E0E0E10032C2D2EFE
:105C70002F303103323333340E352422031D0321F8
:105C800024360E3733333803393A3B030303030317
:105C900003030D0E0F030303030303030F0E10038F
:105CA0000303030303033C3D3E033F0505400E1D74
:105CB000034142434445031D0E4605054703484939
:105CC0004A4B4C4D03030303030E0303100303036A
:105CD0000D03030E03030303034E4F5051525303AE
:105CE000543333340E2303550505055603230E376D
:105CF0003333570358595A030303030303030D0EA9
:105D00000F030303030303030F0E10030303030333
:105D100003030B0C0303040505400E1D032124257A
:105D20002422031D0E4605050703030B0C12135B0B
:105D3000030D0E0E0E0E0E0E0E0E0F0E0E0E0E0E8E
:105D40000E0E0E10035B121317180A030D0E215CC2
:105D50000E2124220E1D0E2124220E5D220E100380
:105D60000A171803085E030D190E0F0E0E0E0E0E05
:105D7000030E0E0E0E0E0F0E1910035F0203030327
:105D8000030360220E1D0E230E21242524220E2340
:105D90000E1D0E216103030303626364030D0E0EE7
:105DA0000E0E0F0E0E0E0F0E0E0E0F0E0E0E0E100E
:105DB00003626364656667030D0E21242468242250
:105DC0000E1D0E2124682424220E100365696765C8
:105DD0006667030D0E0E0E0E0E0E0E0E0E0E0E0E3E
:105DE0000E0E0E0E0E1003656A67656B6703323385
:105DF0003333333333333333333333333333333373
:105E00003803656C676D6E6F0303030303030303BD
:105E1000030303030303030303030303036D6E6F11
:105E20000303030303030303030303030303030342
:105E30000303030303030303030303030303030332
:105E40000303030303707172737471750303030317
:105E500003030303030302022A2B30310202262725
:105E60002C2D02023D3E4C4D0202494A4F50020287
:105E70007677303102027879303102027A277B7CE2
:105E8000020226277D7E02027F804C4D0202818223
:105E90008384020285864F87020288898A8B0101EA
:105EA0008C05018D8E8F9091070192939495969712
:105EB000980701999A9B9C9D9E9F131604050505C2
:105EC0000505050505060505050505050505070D77
:105ED00003030303030303030F0303030303030386
:105EE00003100D03141503141615030F03141615D0
:105EF00003141503100D031A1B031A1C1B031D03A7
:105F00001A1C1B031A1B03100D03030303030303D3
:105F100003030303030303030303100D03212203FD
:105F200023032124252422032303212203100D030C
:105F30000303030F0303030F0303030F030303030D
:105F4000103233333403352422031D032124360356
:105F5000373333380303030D030F03030303030332
:105F6000030F03100303033F050540031D034142D4
:105F7000434445031D034605054703030303030389
:105F800003100303030D0303030303030354333319
:105F900034032303550505055603230337333357CD
:105FA0000303030D030F030303030303030F031092
:105FB00003030304050540031D03212425242203B4
:105FC0001D03460505070D03030303030303030F26
:105FD0000303030303030303100D03215C032124C4
:105FE00022031D03212422035D2203100D03030F4E
:105FF00003030303030303030303030F03031060FB
:1060000022031D03230321242524220323031D032C
:1060100021610D030303030F0303030F0303030FA6
:1060200003030303100D03212424682422031D030A
:1060300021246824242203100D0303030303030314
:106040000303030303030303030310323333333324
:106050003333333333333333333333333338131648
:10606000A0A1A1A1A1A1A1A1A1A2A1A1A1A1A1A120
:10607000A1A1A3A40303030303030303A5030303D1
:106080000303030303A6A403A7A803A7A9A803A5C2
:1060900003A7A9A803A7A803A6A403AAAB03AAACB5
:1060A000AB03AD03AAACAB03AAAB03A6A4030303E3
:1060B0000303030303030303030303030303A6A46C
:1060C00003AEAF03B003AEB1B2B1AF03B003AEAF36
:1060D00003A6A403030303A5030303A5030303A566
:1060E00003030303A6B3B4B4B503B6B1AF03AD0362
:1060F000AEB1B703B8B4B4B9030303A403A5030353
:106100000303030303A503A6030303BAA1A1BB036F
:10611000AD03414243444503AD03BCA1A1BD03030C
:106120000303030303100303030D03030303030328
:1061300003BEB4B4B503B003550505055603B0035B
:10614000B8B4B4BF030303A403A503030303030309
:1061500003A503A6030303A0A1A1BB03AD03AEB136
:10616000B2B1AF03AD03BCA1A1A3A4030303030316
:10617000030303A50303030303030303A6A403AE5E
:10618000C003AEB1AF03AD03AEB1AF03C1AF03A661
:10619000A40303A50303030303030303030303A5EA
:1061A0000303A6C2AF03AD03B003AEB1B2B1AF03F8
:1061B000B003AD03AEC3A403030303A5030303A508
:1061C000030303A503030303A6A403AEB1B1C4B143
:1061D000AF03AD03AEB1C4B1B1AF03A6A4030303D3
:1061E0000303030303030303030303030303A6B32C
:1061F000B4B4B4B4B4B4B4B4B4B4B4B4B4B4B4B45F
:10620000B4B9FEFEFEFEFEFEFEFEFEFEFEF2F2FE55
:10621000FEFEFEFEF2FEFEF2FEF2FEFEFEFEFEF2CE
:10622000FEF2FEFEFEFEF2FEFEF2FEFEFEF2FEFEBE
:10623000FEF2FEFEF2F2F2F2FEFEFEFEFEFEFEFEBA
:10624000FEFEFEFEFEFEFEFEFEFEF2FEFEFEF2FE86
:10625000FEFEFEF2FEF2FEF2FEFEFEF2FEF2FEF2A6
:10626000FEFEFEF2FEF2FEF2FEFEFEF2FEF2FEF296
:10627000FEFEF2FEFEFEF2FEFEFEFEFEFEFEFEFE56
:10628000FEFEFEFEFEFEFEFEFEFEFEFEF2FEFEFE3A
:10629000FEFEFEFEF2FEFEFEFEF2FEFEF2FEF2FE4E
:1062A000FEF2FEFEF2F2F2F2FEF2FEFEFEFEF2FE62
:1062B000FEF2FEFEFEFEF2FEFEFEFEFEFEFEFEFE16
:1062C000FEFEFEFEFEFEFEFEFEFEFEFEFEF2F2FE06
:1062D000FEFEFEFEF2FEFEF2FEF2FEFEF2FEFEF21A
:1062E000FEF2FEFEFEF2F2FEFEF2FEFEF2FEFEF216
:1062F000FEF2FEFEFEF2F2FEFEFEFEFEFEFEFEFEE2
:10630000FEFEFEFEFEFEFEFEFEFEFEF2FEFEFEF2C5
:10631000F2FEF2F2FEFEF2FEFEFEFEF2FEFEF2FEE5
:10632000FEFEFEF2FEFEF2F2F2FEFEF2FEFEF2FED5
:10633000FEF2F2F2F2FEFEF2F2FEFEFEFEFEFEFEC5
:10634000FEFEFEFEFEFEFEFEFEFEFEFEF2FEFEFE79
:10635000F2FEFEF2FEF2FEF2FEF2FEF2FEF2FEF2BD
:10636000FEF2FEF2FEF2FEF2FEF2FEF2FEF2FEF2AD
:10637000FEF2FEFEF2FEFEFEF2FEFEFEFEFEFEFE61
:10638000FEFEFEFEFEFEFEFEFEFEFEFEFEFEAFFE7C
:10639000FEFEFEFEFEAFAFFEFEAFFEFEFEFEAFFE59
:1063A000FEAFFEFEFEFEAFFEFEAFFEFEFEFEAFFE49
:1063B000FEAFFEFEFEAFAFAFFEFEFEFEFEFEFEFE39
:1063C000FEFEFEFEFEFEFEFEFEFEAFFEFEFEAFFE8B
:1063D000FEFEFEAFFEAFFEAFFEFEFEAFFEAFFEAFB7
:1063E000FEFEFEAFFEAFFEAFFEFEFEAFFEAFFEAFA7
:1063F000FEFEAFFEFEFEAFFEFEFEFEFEFEFEFEFE5B
:10640000FEFEFEFEFEFEFEFEFEFEFEFEAFAFAFFE99
:10641000FEFEFEFEFEFEFEAFFEAFFEFEFEFEFEAF89
:10642000FEAFFEFEFEAFAFFEFEAFFEFEFEFEFEAF17
:10643000FEAFFEFEAFAFAFFEFEFEFEFEFEFEFEFEB8
:10644000FEFEFEFEFEFEFEFEFEFEFEFEAFAFAFAFA8
:10645000FEFEFEFEAFFEFEFEFEAFFEFEAFFEFEFE49
:10646000FEAFFEFEFEAFAFFEFEAFFEFEFEFEFEAFD7
:10647000FEAFFEFEAFAFAFFEFEFEFEFEFEFEFEFE78
:10648000FEFEFEFEFEFEFEFEFEFEFEFEAFAFAFAF68
:10649000FEFEFEFEFEFEFEAFFEAFFEFEFEFEAFFE09
:1064A000FEAFFEFEFEAFFEFEFEAFFEFEFEAFFEFE48
:1064B000FEAFFEFEFEAFFEFEFEFEFEFEFEFEFEFE9A
:1064C000FEFEFEFEFEFEFEFEFEFEFEFEAFFEFEFE3B
:1064D000AFFEFEAFAFFEFEAFFEAFFEFEAFFEFEAF05
:1064E000FEAFFEFEAFFEFEAFFEAFFEFEAFFEFEAFA6
:1064F000FEAFFEAFAFAFFEFEAFFEFEFEFEFEFEFE47
:10650000FEFEFEFEFEFEFEFEFEFEFEFEAFFEFEFEFA
:10651000AFFEFEAFFEAFFEAFFEAFFEAFFEAFFEAF13
:10652000FEAFFEAFFEAFFEAFFEAFFEAFFEAFFEAF03
:10653000FEAFFEFEAFFEFEFEAFFEFEFEFEFEFEFE68
:10654000FEFEFEFEFEFEFEFEFEFEFEAFAFFEFEFE09
:10655000AFFEAFFEFEAFFEAFFEAFFEFEFEAFFEAF84
:10656000FEAFFEFEAFFEFEAFFEAFFEAFFEFEFEAF25
:10657000FEAFAFAFAFAFFEFEAFFEFEFEFEFEFEFE15
:10658000FEFEFEFEFEFEFEFEFEFEAFAFAFFEFEFE18
:10659000AFFEFEFEFEAFFEAFFEAFFEFEFEAFFEAFF5
:1065A000FEAFFEAFAFFEFEAFFEAFFEFEFEAFFEAF34
:1065B000FEAFAFAFAFFEFEFEAFFEFEFEFEFEFEFE86
:1065C000FEFEFEFEFEFEFEFEFEFEAFAFAFAFFEFE27
:1065D000AFFEAFFEFEFEFEAFFEAFAFFEFEFEFEAFB5
:1065E000FEAFFEAFAFFEFEAFFEAFFEFEFEAFFEAFF4
:1065F000FEAFAFAFAFFEFEFEAFFEFEFEFEFEFEFE46
:10660000FEFEFEFEFEFEFEFEFEFEFEFEFEFEFEFEAA
:10661000FEFEFEFEFEFEFEFE3F3FFEFEFEFE3F3F96
:106620003F3FFEFEFE3F3F3F3F3FFEFEFE3F3F3F00
:106630003F3FFEFE3F3F3F3F3F3FFEFE3F3F3F3F6E
:106640003F3FFEFEFEFEFEFEFEFEFEFEFEFEFEFEE8
:10665000FEFE3F3FFEFEFEFEFEFE3F3F3F3FFEFED4
:10666000FEFE3F3F3F3F3FFEFEFE3F3F3F3F3FFEC0
:10667000FEFE3F3F3F3F3F3FFEFE3F3F3F3F3F3F2E
:10668000FEFEFEFE3F3F3F3F3F3FFEFE3F3F3F3FA0
:106690003F3FFEFEFE3F3F3F3F3FFEFEFE3F3F3F90
:1066A0003F3FFEFEFEFE3F3F3F3FFEFEFEFEFEFE84
:1066B0003F3FFEFEFEFEFEFEFEFEFEFEFEFEFEFE78
:1066C000FEFE3F3F3F3F3F3FFEFE3F3F3F3F3F3FDE
:1066D000FEFE3F3F3F3F3FFEFEFE3F3F3F3F3FFE50
:1066E000FEFE3F3F3F3FFEFEFEFE3F3FFEFEFEFE44
:1066F000FEFEFEFEFEFEFEFEFEFEFEFEFEFEFEFEBA
:10670000FEFEFEFEFEFEFEFEFEFEFEFEFEFEFEFEA9
:10671000FEFE3F3F3FFEFEFEFEFE3F3F3F3F3FFE91
:10672000FEFE3F3F3F3F3F3FFEFE3F3F3F3FFEFEFF
:10673000FEFE3F3FFEFEFEFEFEFEFEFEFEFEFEFEF7
:10674000FEFEFEFEFEFEFEFEFEFE3F3FFEFEFEFEE7
:10675000FEFE3F3F3F3FFEFEFEFE3F3F3F3F3F3FCF
:10676000FEFE3F3F3F3F3FFEFEFE3F3F3FFEFEFE41
:10677000FEFEFEFEFEFEFEFEFEFEFEFEFEFEFEFE39
:10678000FEFEFEFEFEFEFEFEFEFEFEFEFEFEFEFE29
:10679000FEFEFEFEFEFEFEFEFEFEFEFEFEFEFEFE19
:1067A000FE3FFEFEFEFEFEFE3F3FFEFEFEFEFEFE46
:1067B0003F3FFEFEFEFEFE3F3F3FFEFEFEFEFE3F73
:1067C0003F3FFEFEFEFEFEFEFEFEFEFEFEFEFEFE67
:1067D000FEFEFE3F3F3F3F3FFEFE3F3F3F3F3FFE4F
:1067E000FEFE3F3F3F3FFEFEFEFE3F3F3FFEFEFE02
:1067F000FEFE3F3FFEFEFEFEFEFE3FFEFEFEFEFEF6
:10680000FEFEFEFEFEFEFE3F3F3FFEFEFEFEFE3FA4
:106810003F3FFEFEFEFEFEFE3F3FFEFEFEFEFEFE94
:106820003F3FFEFEFEFEFEFEFE3FFEFEFEFEFEFEC5
:10683000FEFEFEFEFEFEFEFEFEFEFEFEFEFEFEFE78
:10684000FEFE3FFEFEFEFEFEFEFE3F3FFEFEFEFEA5
:10685000FEFE3F3F3FFEFEFEFEFE3F3F3F3FFEFE91
:10686000FEFE3F3F3F3F3FFEFEFEFE3F3F3F3F3FBE
:10687000FEFEFEFEFEFEFEFEFEFEFEFEFEFEFEFE38
:10688000FEFEFEFEFEFEFEFEFEFEFEFEFEFEFEFE28
:10689000FEFEFEFEFEFEFEFEFEFEFEFEFEFEFEFE18
:1068A000FEFEFEFEFEFEFEFEEFEFFEFEFEFEFE071D
:1068B00007EFFEFEFE0707070707FEFE07070707AD
:1068C0000707FEFEFEFFFEFEFFFEFEFEFFFFC9FF06
:1068D000FFC9FEFEFFFFC9FFFFC9EFEFEFFFEFEFBC
:1068E000FFFEEFEFEFEFEFEFFEFEEFEFEFEFFEFE5D
:1068F000FEFEEFEFEFEFFEFEFEFE07EFEFFEFEFE09
:10690000FEFEFEFEFEFEFEFEFEFEFEFEFEFEFEFEA7
:10691000FEFEFEFEFEFEFEFEFEFEFEFEFEFEFEFE97
:10692000FEFEFEFEFEFEFEFEEFEFFEFEFEFEFE079C
:1069300007EFFE07FE070707070707070707070711
:106940000707FEFEFEFFFEFEFFFEFEFEFFFFC9FF85
:10695000FFC9FEFEFFFFC9FFFFC9EFEFEFFFEFEF3B
:10696000FFFEEFEFEFEFEFEFFEFEEFEFEFEFFEFEDC
:10697000FEFEEFEFEFEFEFFEFEFE07FEFEEFEFFE97
:10698000FEFEFEFE3F3F3F3FFEFEFE3F3F3F3F3FDE
:106990003FFE3F3F3F3F3F3F3F3F3F3F3F3F3F3F48
:1069A0003F3F3F3F3F3F3F3F3F3F3F3F3F3F3F3FF7
:1069B0003F3FFE3F3F3F3F3F3FFEFEFE3F3F3F3FEB
:1069C000FEFEFE3FFEFEFEFE3FFE3F3FFEFEFEFEE3
:1069D0003F3F3F3F3FFEFE3F3F3F3F3F3FFEFE3FCB
:1069E0003F3F3F3F3F3F3F3F3F3FFE3F3F3F3F3FF8
:1069F0003FFEFE3F3F3F3F3F3FFEFEFE3F3F3F3FEC
:106A0000FEFEFEFEFE3F3F3F3FFEFE3F3F3F3F3F5D
:106A10003F3F3F3F3F3F3F3FFEFE3F3F3F3FFEFE8A
:106A2000FEFE3F3F3F3FFEFEFEFE3F3F3F3F3F3FFC
:106A3000FEFEFE3F3F3F3F3F3F3FFEFEFE3F3F3FEC
:106A40003FFEFEFE3F3F3F3FFEFEFE3F3F3F3F3FDC
:106A50003FFEFE3F3F3F3F3F3FFE3F3F3F3F3F3F09
:106A60003F3F3F3F3FFEFE3F3F3F3F3F3FFEFE3F3A
:106A70003F3F3F3FFEFEFEFE3F3FFE3FFEFEFEFE6F
:106A80003FFEFE3F3F3F3FFEFEFE3F3F3F3F3F3F5B
:106A90003FFEFEFE3F3F3F3F3F3FFEFEFEFE3F3FCD
:106AA0003F3FFEFEFEFE3F3F3F3FFEFE3F3F3F3F7C
:106AB0003F3F3F3F3F3F3F3F3FFEFE3F3F3F3FFEA9
:106AC000FEFE3FFEFEFEFEFEFE3F3F3FFEFEFEFEE2
:106AD0003F3F3F3FFEFEFEFE3F3F3F3F3FFEFE3F4C
:106AE0003F3F3F3F3F3F3F3F3F3FFE3F3F3F3F3FF7
:106AF0003FFEFE3F3F3F3F3F3FFEFEFEFE3F3FFE6D
:106B0000FEFEFEFEFE3F3F3F3F3FFE3F3F3F3F3F1B
:106B10003FFEFE3F3F3F3FFEFEFE3F3F3F3FFEFE4C
:106B2000FEFE3F3F3F3FFEFEFEFEFE3F3F3F3FFE7D
:106B3000FEFEFE3F3F3F3F3F3FFEFEFEFE3F3F3F2C
:106B40003F3FFEFEFE3F3FFEFEFEFE3F3F3F3F3F1C
:106B50003FFEFE3F3F3F3F3F3FFE3F3F3F3F3F3F08
:106B60003F3F3F3F3FFEFE3F3F3F3F3FFEFEFEFEBB
:106B70003F3F3F3FFEFEFEFE3F3F3FFEFEFEFEFE6E
:106B8000FE3F3F3F3F3F3FFEFEFEFE3F3F3F3F3F5A
:106B90003FFEFEFEFE3F3F3F3FFEFEFEFEFE3F3F4E
:106BA0003F3FFEFEFEFE3F3F3F3FFEFEFE3F3F3FBC
:106BB0003FFEFE3F3F3F3F3F3FFE3F3F3F3F3FFEE9
:106BC000FEFEFEFEFEFEFEFEFEFEFE3FFEFEFEFEA4
:106BD0003FFE3F3FFEFEFEFE3F3F3F3F3FFEFE3F8C
:106BE0003F3F3F3F3F3F3F3F3F3FFE3F3F3F3F3FF6
:106BF0003FFEFE3F3F3F3F3F3FFEFEFE3FFEFE3F6C
:106C0000FEFEFEFEFEFEFEFEFEFEFEFEFEFEFEFEA4
:106C1000FEFEFEFEFEFEFEFEFEFE3FFEFEFEFEFE53
:106C2000FE3F3F3FFEFEFEFE3F3F3F3F3F3F3F3FB9
:106C30003F3FFE3F3F3F3F3F3FFEFEFE3FFEFE3FEA
:106C4000FEFEFEFEFEFEFEFEFEFEFEFEFEFEFEFE64
:106C5000FEFEFEFEFEFEFEFEFEFE3F3FFEFEFEFED2
:106C60003F3F3F3F3F3F3F3F3F3F3F3F3F3F3F3F34
:106C70003F3FFE3F3F3F3F3F3FFEFEFE3FFEFE3FAA
:106C8000FEFEFEFEFEFEFEFEFEFEFEFEFEFEFEFE24
:106C9000FEFEFEFEFEFEFEFEFEFEFEFE3F3F3F3F10
:106CA000FEFE3F3F3F3F3F3F3F3F3F3F3F3F3F3F76
:106CB0003F3FFE3F3F3F3F3F3FFEFEFE3FFEFE3F6A
:106CC000FEFEFEFEFEFEFEFEFEFEFEFEFEFEFEFEE4
:106CD000FEFEFEFE3F3F3F3FFEFEFE3F3F3F3F3F8B
:106CE0003FFE3F3F3F3F3F3F3F3F3F3F3F3F3F3FF5
:106CF0003F3F3F3F3FFEFE3F3F3FFE3FFEFEFEFE6B
:106D00003FFEFEFEFEFEFEFEFEFEFEFEFE3F3FFEE0
:106D1000FEFEFEFE3F3F3F3FFEFEFE3F3F3F3F3F4A
:106D20003FFEFE3F3F3F3F3F3FFE3F3F3F3F3F3F36
:106D30003F3F3F3F3FFEFE3F3F3F3F3FFEFEFEFEE9
:106D40003F3FFEFEFEFEFEFEFEFEFEFEFE3F3FFE5F
:106D5000FEFEFEFE3F3F3F3FFEFEFEFE3F3F3F3F4B
:106D6000FEFEFE3F3F3F3F3F3FFEFE3F3F3F3F3F78
:106D70003FFE3F3F3F3F3F3F3F3F3F3F3FFEFE3FE6
:106D80003F3FFEFEFEFEFEFEFEFEFEFEFE3F3FFE1F
:106D9000FEFEFEFE3F3F3F3FFEFEFEFE3F3F3F3F0B
:106DA000FEFEFEFE3F3F3F3FFEFEFE3F3F3F3F3FBA
:106DB0003FFEFEFE3FFEFE3FFEFEFEFEFEFEFEFE30
:106DC000FEFEFEFEFEFEFEFEFEFEFEFEFEFEFEFEE3
:106DD000FEFEFEFEFE3F3FFEFEFEFEFEFE3F3FFECF
:106DE000FEFEFEFEFE3F3FFEFEFEFEFEFE3F3FFEBF
:106DF000FEFEFEFEFEFEFEFEFEFEFEFEFEFEFEFEB3
:106E0000FEFEFE3FFEFEFE3FFEFEFEFE3FFE3FFE9E
:106E1000FE3F3FFEFEFEFEFE3FFEFE3FFEFEFEFE8E
:106E2000FEFEFEFEFEFEFEFE3FFEFE3FFEFEFEFE00
:106E3000FE3F3FFEFE3FFE3FFEFEFEFE3FFEFEFE2D
:106E40003FFEFEFE07070707FEFEFE0707070707D0
:106E500007FEFE07FF0707FF07FEFEFFFFFFFFFF1E
:106E6000FFFE07FFC9FFFFC9FF070707C90707C9DB
:106E70000707070707FEFE07070707FE07FEFE07CF
:106E8000FE07FEFE07070707FEFEFE0707070707C8
:106E900007FEFE07FF0707FF07FEFEFFFFFFFFFFDE
:106EA000FFFE07FFC9FFFFC9FF070707C90707C99B
:106EB00007070707070707070707FE07FE0707FE7D
:106EC00007FEFEFEC90707C9FEFEFEFFC9FFFFC998
:106ED000FFFEFEFFFFFFFFFFFFFEFE07FF0707FFAE
:106EE00007FE07070707070707070707070707073B
:106EF0000707070707FEFE07070707FE07FEFE074F
:106F0000FE07FEFEC90707C9FEFEFEFFC9FFFFC957
:106F1000FFFEFEFFFFFFFFFFFFFEFE07FF0707FF6D
:106F200007FE0707070707070707070707070707FA
:106F300007070707070707070707FE07FE0707FEFC
:106F400007FEFEFE07070707FEFEFE07FF0707FF17
:106F500007FEFEC9FFFFC9FFFFFEFEC9FFFFC9FF15
:106F6000FFFE0707FF0707FF0707070707070707D2
:106F70000707070707FEFE07070707FE07FEFE07CE
:106F8000FE07FEFE07070707FEFEFE07FF0707FFD7
:106F900007FEFEC9FFFFC9FFFFFEFEC9FFFFC9FFD5
:106FA000FFFE0707FF0707FF070707070707070792
:106FB00007070707070707070707FE07FE0707FE7C
:106FC00007FEFEFE07070707FEFEFE07FF0707FF97
:106FD00007FEFEFFFFC9FFFFC9FEFEFFFFC9FFFF5F
:106FE000C9FE0707FF0707FF070707070707070788
:106FF0000707070707FEFE07070707FE07FEFE074E
:10700000FE07FEFE07070707FEFEFE07FF0707FF56
:1070100007FEFEFFFFC9FFFFC9FEFEFFFFC9FFFF1E
:10702000C9FE0707FF0707FF070707070707070747
:1070300007070707070707070707FE07FE0707FEFB
:1070400007FEFEFEF2F2F2F2FEFEFEF2F2F2F2F2C3
:10705000F2FEFEF2FFF2F2FFF2FEFEFFFFFFFFFF85
:10706000FFFEF2FFC9FFFFC9FFF2F2F2C9F2F2C957
:10707000F2F2F2F2F2FEFEF2F2F2F2FEF2FEFEF2B4
:10708000FEF2FEFEF2F2F2F2FEFEFEF2F2F2F2F298
:10709000F2FEFEF2FFF2F2FFF2FEFEFFFFFFFFFF45
:1070A000FFFEF2FFC9FFFFC9FFF2F2F2C9F2F2C917
:1070B000F2F2F2F2F2F2F2F2F2F2FEF2FEF2F2FE8C
:1070C000F2FEFEFEC9F2F2C9FEFEFEFFC9FFFFC9D5
:1070D000FFFEFEFFFFFFFFFFFFFEFEF2FFF2F2FFEB
:1070E000F2FEF2F2F2F2F2F2F2F2F2F2F2F2F2F274
:1070F000F2F2F2F2F2FEFEF2F2F2F2FEF2FEFEF234
:10710000FEF2FEFEC9F2F2C9FEFEFEFFC9FFFFC994
:10711000FFFEFEFFFFFFFFFFFFFEFEF2FFF2F2FFAA
:10712000F2FEF2F2F2F2F2F2F2F2F2F2F2F2F2F233
:10713000F2F2F2F2F2F2F2F2F2F2FEF2FEF2F2FE0B
:10714000F2FEFEFEF2F2F2F2FEFEFEF2FFF2F2FFBD
:10715000F2FEFEC9FFFFC9FFFFFEFEC9FFFFC9FF28
:10716000FFFEF2F2FFF2F2FFF2F2F2F2F2F2F2F2CC
:10717000F2F2F2F2F2FEFEF2F2F2F2FEF2FEFEF2B3
:10718000FEF2FEFEF2F2F2F2FEFEFEF2FFF2F2FF7D
:10719000F2FEFEC9FFFFC9FFFFFEFEC9FFFFC9FFE8
:1071A000FFFEF2F2FFF2F2FFF2F2F2F2F2F2F2F28C
:1071B000F2F2F2F2F2F2F2F2F2F2FEF2FEF2F2FE8B
:1071C000F2FEFEFEF2F2F2F2FEFEFEF2FFF2F2FF3D
:1071D000F2FEFEFFFFC9FFFFC9FEFEFFFFC9FFFF72
:1071E000C9FEF2F2FFF2F2FFF2F2F2F2F2F2F2F282
:1071F000F2F2F2F2F2FEFEF2F2F2F2FEF2FEFEF233
:10720000FEF2FEFEF2F2F2F2FEFEFEF2FFF2F2FFFC
:10721000F2FEFEFFFFC9FFFFC9FEFEFFFFC9FFFF31
:10722000C9FEF2F2FFF2F2FFF2F2F2F2F2F2F2F241
:10723000F2F2F2F2F2F2F2F2F2F2FEF2FEF2F2FE0A
:10724000F2FEFEFE2F2F2F2FFEFEFE2F2F2F2F2FB1
:107250002FFEFE2FFF2F2FFF2FFEFEFFFFFFFFFF52
:10726000FFFE2FFFC9FFFFC9FF2F2F2FC92F2FC9E7
:107270002F2F2F2F2FFEFE2F2F2F2FFE2FFEFE2F13
:10728000FE2FFEFE2F2F2F2FFEFEFE2F2F2F2F2F34
:107290002FFEFE2FFF2F2FFF2FFEFEFFFFFFFFFF12
:1072A000FFFE2FFFC9FFFFC9FF2F2F2FC92F2FC9A7
:1072B0002F2F2F2F2F2F2F2F2F2FFE2FFE2F2FFE71
:1072C0002FFEFEFEC92F2FC9FEFEFEFFC9FFFFC91C
:1072D000FFFEFEFFFFFFFFFFFFFEFE2FFF2F2FFF32
:1072E0002FFE2F2F2F2F2F2F2F2F2F2F2F2F2F2FDF
:1072F0002F2F2F2F2FFEFE2F2F2F2FFE2FFEFE2F93
:10730000FE2FFEFEC92F2FC9FEFEFEFFC9FFFFC9DB
:10731000FFFEFEFFFFFFFFFFFFFEFE2FFF2F2FFFF1
:107320002FFE2F2F2F2F2F2F2F2F2F2F2F2F2F2F9E
:107330002F2F2F2F2F2F2F2F2F2FFE2FFE2F2FFEF0
:107340002FFEFEFE2F2F2F2FFEFEFE2FFF2F2FFFD3
:107350002FFEFEC9FFFFC9FFFFFEFEC9FFFFC9FFE9
:10736000FFFE2F2FFF2F2FFF2F2F2F2F2F2F2F2FEE
:107370002F2F2F2F2FFEFE2F2F2F2FFE2FFEFE2F12
:10738000FE2FFEFE2F2F2F2FFEFEFE2FFF2F2FFF93
:107390002FFEFEC9FFFFC9FFFFFEFEC9FFFFC9FFA9
:1073A000FFFE2F2FFF2F2FFF2F2F2F2F2F2F2F2FAE
:1073B0002F2F2F2F2F2F2F2F2F2FFE2FFE2F2FFE70
:1073C0002FFEFEFE2F2F2F2FFEFEFE2FFF2F2FFF53
:1073D0002FFEFEFFFFC9FFFFC9FEFEFFFFC9FFFF33
:1073E000C9FE2F2FFF2F2FFF2F2F2F2F2F2F2F2FA4
:1073F0002F2F2F2F2FFEFE2F2F2F2FFE2FFEFE2F92
:10740000FE2FFEFE2F2F2F2FFEFEFE2FFF2F2FFF12
:107410002FFEFEFFFFC9FFFFC9FEFEFFFFC9FFFFF2
:10742000C9FE2F2FFF2F2FFF2F2F2F2F2F2F2F2F63
:107430002F2F2F2F2F2F2F2F2F2FFE2FFE2F2FFEEF
:107440002FFEFEFEEFEFEFEFFEFEFEEFEFEFEFEFB2
:10745000EFFEFEEFFFEFEFFFEFFEFEFFFFFFFFFF90
:10746000FFFEEFFFC9FFFFC9FFEFEFEFC9EFEFC965
:10747000EFEFEFEFEFFEFEEFEFEFEFFEEFFEFEEFD1
:10748000FEEFFEFEEFEFEFEFFEFEFEEFEFEFEFEFB2
:10749000EFFEFEEFFFEFEFFFEFFEFEFFFFFFFFFF50
:1074A000FFFEEFFFC9FFFFC9FFEFEFEFC9EFEFC925
:1074B000EFEFEFEFEFEFEFEFEFEFFEEFFEEFEFFEAF
:1074C000EFFEFEFEC9EFEFC9FEFEFEFFC9FFFFC9DA
:1074D000FFFEFEFFFFFFFFFFFFFEFEEFFFEFEFFFF0
:1074E000EFFEEFEFEFEFEFEFEFEFEFEFEFEFEFEF9D
:1074F000EFEFEFEFEFFEFEEFEFEFEFFEEFFEFEEF51
:10750000FEEFFEFEC9EFEFC9FEFEFEFFC9FFFFC999
:10751000FFFEFEFFFFFFFFFFFFFEFEEFFFEFEFFFAF
:10752000EFFEEFEFEFEFEFEFEFEFEFEFEFEFEFEF5C
:10753000EFEFEFEFEFEFEFEFEFEFFEEFFEEFEFFE2E
:10754000EFFEFEFEEFEFEFEFFEFEFEEFFFEFEFFFD1
:10755000EFFEFEC9FFFFC9FFFFFEFEC9FFFFC9FF27
:10756000FFFEEFEFFFEFEFFFEFEFEFEFEFEFEFEFEC
:10757000EFEFEFEFEFFEFEEFEFEFEFFEEFFEFEEFD0
:10758000FEEFFEFEEFEFEFEFFEFEFEEFFFEFEFFF91
:10759000EFFEFEC9FFFFC9FFFFFEFEC9FFFFC9FFE7
:1075A000FFFEEFEFFFEFEFFFEFEFEFEFEFEFEFEFAC
:1075B000EFEFEFEFEFEFEFEFEFEFFEEFFEEFEFFEAE
:1075C000EFFEFEFEEFEFEFEFFEFEFEEFFFEFEFFF51
:1075D000EFFEFEFFFFC9FFFFC9FEFEFFFFC9FFFF71
:1075E000C9FEEFEFFFEFEFFFEFEFEFEFEFEFEFEFA2
:1075F000EFEFEFEFEFFEFEEFEFEFEFFEEFFEFEEF50
:10760000FEEFFEFEEFEFEFEFFEFEFEEFFFEFEFFF10
:10761000EFFEFEFFFFC9FFFFC9FEFEFFFFC9FFFF30
:10762000C9FEEFEFFFEFEFFFEFEFEFEFEFEFEFEF61
:10763000EFEFEFEFEFEFEFEFEFEFFEEFFEEFEFFE2D
:10764000EFFEFEFEE2E2E2E2FEFEFEE2E2E2E2E265
:10765000E2FEFEE2EEE2E2EEE2FEFEE2E2E2E2E282
:10766000E2FEE2EEE2EEEEE2EEE2EEE2EEE2E2EE8A
:10767000E2EEE2E2E2FEFEE2E2E2E2FEE2FEFEE252
:10768000FEE2FEFEE2E2E2E2FEFEFEE2E2E2E2E232
:10769000E2FEFEE2EEE2E2EEE2FEFEE2E2E2E2E242
:1076A000E2FEE2EEE2EEEEE2EEE2EEE2EEE2E2EE4A
:1076B000E2EEE2E2E2E2E2E2E2E2FEE2FEE2E2FE4A
:1076C000E2FEFEFEFFFFFFFFFEFEFEFFFFFFFFFFED
:1076D000FFFEFEFFEEFFFFEEFFFEFEFFFFFFFFFFE0
:1076E000FFFEFFEEFFEEEEFFEEFFEEFFEEFFFFEE22
:1076F000FFEEFFFFFFFEFEFFFFFFFFFEFFFEFEFFB0
:10770000FEFFFEFEFFFFFFFFFEFEFEFFFFFFFFFF8F
:10771000FFFEFEFFEEFFFFEEFFFEFEFFFFFFFFFF9F
:10772000FFFEFFEEFFEEEEFFEEFFEEFFEEFFFFEEE1
:10773000FFEEFFFFFFFFFFFFFFFFFEFFFEFFFFFE6D
:10774000FFFEFEFEFEFEFEFEFEFEFEFEFEFEFEFE58
:10775000FEFEFEFEFFFEFEFFFEFEFEFFFFFFFFFF42
:10776000FFFEFEFFC9FFFFC9FFFEFEFEC9FEFEC908
:10777000FEFEFEFEFEFEFEFEFEFEFEFEFEFEFEFE29
:10778000FEFEFEFEFEFEFEFEFEFEFEFEFEFEFEFE19
:10779000FEFEFEFEC9FEFEC9FEFEFEFFC9FFFFC9DA
:1077A000FFFEFEFFFFFFFFFFFFFEFEFEFFFEFEFFF0
:1077B000FEFEFEFEFEFEFEFEFEFEFEFEFEFEFEFEE9
:1077C000FEFEFEFEFEFEFEFEFEFEFEFEFEFEFEFED9
:1077D000FEFEFEFEFFFEFEFFFEFEFEC9FFFFC9FF2E
:1077E000FFFEFEC9FFFFC9FFFFFEFEFEFFFEFEFF1C
:1077F000FEFEFEFEFEFEFEFEFEFEFEFEFEFEFEFEA9
:10780000FEFEFEFEFEFEFEFEFEFEFEFEFEFEFEFE98
:10781000FEFEFEFEFFFEFEFFFEFEFEFFFFC9FFFFB7
:10782000C9FEFEFFFFC9FFFFC9FEFEFEFFFEFEFF11
:10783000FEFEFEFEFEFEFEFEFEFEFEFEFEFEFEFE68
:10784000FEFEFEFE07070707FEFEFE07FF0707FF17
:1078500007FEFEC9FFFFC9FFFFFEFEC9FFFFC9FF0C
:10786000FFFE0707FF0707FF07EF070707070707E1
:10787000EF07070707FEFEEF070707FE07FEFE07F5
:10788000FE07FEFE07070707FEFEFE07FF0707FFCE
:1078900007FEFEC9FFFFC9FFFFFEFEC9FFFFC9FFCC
:1078A000FFFE0707FF0707FF07EF070707070707A1
:1078B000EF070707070707EF0707FE07FE0707FEA3
:1078C00007FE0000000000000000000000000000B3
:1078D00000000000000000000000000000000000A8
:1078E0000000000000000000000000000000000098
:1078F0000000000000000000000000000000000088
:107900000000020100010201020102010301020163
:107910000405020106070201080702010907020126
:107920000A0702010B0C02010D0C02010E0C0201F0
:107930000F0C02021011121302021014121502028F
:107940001617181902011A1B02011C1D01015B0206
:10795000025B5B5B5B1E1F231F1E2226221E21254E
:10796000211E2024202728292A2B2C2D2E2F3010B1
:10797000111213101412151617181910141215518C
:107980005253545152565755583334353631323795
:1079900038595A1A1B1C1D4B4C4D4E494A4F503BEF
:1079A0003C3D3E393A3F4043444546414247480109
:1079B000010104000002557901010104000002598F
:1079C00079010101040000025D7901010104000058
:1079D0000261790101010A000008657904020210C0
:1079E0000000026F790101010200000489790101A0
:1079F00001020000048B79010101020000048D796D
:107A0000010101020000048F79010101020000045C
:107A10007F79010101040000048179010101010065
:107A2000000485790101010100000486790101014A
:107A30000100000487790101010100000488790137
:107A40000101020000049179020201040000049384
:107A5000790101010200000497790101010200008F
:107A6000049979010101020000049B7901010102DE
:107A70000000049D79010101020000047F790101E9
:107A800001040000048179010101010000048579ED
:107A900001010101000004867901010101000004D7
:107AA00087790101010100000488790101010200C8
:107AB00000049F7901010102000004A17901010184
:107AC00002000004A37901010102000004A579016C
:107AD0000101020000047F7901010104000004811A
:107AE0007901010101000004857901010101000013
:107AF0000486790101010100000487790101010177
:107B0000000004887901010102000004A779010145
:107B10000102000004A97901010102000004AB790F
:107B200001010102000004AD79010101020000041D
:107B30007F79010101040000048179010101010044
:107B40000004857901010101000004867901010129
:107B50000100000487790101010100000488790017
:107B6000020100085000041A01030301030301038A
:107B70000301030401041001050000FF00020100DD
:107B8000085000041D010303010303010303010363
:107B90000401040D01050000FF000202000850006E
:107BA00004120104040103010103010303010104A0
:107BB000030104030104030104030303030103039A
:107BC0000103030103030104010103010103010592
:107BD000050000FF00020800040102040102040184
:107BE0000204010204010204010204010203010271
:107BF0000301020301020301020401020401020461
:107C00000102040102040102030102030102030153
:107C1000020401020401020401020401020401023F
:107C20000301020301020301020401020401020430
:107C30000102040102040102030102030102030123
:107C40000002020003060303060303060303060300
:107C500004180003060303060303060303060305D3
:107C60000000FF00020200041201030101030101F0
:107C700003010103010103010103010103010103E8
:107C800001010301010301010301010301010301DA
:107C900001030101030101030101040101040101C8
:107CA00004010104010104010104010104010104B2
:107CB00001010401010401010401010401010401A5
:107CC00001040101040101050000FF00020200049B
:107CD0000F0103010103010103010103010103017C
:107CE000010301010301010301010301010301017A
:107CF0000301010301010301010301010301010368
:107D00000101040101040101040101040101040154
:107D10000104010104010104010104010104010144
:107D20000401010401010401010401010401010530
:107D30000000FF00020200040C0103010103010125
:107D40000301010301010301010301010301010317
:107D50000101030101030101030101030101030109
:107D600001030101030101030101040101040101F7
:107D700004010104010104010104010104010104E1
:107D800001010401010401010401010401010401D4
:107D900001040101040101050000FF0002020008C6
:107DA000410004180000F400030501030501030568
:107DB0000103050103050103050103050103050195
:107DC000050000FF0002040000FD00083C0104055E
:107DD000010404010403010402010401000204007F
:107DE0000990000A6002030502030502030502036D
:107DF0000402030402030402030302030302030355
:107E0000020302020302020302020302020302024D
:107E1000030201050000FF00020000085500030CEA
:107E2000010402010402010402010402010402012E
:107E3000040201040201040201040201040201041B
:107E4000020104020104020104020104020105000E
:107E500000FF0002080008490000F400FF000208CB
:107E60000007A00106000100E000FF00020100077A
:107E7000900100F600FF00020500040C000720003E
:107E800000140100000400F100FF00020600040CD1
:107E90000007A00100F100FF0000005F7B00000070
:107EA000000000007C7B00000000000000997B00C7
:107EB000000000000000D47B000000000000006310
:107EC0007C00000000000000CB7C000000000000EF
:107ED00000337D000000000000009B7D00000000DA
:107EE000000000C47D00000000000000177E0000BC
:107EF0000000000000527E000000000000005D7ED7
:107F0000000000000000006B7E0000000000000088
:107F1000767E000000000000008A7E000000000065
:107F2000C00B00B0077800C00B0090487F00C10C68
:107F30000091247F04904800049124000090547F15
:107F4000045400044F7F044F00044C7F0091307FA5
:107F500004904C00049130000090547F0091247FE5
:107F600004905400004F7F044F00009124000890BB
:107F70004C7F0891307F04904C00049130000090B9
:107F8000497F0091257F04904900049125000090CD
:107F9000557F04550004507F045000044D7F00912C
:107FA000317F04904D00049131000090557F009185
:107FB000257F0490550000507F045000009125005B
:107FC00008904D7F0891317F04904D00049131005D
:107FD0000090487F0091247F049048000491240081
:107FE0000090547F045400044F7F044F00044C7FE2
:107FF0000091307F04904C00049130000090547F39
:108000000091247F04905400004F7F044F000091A2
:10801000240008904C7F0891307F04904C0004911C
:10802000300000904C7F00912B7F04904C00004D5D
:108030007F044D0000912B0000904E7F044E000401
:108040004E7F00912D7F04904E00004F7F044F0023
:1080500000912D000090507F04500004507F00914B
:108060002F7F0490500000517F04510000912F0099
:108070000090527F04520004547F0091307F0830FA
:10808000000090540000FF2F0000B0077F00C00DDB
:1080900000904C7F00B1077F00C10E0091357F003A
:1080A000BB077F01904C00004D7F084D00004C7FC6
:1080B000024C00004D7F0291350000357F063500EF
:1080C00000904D00004C7F0091357F02904C0000E5
:1080D0004D7F084D0000497F014900004A7F029111
:1080E000350000357F02904A0000487F04480000B8
:1080F00091350000904D7F0091357F06904D000036
:108100004D7F084D00009135000090507F00913563
:108110007F0290500000517F0491350000397F04A8
:108120003900003A7F053A00003B7F053B00003CE8
:108130007F053C0000905100004C7F0091357F028C
:10814000904C00004D7F084D00004C7F024C000019
:108150004D7F0291350000357F05350000904D00C0
:10816000004C7F0091357F02904C00004D7F084D00
:108170000000497F024900004A7F02913500003526
:108180007F02904A0000487F0448000091350000BB
:10819000904D7F0091357F06904D00004D7F074D3B
:1081A00000009135000090497F0091357F02904991
:1081B00000004A7F0491350000397F053900003AFC
:1081C0007F053A00003B7F053B00003C7F043C00FC
:1081D00000904A00004C7F0091357F02904C0000D7
:1081E0004D7F084D00004C7F024C00004D7F0291F6
:1081F000350000357F06350000904D00004C7F00B3
:1082000091357F02904C00004D7F084D0000497F62
:10821000014900004A7F0291350000357F02904AF3
:108220000000487F0448000091350000904D7F0019
:1082300091357F06904D00004D7F084D000091352F
:108240000000904F7F0091357F02904F0000507FDB
:108250000491350000397F0390500000517F019157
:108260003900003A7F0190510000527F04913A009A
:10827000003B7F053B00003C7F0190520000527F95
:1082800002520000537F02913C0000417F0A4100EE
:108290000090530000517F00913C7F0290510000FC
:1082A000527F03913C00003B7F043B000090520052
:1082B000004F7F00913A7F02904F0000507F039162
:1082C0003A0000387F05380000905000004D7F00D4
:1082D00091357F05350000347F05340000904D0056
:1082E000004F7F0091337F02904F0000507F079135
:1082F000330000347F02905000004C7F024C00009D
:108300004D7F0691340000357F0F904D000291356E
:108310000000FF2F00000015000000000014000105
:108320000000000900010000000600010000000438
:10833000000100010104000100000005000200002E
:108340000002000100000003000300000001000122
:10835000000101010001000101030003000000020F
:1083600000030005030302010103030502050106E2
:108370000A0C04090B02080A02020A050305050695
:108380000605040302010000000000003FFFCFFFCC
:10839000F030C0CC0C3030C0CC0C303FFFFFFFF0D1
:1083A00030CC00CC303FCFCFCFF000C0880C0000E5
:1083B000CAAA8C0000C8008C00AAE8A8AEA800C811
:1083C000008C0000CAAA8C0000C8008C003FFFCFC0
:1083D000FFF030C0CC0C303CFFFFFCF00CCC00CCEC
:1083E000C03FCFCFCFF03000CC00303FFFFFFFF0D9
:1083F0000000000000EAAAAAAAAA31555000484984
:1084000047482053434F524500505553482053543A
:1084100041525420425554544F4E003120504C414B
:10842000594552204F4E4C5900424F4E5553205003
:1084300041432D4D414E20464F5220313030303097
:1084400020505453005C2031393830204D49445776
:108450004159204D46472E20434F2E00435245445C
:108460004954202020202000494E53455254204397
:108470004F494E00434841524143544552202F201A
:108480004E49434B4E414D45002D534841444F57B3
:10849000002D535045454459002D424153484655FF
:1084A0004C002D504F4B4559005054530022424C24
:1084B000494E4B5922002250494E4B592200224925
:1084C0004E4B59220022434C5944452200001124AE
:1084D0001FBECFEFD0E1DEBFCDBF14BE88E10FB627
:1084E000F89480936000109260000FBE11E0A0E04D
:1084F000B1E0E8EFF3EF02C005900D92A438B107A8
:10850000D9F71DE0A0EAB1E001C01D92A53DB10779
:10851000E1F7F894E1E6F9E080E090E020E802C0BD
:108520002193019632E08C309307D4F381E699E0F1
:1085300090936E0B80936D0B10926F0BE2E7FBE054
:1085400080E090E003C0108201963A968430910555
:10855000D4F381E08093920B8093930B8093910BE3
:108560001092810015BCE3E1FCE080E090E020EE99
:1085700003C020830196349689309105D4F39093FB
:10858000A60B8093A50B8FEF87B984B980E88AB9D1
:108590008CE081B98BEF82B91092380986E0809324
:1085A0003909109285001092840083E0809389003D
:1085B0008DE88093880089E08093810082E0809339
:1085C0006F0082E484BD17BC91E095BD83E8809381
:1085D000B0001092B3009093B10081E185B9109280
:1085E000490910923C0910923D09109244091092D9
:1085F000430910924809109247091092A70B0E9454
:10860000664E80E00E94284680FF03C084E00E94FE
:10861000254678940E94EF4E0E946E780C94FA7969
:108620000C940000794483449144E543E6E0F9E08A
:10863000C0EAD1E02091380C0027A081B181AC0FB5
:10864000BD1F1C911283021708F4102F1C93339640
:108650000395003190F309E4005116E01A95F1F703
:108660000A95D9F716E01A95F1F700C0C0EAD1E0F3
:1086700000EEA02E662778E02DD132E23A95F1F790
:108680000E947C4330E13A95F1F700C0AA94A9F02A
:108690000000639500000000683029F0C895C89577
:1086A000C8950000E9CF662700243EE1C30FD01D26
:1086B0000000000000000000DFCFC895C895C895F5
:1086C000C895C8950000000005D10E94045411E02F
:1086D00000913B09012700933B0920913C090023AD
:1086E00009F0212720933C09E1E0E0933A09E2E018
:1086F000E093360011240895DE01679F0000009189
:108700003E0910913F0900501440000D111D180141
:1087100006E015E0000D111D280130E41EE12D9149
:1087200020316FB660FA239FA1010EF4A201040E5E
:10873000151EF001F6F0059108B92D91059108B9C3
:10874000239F059108B920316FB6059108B908F447
:10875000A201059108B960FA040E059108B9151E29
:108760001A95059108B9059139F1F00108B91EF77C
:1087700000C0019108B92D910191000008B9239F13
:108780000191000008B920316FB660FA019108B973
:108790000EF0A1010191040E08B9151E00C001914F
:1087A00008B9000000C0019108B901911A9521F0A3
:1087B000F00108B906F6DDCF08B90027C89500001A
:1087C00008B905E00A95F1F7089528980E94A24794
:1087D000E7E1EA95F1F7289AE3D0E0E0F6E0C6D0C9
:1087E000E0FF05D0E0FF02C00E94C7460895EF9366
:1087F000E0913909E93EE0F5E930D0F12F923F925E
:108800004F925F926F927F928F929F92AF92BF92A0
:10881000CF92DF92EF92FF920F931F932F933F938C
:108820004F935F936F937F938F939F93AF93BF9378
:10883000CF93DF930E941643DF91CF91BF91AF9109
:108840009F918F917F916F915F914F913F912F9168
:108850001F910F91FF90EF90DF90CF90BF90AF905E
:108860009F908F907F906F905F904F903F902F9050
:10887000EF910895FF93EF93EFB7EF93E0918400AA
:10888000EE50E13000F0E23000F0E33000F0E43090
:1088900000F0E53000F0E63000F0E73000F0E830BE
:1088A00000F0E93000F005D0EF91EFBFEF91FF91BC
:1088B00018950F921F92E4E2F6E800903809000C38
:1088C0001124E00DF11D05901490F00109951F9001
:1088D0000F90089528980E94A247E5E1EA95F1F7E4
:1088E000E0913909EA95E0933909289A00000000DF
:1088F000089528980E94CB47289A0000E1E0F6E00E
:1089000035D047D0089528980E94CB47E0EB00006F
:10891000EA95E9F700000000289AF6E0E2E026D0A8
:10892000089528980E94CB47289A0000E3E0FDEFC5
:108930001DD0E0913909E53091F4E0913B09E13037
:108940000000F091490919F4F0914909F195E3E02B
:10895000E0938900EDE8EF0FE09388000895E3E0ED
:10896000E0938900EDE8E0938800089500903909CC
:108970000A9410905F0011FC0F2E009239090090AC
:10898000380911FC0E2E00923809E0E011FCE1E0FC
:108990000895E3E0E0938900EDE8E093880008950E
:1089A000E7E0E0938900EBE1E09388000895E6E6D4
:1089B000F3E0A0EAB1E060E16D933197E9F71124AB
:1089C0000895CC03CC03CC03CC03CC03CC03CC0361
:1089D000CC03CC03CC03CC03CC03CC03CC03CC031F
:1089E000CC03CC03CC03CC03CC03CC03CC03CC030F
:1089F000CC03CC03CC03CC03CC03CC03CC03CC03FF
:108A0000CC03CC03CC03CC03CC03CC03CC03CC03EE
:108A1000CC03CC03CC03CC03CC03CC03CC03CC03DE
:108A2000CC03CC03CC03992777272EE1629F080E55
:108A3000191EA0EAB1E0A00DB11D405F4C931124B6
:108A40000895089599272EE1629F080E191EA0EA45
:108A5000B1E0A00DB11D50914009450F4C93112478
:108A600008958093400908958093360990933709BB
:108A7000089580933E0990933F09089580913A09A3
:108A80000895112410923A09089580E891E08093A6
:108A9000610090936100089580E890E08093610008
:108AA00090936100089520E4E0913E09F0913F0920
:108AB0008051829FE00DF11DA6E0B5E0629FA00D00
:108AC000B11D002405900D9205900D9205900D9218
:108AD00005900D9205900D9205900D9205900D92C6
:108AE00005900D9205900D9205900D9205900D92B6
:108AF00005900D9205900D9205900D9205900D92A6
:108B000005900D9205900D9205900D9205900D9295
:108B100005900D9205900D9205900D9205900D9285
:108B200005900D9205900D9205900D9205900D9275
:108B300005900D9205900D9205900D9205900D9265
:108B400005900D9205900D9205900D9205900D9255
:108B500005900D9205900D9205900D9205900D9245
:108B600005900D9205900D9205900D9205900D9235
:108B700005900D9205900D9205900D9205900D9225
:108B800005900D9205900D9205900D9205900D9215
:108B900005900D9205900D9205900D9205900D9205
:108BA00005900D9205900D9205900D9205900D92F5
:108BB00005900D9205900D9205900D9205900D92E5
:108BC00005900D921124089594E0899FE2E1FCE064
:108BD000E00DF11D8281E0913609F091370990E4B2
:108BE000899FE00DF11DA6E0B5E0699FA00DB11DC4
:108BF0001124403021F4A20FB11D822F04C088E05F
:108C0000821BE80FF11D503031F498E0939FA00DC6
:108C1000B11D932F06C098E0931B58E0599FE00DBB
:108C2000F11D11243EEF58E0591B48E0481B2591E7
:108C300023132C9311964A95D1F7E80FF11DA80F35
:108C4000B11D5A9591F7112408958093490908950B
:108C5000882329F4809141099091420908958091D7
:108C60004509909146090895882329F48091430984
:108C70009091440908958091470990914809089579
:108C800078E07A95F1F700000197D1F70895F99906
:108C9000FECF92BD81BD60BDF894FA9AF99A78949E
:108CA0000895F999FECF92BD81BDF894F89A80B5E8
:108CB000789408950000000000000000000000000B
:108CC00000000000000000000000000000000000A4
:108CD0000000000000000000000000000000000094
:108CE0000000000000000000000000000000000084
:108CF0000000000000000000000000000000000074
:108D000099277727833008F00895E0E0FAE9660FA5
:108D1000771FE60FF71FA591B491E2E7FBE02AE089
:108D2000289FE00DF11DA183B28311240895909135
:108D3000910B9170880F892B8093910B089599273F
:108D40007727E2E7FBE02AE0289FE00DF11D6E3F68
:108D500031F46091910B6E7F6093910B0BC06F3F6C
:108D600031F46091910B6E6F6093910B03C070E9C9
:108D7000760F75831124089599277727E2E7FBE0A2
:108D80002AE0289FE00DF11D6083112408952F93A0
:108D90003F934F935F936F937F938F939F93AF9383
:108DA000BF93789411240E9494540E94CF540E943F
:108DB000AF4E0E94E8502F923F924F925F926F9277
:108DC0007F928F929F92AF92BF92CF92DF92EF925B
:108DD000FF920F931F93CF93DF9300906F0B0020B0
:108DE00019F4A1E6B9E002C0A7E6BAE001E0002666
:108DF00000926F0B02E00093700B5091900B60910A
:108E0000920B7091930B8091940B2090730B309088
:108E1000740B4090760B5090770B6090750B10910F
:108E2000720B70907D0B80907E0B90907F0BA090CA
:108E3000800BB090810B20917C0BC090870BD09061
:108E4000880BE0908A0BF0908B0B0091890B30918E
:108E5000860B9FEF620C431CF201449141030024F6
:108E60000008C12DD02D970CA81CF5014491420398
:108E700000240008C10DD01D0C0DED1CF70144911C
:108E8000430300240008C10DD01D8A956AF4409167
:108E9000910B842F8695062E0694062600FA769569
:108EA000679576F940FF66F940E860FD4FE74503B6
:108EB00000240008C10DD01D0024C038D0050CF0DE
:108EC000CFE70A94C038D0050CF4C0E8C058CD9361
:108ED0009A9509F0BFCF4091700B4A954093700B63
:108EE00097E009F0B7CF6092750B4092760B9092A5
:108EF0007F0BA092800B0093890BE0928A0B60930A
:108F0000920B7093930B8093940BDF91CF911F91F1
:108F10000F91FF90EF90DF90CF90BF90AF909F9018
:108F20008F907F906F905F904F903F902F90BF9168
:108F3000AF919F918F917F916F915F914F913F91F1
:108F40002F9108950C94A4470C94A6470F931F9358
:108F50002ABDE0916D0BF0916E0B01910000009322
:108F6000B3000BE0ED36F00710F40000000010F045
:108F7000E1E6F9E0E0936D0BF0936E0BC895C895B0
:108F8000C895C895C895C8950000000000002AB58E
:108F90001F910F9108950000E0913909E0FFD6CFAD
:108FA000E1E1EA95F1F700000000089500000000FB
:108FB00000000000000000000000000000000000B1
:108FC00000000000000000000000000000000000A1
:108FD0000000000000000000000000000000000091
:108FE0000000000000000000000000000000000081
:108FF0000000000000000000000000000000000071
:10900000000306090C101316191C1F2225282B2EED
:10901000313336393C3F414447494C4E5153555802
:109020005A5C5E60626466686A6B6D6F70717374BF
:10903000757678797A7A7B7C7D7D7E7E7E7F7F7F78
:109040007F7F7F7F7E7E7E7D7D7C7B7A7A7978765E
:1090500075747371706F6D6B6A68666462605E5C74
:109060005A585553514E4C494744413F3C39363389
:10907000312E2B2825221F1C191613100C0906034C
:1090800000FDFAF7F4F0EDEAE7E4E1DEDBD8D5D253
:10909000CFCDCAC7C4C1BFBCB9B7B4B2AFADABA81E
:1090A000A6A4A2A09E9C9A9896959391908F8D8C41
:1090B0008B8A888786868584838382828281818168
:1090C0008181818182828283838485868687888A62
:1090D0008B8C8D8F9091939596989A9C9EA0A2A42C
:1090E000A6A8ABADAFB2B4B7B9BCBFC1C4C7CACDF7
:1090F000CFD2D5D8DBDEE1E4E7EAEDF0F4F7FAFD14
:10910000808182838485868788898A8B8C8D8E8FE7
:10911000909192939495969798999A9B9C9D9E9FD7
:10912000A0A1A2A3A4A5A6A7A8A9AAABACADAEAFC7
:10913000B0B1B2B3B4B5B6B7B8B9BABBBCBDBEBFB7
:10914000C0C1C2C3C4C5C6C7C8C9CACBCCCDCECFA7
:10915000D0D1D2D3D4D5D6D7D8D9DADBDCDDDEDF97
:10916000E0E1E2E3E4E5E6E7E8E9EAEBECEDEEEF87
:10917000F0F1F2F3F4F5F6F7F8F9FAFBFCFDFEFF77
:10918000000102030405060708090A0B0C0D0E0F67
:10919000101112131415161718191A1B1C1D1E1F57
:1091A000202122232425262728292A2B2C2D2E2F47
:1091B000303132333435363738393A3B3C3D3E3F37
:1091C000404142434445464748494A4B4C4D4E4F27
:1091D000505152535455565758595A5B5C5D5E5F17
:1091E000606162636465666768696A6B6C6D6E6F07
:1091F000707172737475767778797A7B7C7D7E7FF7
:1092000000020406080A0C0E10121416181A1C1E6E
:1092100020222426282A2C2E30323436383A3C3E5E
:1092200040424446484A4C4E50525456585A5C5E4E
:1092300060626466686A6C6E70727476787A7C7E3E
:109240007F7D7B79777573716F6D6B69676563611E
:109250005F5D5B59575553514F4D4B49474543410E
:109260003F3D3B39373533312F2D2B2927252321FE
:109270001F1D1B19171513110F0D0B0907050301EE
:10928000FFFDFBF9F7F5F3F1EFEDEBE9E7E5E3E1DE
:10929000DFDDDBD9D7D5D3D1CFCDCBC9C7C5C3C1CE
:1092A000BFBDBBB9B7B5B3B1AFADABA9A7A5A3A1BE
:1092B0009F9D9B99979593918F8D8B8987858381AE
:1092C00080828486888A8C8E90929496989A9C9EAE
:1092D000A0A2A4A6A8AAACAEB0B2B4B6B8BABCBE9E
:1092E000C0C2C4C6C8CACCCED0D2D4D6D8DADCDE8E
:1092F000E0E2E4E6E8EAECEEF0F2F4F6F8FAFCFE7E
:109300007F7F7F7F7F7F7F7F7F7F7F7F7F7F7F7F6D
:109310007F7F7F7F7F7F7F7F7F7F7F7F7F7F7F7F5D
:109320007F7F7F7F7F7F7F7F7F7F7F7F7F7F7F7F4D
:109330007F7F7F7F7F7F7F7F7F7F7F7F7F7F7F7F3D
:109600000309131E28313A40464C5054585B5E61A2
:10961000636567696B6C6E6F707172737475767762
:10962000777879797A7A7B7B7C7C7C7D7D7D7E7E88
:109630007E7E7F7F7F7F7F7F7F7F7F7F7F7F7F7F3C
:109640007F7F7F7F7F7F7F7F7F7F7F7F7F7E7E7E2D
:109650007E7D7D7D7C7C7C7B7B7A7A79797877775F
:10966000767574737271706F6E6C6B696765636128
:109670005E5B5854504C46403A31281E1309030093
:10968000C6CCD5DBDFE3E5E7E9EAEBECEDEEEFEFA7
:10969000F0F0F0F1F1F1F1F2F2F2F2F2F2F2F2F3B3
:1096A000F3F3F3F3F3F3F3F3F3F3F3F3F3F3F3F38A
:1096B000F3F3F3F3F3F3F3F3F3F3F3F3F3F3F3F37A
:1096C000F3F3F3F3F3F3F3F3F3F3F3F3F3F3F3F36A
:1096D000F3F3F3F3F3F3F3F3F3F3F3F3F3F3F3F35A
:1096E000F2F2F2F2F2F2F2F2F1F1F1F1F0F0F0EF67
:1096F000EFEEEDECEBEAE9E7E5E3DFDBD5CCC60026
:1097000000283D42302D2C2B2C2D2E2F303233357E
:1097100037393B3D3F414345484A4C4E50535557DE
:10972000595B5D5F61636567696B6C6E70717374C3
:10973000757778797A7B7C7D7D7E7E7F7F7F7F7F6A
:109740007F7F7F7F7F7F7E7E7D7D7C7B7A79787750
:1097500075747371706E6C6B69676563615F5D5B77
:1097600059575553504E4C4A484543413F3D3B396C
:1097700037353332302F2E2D2C2B2C2D30423D28D7
:1097800000E9E5FED4D7D7D7D6D4D2D0CECCCAC83C
:10979000C6C3C1BFBDBAB8B6B4B1AFADABA9A7A57A
:1097A000A3A19F9E9C9A999795949391908F8D8C4D
:1097B0008B8A89888887868585848484838383834C
:1097C0008383838383848484858586878888898A44
:1097D0008B8C8D8F909193949597999A9C9E9FA135
:1097E000A3A5A7A9ABADAFB1B4B6B8BABDBFC1C34D
:1097F000C6C8CACCCED0D2D4D6D7D7D7D4FEE5E906
:10980000F9F8F9F5EBE1DDDEE0E2E4E5E6E5E4E2D6
:10981000DED9D2CAC1B7ACA299918A8683818080F1
:109820008182838586888A8C8D8F90929395969776
:1098300098999A9B9B9C9D9D9D9E9E9E9F9F9F9F5E
:109840009F9F9F9E9E9E9D9D9D9C9B9B9A99989756
:1098500096959392908F8D8C8A888685838281805D
:10986000808183868A9199A2ACB7C1CAD2D9DEE23F
:10987000E4E5E6E5E4E2E0DEDDE1EBF5F9F8F90048
:109880000708070B151F2322201E1C1B1A1B1C1E5A
:1098900022272E363F49545E676F767A7E7F7F7F20
:1098A0007F7E7D7B7A7876747371706E6D6B6A697A
:1098B0006867666565646463636262626161616171
:1098C000616161626262636363646565666768695A
:1098D0006A6B6D6E7071737476787A7B7D7E7F7F34
:1098E0007F7F7E7A766F675E54493F362E27221E31
:1098F0001C1B1A1B1C1E2022231F150B0708070008
:109900001F313D444E5354565A5F64696E747679E4
:109910007C7F7F7F7F7F7F7F7F7F7F7F7F7F7F7F5A
:109920007F7F7F7F7F7F7F7F7F7F7F7F7F7F7F7F47
:109930007F7F7F7F7F7F7F7F7F7F7F7F7F7F7F7F37
:109940007F7F7F7F7F7F7F7F7F7F7F7F7F7F7F7F27
:109950007F7F7F7F7F7F7F7F7F7F7F7F7F7F7F7F17
:109960007F7F7F7F7F7F7F7F7F7F7F7F7F7F7F7F07
:109970007F7F7F7F7F7F7F7F7F7F7F7C7871684C59
:109980002C1C120C0A0B0A05FDF3E9DFD4CAC0B780
:10999000AEA69E97918B8685828080808080808015
:1099A00080808080808080808080808080808080B7
:1099B00080808080808080808080808080808080A7
:1099C0008080808080808080808080808080808097
:1099D0008080808080808080808080808080808087
:1099E0008080808080808080808080808080808077
:1099F000808080808087919DACC4CBD4DDF2FAFA60
:109A000022002400260028002B002D003000330007
:109A1000360039003D004000440048004C00510031
:109A200056005B00600066006C00730079008100E6
:109A3000880090009900A200AC00B600C100CC00E4
:109A4000D800E500F30001011001210132014401B9
:109A500057016C0181019801B001CA01E5010202C0
:109A60002102410264028802AE02D70203033003DE
:109A700061039403CB03050442048304C704100567
:109A80005D05AF0505066106C206290796070908A8
:109A9000830805098E09200ABA0A5D0B0A0CC10C5D
:109AA000840D510E2B0F121007110A121D134014B2
:109AB0007415BA1614188319071BA31C571E2420EB
:109AC0000E22142439267F28E82A752D29300633E2
:109AD0000F364539AD3C49401B442848734CFE5075
:109AE000CF55EA5A51600C661D6C8B725A79928080
:109AF00037885090E598FDA19FABD3B5A3C0000077
:109B0000FB01DC0102C005900D9241505040D8F796
:109B100008951F9380E090E00E945146182F81E045
:109B200090E00E94514690E0382F20E0210F311D37
:109B30002A55354509F491E0892F1F910895BF9268
:109B4000CF92DF92EF92FF920F931F93CF93DF9309
:109B50006C01062FB72E0E94894D8823F1F18FEFFB
:109B6000C8168FEFD80611F481E03AC0EE24FF2426
:109B7000C7010E945146182FC70101960E94514605
:109B8000D82FC0E0CE01810F911D8C159D0521F4C9
:109B9000E114F10459F423C080E290E0E80EF91ECC
:109BA00090E0E91694E0F90619F719C0802F9B2D73
:109BB0009C01E90180E2C82ED12CC20ED31E870180
:109BC0000F5F1F4FC7010E9451468993CC15DD05D9
:109BD00011F480E005C07801F2CF84E001C083E099
:109BE000DF91CF911F910F91FF90EF90DF90CF9079
:109BF000BF900895BF92CF92DF92EF92FF920F93A2
:109C00001F93CF93DF936C010E94894D882311F439
:109C100084E04EC0F60180819181FFEF8F3F9F0766
:109C200009F445C08A55954509F441C002E010E0A9
:109C300020E4E22EF12CC7010E945146B82EC70144
:109C400001960E945146D82FC0E09E012B0D311D78
:109C5000F601808191812817390719F41123B1F099
:109C60000EC02F5F3F4F19F4112309F4102F0F5F1F
:109C700080E290E0E80EF91E0034E9F623C0E12E00
:109C8000FF2495E0EE0CFF1C9A95E1F7C0E0D0E0D0
:109C9000F601EC0FFD1FCE018E0D9F1D60810E940D
:109CA00047462196C032D10599F780E001C081E096
:109CB000DF91CF911F910F91FF90EF90DF90CF90A8
:109CC000BF9008951123D9F682E0F2CFFF920F934F
:109CD0001F93CF93DF93129A8091A70B882329F0CB
:109CE00081E090E00E94404602C0C895C895129855
:109CF00000E010E0C0E0D0E0FF2416950795D6956F
:109D0000C79513988091A70B882329F085E090E0F0
:109D10000E94404602C0C895C895009B1068019BF0
:109D2000D068139A8091A70B882329F085E090E0F2
:109D30000E94404602C0C895C895F39480E1F81689
:109D4000E1F61093420900934109D0934609C0936C
:109D50004509DF91CF911F910F91FF900895FF92D8
:109D60000F931F93CF93DF930E94664E809141091A
:109D70009091420997FD06C080914509909146094E
:109D800097FF27C081E090E00E94404600E010E08D
:109D9000C0E0D0E0FF24000F111FCC0FDD1F13988F
:109DA000C895C895C895C895009B0160019BC16086
:109DB000139A88E090E00E944046F39480E1F81600
:109DC00051F71093440900934309D0934809C09375
:109DD0004709DF91CF911F910F91FF9008950F9345
:109DE0001F9302ED18E0C8010E948C4F84E990E0B7
:109DF0000E9439450E94D7448FE090E00E94B854F9
:109E0000C8010E948C4F80E06FEF41E00E944153F7
:109E100004E918E08DE06CE0A8010E941E5483E084
:109E200090E00E94B8548DE06CE04AEA58E00E944D
:109E30001E5482E090E00E94B8548DE06CE0A801CE
:109E40000E941E5484E190E00E94B8548AE090E0A1
:109E50000E94B8540E94D74484E190E00E94B85414
:109E60001F910F91089590E026E130E0829FF0016C
:109E7000839FF00D929FF00D1124E655F44F6287F9
:109E800008956093910B089590E026E130E0829F61
:109E9000F001839FF00D929FF00D1124E655F44FD1
:109EA00013861182089590E026E130E0829FF00150
:109EB000839FF00D929FF00D1124E655F44F81E041
:109EC000838B089590E026E130E0829FF001839F2C
:109ED000F00D929FF00D1124E655F44F618708951F
:109EE00090E026E130E0829FF001839FF00D929F89
:109EF000F00D1124E655F44F6483089590E026E1B7
:109F000030E0829FF001839FF00D929FF00D1124AD
:109F1000E655F44F658308959093050C8093040CE7
:109F20008FE680930A0C10926009EAEAFBE021E0D8
:109F30008FEF98E1208310868683878314861182B1
:109F4000958376963CE0E230F307A1F708951092EE
:109F5000AB0B1092C10B1092D70B1092ED0B019628
:109F600090930E0C80930D0C9093A90B8093A80BEB
:109F70009093110C8093100C10920C0C10920B0CFF
:109F80001092030C1092020C1092060C81E0809348
:109F900060091092090C1092080C08958091B40B7E
:109FA00087FD03C08AEF8093B40B8091CA0B87FDB5
:109FB00003C08AEF8093CA0B8091E00B87FD03C03A
:109FC0008AEF8093E00B8091F60B87FD03C08AEF48
:109FD0008093F60B109260090895DC01ED91FC91DD
:109FE0001197AF014F5F5F4F11965C934E93E491D1
:109FF0002E2F30E0E7FF13C02F7730703695322FC9
:10A00000222737952795FA014F5F5F4FE4918E2FF6
:10A010008F77280F311DE7FDF1CF4D935C93C90178
:10A02000089580930A0C08950E949F460895EF9228
:10A03000FF920F931F93CF93DF93182F062FF42EC9
:10A04000E22EC82FD0E086E190E0C89FF001C99FC2
:10A05000F00DD89FF00D1124E655F44F8385882329
:10A0600021F08181882309F0ACC0EE2091F486E1D3
:10A0700090E0C89FF001C99FF00DD89FF00D11240A
:10A08000E655F44F138A8285882309F09AC010861A
:10A0900098C0133059F481E091E09093930B809332
:10A0A000920B81E08093910B0F2D08C0812F60E00F
:10A0B0000E949F46812F6F2D0E9480460F3799F492
:10A0C00086E190E0C89FF001C99FF00DD89FF00D88
:10A0D0001124E655F44F8091070C878788E09CE0B7
:10A0E000958B848B30C089E0089FC0011124E091DA
:10A0F000040CF091050CE80FF91F3396459154912B
:10A100004115510571F486E190E0C89FF001C99FA7
:10A11000F00DD89FF00D1124E655F44F158A148ADE
:10A1200012C0FA01249186E190E0C89FF001C99F16
:10A13000F00DD89FF00D1124E655F44F27874F5F9F
:10A140005F4F558B448B86E190E0C89FD001C99F3B
:10A15000B00DD89FB00D1124A655B44F50961C9247
:10A1600050971A961C921A971C960C931C9711964E
:10A170001C9211972FEF19962C9319971896EC9221
:10A1800018978BE090E0C89FF001C99FF00DD89F11
:10A19000F00D1124EE0FFF1FE455F44FF08251969D
:10A1A0001C92519781E01B968C931B9753961C929F
:10A1B000539752961C92529714961C921497169687
:10A1C0002C93DF91CF911F910F91FF90EF90089505
:10A1D000CF92DF92FF920F931F93CF93DF93E3EB26
:10A1E000FBE08181282F332727FD30958081280FC0
:10A1F000311D2F3F310519F014F02FEF30E0C90168
:10A2000037FF02C080E090E0808376964CE0EB3030
:10A21000F40739F780916009882309F028C144C107
:10A22000E0910D0CF0910E0C9F012F5F3F4F30938A
:10A230000E0C20930D0C44914F3F69F5A9014F5F1F
:10A240005F4F50930E0C40930D0CF90184918F32A7
:10A2500019F41092600919C1863009F0FBC0FA01A7
:10A260003196CF01019690930E0C80930D0CE491E2
:10A27000E33529F49093110C8093100CEBC0E53476
:10A2800009F0E8C08091100C9091110C90930E0C85
:10A2900080930D0CDFC047FF02C04093060C542F83
:10A2A0005F70842F90E0807F9070803B910531F14A
:10A2B000803C910581F18039910509F043C0C901C5
:10A2C0000196F9014491019690930E0C80930D0C28
:10A2D0000197FC012491852F90E08C9FF0018D9FC8
:10A2E000F00D9C9FF00D1124E655F44F80818823DA
:10A2F00009F4B0C0220F852F648553C0C9010196AF
:10A30000F9014491019690930E0C80930D0C0197E6
:10A31000FC01249153C02F5F3F4F30930E0C2093CC
:10A320000D0C21503040F9012491852F90E08C9F35
:10A33000F0018D9FF00D9C9FF00D1124E655F44F18
:10A34000248788C08091060C582F5F7090E0807F32
:10A350009070803B910541F1803C910509F46EC0FD
:10A360008039910509F076C02F5F3F4F30930E0C76
:10A3700020930D0C21503040F9012491852F90E05D
:10A380008C9FD0018D9FB00D9C9FB00D1124A655C0
:10A39000B44F8C91882309F45DC0220F852F1C9641
:10A3A0006C910E94175056C02F5F3F4F30930E0C98
:10A3B00020930D0C21503040F9012491473071F465
:10A3C000852F90E08C9FF0018D9FF00D9C9FF00DEC
:10A3D0001124E655F44F220F27833CC04B3071F413
:10A3E000852F90E08C9FF0018D9FF00D9C9FF00DCC
:10A3F0001124E655F44F220F26832CC04C3571F4FE
:10A40000852F90E08C9FF0018D9FF00D9C9FF00DAB
:10A410001124E655F44F220F24831CC04436D1F496
:10A42000852F90E08C9FF0018D9FF00D9C9FF00D8B
:10A430001124E655F44F220F25830CC0852F90E0A0
:10A440008C9FF0018D9FF00D9C9FF00D1124E6551F
:10A45000F44F44878DE09CE00E94ED4F90930C0CEC
:10A4600080930B0C1092030C1092020C02C0C6E1F8
:10A47000D0E06091020C7091030C80910B0C9091D4
:10A480000C0C6817790709F4CBCE6F5F7F4F709380
:10A49000030C6093020C8091080C9091090C0196BA
:10A4A0009093090C8093080C02E71BE0CBEADBE0F9
:10A4B000FF24BFEFCB2ED12C8A89882309F05EC000
:10A4C0008B899C89892B09F456C09F858E859817A6
:10A4D00008F04CC050C08B852B893C898F37E9F43C
:10A4E000D9018D91BC8BAB8B8F3F01F1F90161815B
:10A4F0001196BC8BAB8BE82FF0E0EE0FFF1FE552FF
:10A50000F74F0190F081E02D8F2D0995EB89FC89A3
:10A5100081918E87FC8BEB8B28C0A9014F5F5F4F29
:10A520005C8B4B8BF90184918F3F21F418821C8A3C
:10A530001B8A21C04F5F5F4F5C8B4B8B415050405B
:10A54000FA01649190E0880F991F8552974FFC01A2
:10A55000259134918F2DF9010995EB89FC8931966C
:10A56000FC8BEB8B3197E491EE871F869F858E8560
:10A57000981709F4B0CF8F858F5F8F878A858823DE
:10A5800019F420E030E06BC088898F3F11F08F5FB5
:10A59000888B9F81992309F45CC02885222309F4C4
:10A5A00058C08E81882309F454C040910A0C44237A
:10A5B00009F44FC0899FC001112480509F4F892FFB
:10A5C000992730E0B901869F9001879F300D969FB3
:10A5D000300D112420503F4F232F33278D8190E0E1
:10A5E000FC012E9FC0012F9F900D3E9F900D1124C6
:10A5F00080509F4F892F9927242F30E0AC01429F34
:10A60000C001439F900D529F900D112480509F4F89
:10A61000292F33278B818823F1F0EA81F0E0E05085
:10A62000F047E491E058E89FC001112480509F4F0B
:10A63000892F9927B601681B790B629FC001639F20
:10A64000900D729F900D112480509F4F292F33271A
:10A6500002C020E030E08A819C81890F8A83F80162
:10A660002083F394065F1F4F6696F4E0FF1609F00F
:10A6700023CFDF91CF911F910F91FF90DF90CF906B
:10A6800008951F93CF93DF93582F89E0589FC001FF
:10A6900011242091040C3091050C280F391FC90199
:10A6A0000396FC01A591B491F90184918150823007
:10A6B00010F413E01DC08091C10B8823B1F080918C
:10A6C000CD0B851711F4442381F48091D70B882397
:10A6D00071F08091E30B851711F4442341F49091BC
:10A6E000D10B8091E70B891710F411E001C012E043
:10A6F000212F30E0FD01449186E190E0289FE001A8
:10A70000299FD00D389FD00D1124C655D44F4F87A7
:10A710001196BD8BAC8B188A8BE090E0289FF001DE
:10A72000299FF00D389FF00D1124EE0FFF1FE45507
:10A73000F44F80E5808368878FEF89871A861B8AAC
:10A74000198A21E02B871A8A5D8729831C828E83D0
:10A75000133049F481E091E09093930B8093920B36
:10A760002093910B08C0812F60E50E948046812FC5
:10A770006A890E949F46DF91CF911F910895FF92B1
:10A780000F931F93082FF62E0E94804610E08BE057
:10A7900090E0089FF001099FF00D189FF00D112423
:10A7A000EE0FFF1FE455F44FF0821F910F91FF90C1
:10A7B0000895962F482F50E02BE030E0429FF001A3
:10A7C000439FF00D529FF00D1124EE0FFF1FE45533
:10A7D000F44F6081691B60830E9480460895482F72
:10A7E00050E02BE030E0429FF001439FF00D529F7C
:10A7F000F00D1124EE0FFF1FE455F44F9081690F07
:10A8000060830E94804608953091380C20E010C08B
:10A81000822F90E0FC01EE0FFF1FE80FF91FEA5FA7
:10A82000F64FA081B181A056BE4F82818C932F5FDD
:10A83000231770F308958093000108951F93CF9319
:10A84000DF93FA01749131961491C72FD0E0AF01D4
:10A850004F5F5F4F9EE1699F90011124280F311DCA
:10A8600060E00CC08491805F8D939F5F3196971755
:10A87000C8F36F5F4C0F5D1F225E3F4F611730F4CE
:10A88000D901A056BE4FFA0190E0F1CFDF91CF91F0
:10A890001F9108951F93CF93DF93A82FFB0174910D
:10A8A0003196B491C72FD0E0AF014F5F5F4F60E0AA
:10A8B00016C0F9018491E12FF0E0EE0FFF1FEE0FBB
:10A8C000FF1FEC5EF34F80839F5F2F5F3F4F192F79
:10A8D0001A0F971770F3A70F6F5F4C0F5D1F6B1761
:10A8E00018F49A0190E0F3CFDF91CF911F91089572
:10A8F0000F9350E012C0F0E0EE0FFF1FEE0FFF1FAE
:10A90000EE5EF34F308341839F5F385FE92FE80F9E
:10A91000921788F3820F5F5F485F501718F4362F45
:10A9200090E0F4CF0F9108958091390C8823F9F0CD
:10A9300080913A0C8823C1F48091360C80933A0CB4
:10A9400090913B0CE92FF0E0E050FF4F808187B9F8
:10A950008091370C890F80933B0C882311F08D3048
:10A9600031F41092390C0895815080933A0C089577
:10A970000F931F93CF93DF938C01C0E0D0E007C00B
:10A980000E943E458823E1F30E9441452196C0176D
:10A99000D107B4F3DF91CF911F910F9108952F92BA
:10A9A0003F924F925F926F927F928F929F92AF925F
:10A9B000BF92CF92DF92EF92FF920F931F93DF939C
:10A9C000CF9300D00F92CDB7DEB71092380C8091A4
:10A9D0000001882309F49AC052E1852E5CE0952E8F
:10A9E0007724F4019181903E08F071C08081382F66
:10A9F000369536953695282F277019F0F2E0F983B1
:10AA000002C081E08983892F869586958695977007
:10AA100019F042E0642E02C066246394B92EAA2481
:10AA20001501220E311C9EE1899F80011124030F24
:10AA3000111DCC24DD2440C04A815B81400F511F91
:10AA4000F70160816031F0F02091380C203110F571
:10AA5000822F90E0FC01EE0FFF1FE80FF91FEA5F65
:10AA6000F64F518340836283862F622F0E945345A5
:10AA70006091380CF70160836F5F6093380C615010
:10AA8000603140F44A815B81440D551D872D910151
:10AA90000E94E4458A819B8101969B838A83089466
:10AAA000E11CF11C9981891738F20894C11CD11C52
:10AAB000025E1F4FC61458F45C2C442480EAE82E32
:10AAC00081E0F82EE00EF11E1B821A82B5CF73943E
:10AAD000E4E0F0E08E0E9F1EF9E07F1609F081CFD2
:10AAE0003091380C20E010C0822F90E0FC01EE0F76
:10AAF000FF1FE80FF91FEA5FF64FA081B181A05652
:10AB0000BE4F82818C932F5F231770F30F900F90AD
:10AB10000F90CF91DF911F910F91FF90EF90DF90F9
:10AB2000CF90BF90AF909F908F907F906F905F90ED
:10AB30004F903F902F9008951F93FC01162F009780
:10AB400019F460E070E034C08530910518F461E0DC
:10AB500070E015C08131910518F462E070E00FC01B
:10AB60008134910518F463E070E009C081E0E130C0
:10AB7000F80718F065E070E002C064E070E09F0143
:10AB800002C0369527956A95E2F72115310511F433
:10AB900021E030E040E009C0CF01B9010E94B17965
:10ABA000260F371F369527954F5F4117A8F3B90138
:10ABB000CB011F910895282F8091440C82FF0DC076
:10ABC000222319F080E090E0089520E0903109F010
:10ABD00021E081E02827822F0895213011F02131D2
:10ABE00089F4933019F481E090E00895213011F058
:10ABF000213141F420E030E0903111F421E030E0E7
:10AC0000C901089580E090E008958091880C893012
:10AC100048F48630A8F4823069F0833078F48130CB
:10AC2000B9F40AC08F3018F48C3070F40BC0833143
:10AC300078F40CC083E10DC08CE00BC089E109C041
:10AC400080E207C086E205C083E303C080E401C060
:10AC50008DE49091890C981719F08695981729F42E
:10AC600080913C0C816080933C0C08958091880C0D
:10AC700090E0FC013197E231F105F0F4E85CFF4F20
:10AC8000EE0FFF1F0590F491E02D099486E090E00F
:10AC900002C085E090E09093940C8093930C10C0D8
:10ACA00084E090E0F8CF83E090E0F5CF82E090E0A0
:10ACB000F2CF81E090E0EFCF1092940C1092930CC1
:10ACC0008091930C9091940C2CE330E0AC01429F66
:10ACD000C001439F900D529F900D11249093940CAE
:10ACE0008093930C08958091880C8E3048F48C30BA
:10ACF00070F4893061F08A3060F4813060F009C00E
:10AD0000813118F48F3018F404C0823121F483E0CB
:10AD1000089585E0089580E008952091910C309188
:10AD2000920C81E02039380751F083E02032380757
:10AD300069F0283C310569F486E099E702C08AE0B1
:10AD400099E790934A0C8093490C10C08EE099E7E4
:10AD5000F8CF82E099E790934A0C8093490C86E003
:10AD60002034380719F488EC90E003C0C901880F3B
:10AD7000991F9093920C8093910C08956091450CCB
:10AD800063FD35C050910B0D852F8E7081F5A0911C
:10AD9000030D7091040DE5E3FDE040E08085282F70
:10ADA00030E0C90184719070892BE9F480818A17A1
:10ADB000D1F481818717B9F42A703070232B21F4E4
:10ADC0008091460C80FF0AC08091460C80FD09C02E
:10ADD00040934E0C64606093450C03C052605093E6
:10ADE0000B0D81E008954F5FB7964430B9F680E0CF
:10ADF0000895FC018091210D882321F4138215828E
:10AE0000808181838181882359F4838192818F5F3E
:10AE100083838150891769F4138281E081830895C7
:10AE2000858194818F5F85838150891711F4158204
:10AE3000118208952091880C213009F04EC0809134
:10AE40002B0D90912C0DA0912D0DB0912E0D813BCD
:10AE500023E1920720E0A20720E0B20708F0ACC08F
:10AE6000843526E0920720E0A20720E0B20709F42B
:10AE70009EC0883A2CE0920720E0A20720E0B207AB
:10AE800009F495C0843822E1920720E0A20720E06F
:10AE9000B20709F48CC0843A21E0920720E0A207AF
:10AEA00020E0B20709F485C0883F27E0920720E040
:10AEB000A20720E0B20709F47CC0843D2DE0920790
:10AEC00020E0A20720E0B20709F473C0805B934141
:10AED000A040B04009F070C06CC080912B0D9091E3
:10AEE0002C0DA0912D0DB0912E0D253090F5853DA6
:10AEF0002DE0920720E0A20720E0B20708F05CC036
:10AF0000843526E0920720E0A20720E0B20709F48A
:10AF10004EC0883A2CE0920720E0A20720E0B2075A
:10AF200009F445C0843A21E0920720E0A20720E01E
:10AF3000B20709F43EC0883F27E0920720E0A2074D
:10AF400020E0B207B1F1845D9D40A040B040A1F582
:10AF500030C0853E2CE0920720E0A20720E0B20737
:10AF600058F58C3D25E0920720E0A20720E0B207CB
:10AF7000F1F0883B2BE0920720E0A20720E0B20727
:10AF8000B1F08C3221E0920720E0A20720E0B20766
:10AF900081F0883027E0920720E0A20720E0B20786
:10AFA00041F0845E9C40A040B04031F402C081E09A
:10AFB00001C084E08093470C0895CF92DF92EF9216
:10AFC000FF920F931F93DF93CF93CDB7DEB72897F0
:10AFD0000FB6F894DEBF0FBECDBF6B01BA01482F8C
:10AFE0004C199D19FE01319688E0DF011D928A956A
:10AFF000E9F7242F332727FD309537FF03C030951D
:10B0000021953F4F522F292F332727FD309537FFAA
:10B0100003C0309521953F4F322F141614F02FEFB7
:10B0200001C021E0191614F08FEF01C081E035173F
:10B0300020F429838C8381950EC0531738F48A83BA
:10B040002B8321952D838195888708C08A832B8344
:10B050008130B1F48FEF8E8321952F83FB018081A6
:10B06000992787FD909500271127081B190BDE01F2
:10B07000119657E039E0E32EF12CEC0EFD1E0AC0CC
:10B08000982F9195213021F48FEF8D839887E6CF0B
:10B090009E83E2CF4C91842F992787FD909580174E
:10B0A000910789F411962C911197332727FD30953C
:10B0B000FB018181992787FD9095909581959F4F00
:10B0C0002817390731F12C2D240F11963C91119737
:10B0D0008D2D830FF5E08F02C0011124E22FE5953D
:10B0E000E595E80FF0E0EB56F34F808190E0237098
:10B0F000220FE52FE21B0E2E02C0959587950A942C
:10B10000E2F780FF06C0DB0111963C9311974C9348
:10B1100005C01296AE15BF0509F0BCCF28960FB634
:10B12000F894DEBF0FBECDBFCF91DF911F910F917D
:10B13000FF90EF90DF90CF900895582F392F442340
:10B1400089F5282F2F5F85E0989F302D1124E22F5D
:10B15000E595E595E30FF0E0EB56F34F808190E045
:10B160002370220F47E0642F621B062E02C09595C4
:10B1700087950A94E2F780FD43C0852F8150E82F20
:10B18000E595E595E30FF0E0EB56F34F208130E0D5
:10B190008370880F481B02C0359527954A95E2F7C2
:10B1A000822F2CC03F5F282F259525955370550F72
:10B1B00047E0451B55E03502C00111243150E22F14
:10B1C000E80FF0E0EB56F34F808190E0042E02C0D0
:10B1D000959587950A94E2F780FD12C031503502AB
:10B1E000C0011124280FE22FF0E0EB56F34F8081CD
:10B1F00090E002C0959587954A95E2F78170089591
:10B2000081E008952091880C273050F42530A0F576
:10B210002230D9F0233020F5213009F05DC00AC07A
:10B220002B3020F4293008F03FC032C02D3008F018
:10B2300053C046C020937D0C82E199E790937F0C28
:10B2400080937E0C84E690E052C020937D0C86E1D2
:10B2500099E790937F0C80937E0C8CE291E047C03D
:10B2600083E080937D0C8AE199E790937F0C809333
:10B270007E0C84EF91E03BC084E080937D0C8EE1F6
:10B2800099E790937F0C80937E0C8CEB92E02FC01B
:10B2900085E080937D0C82E299E790937F0C809308
:10B2A0007E0C88EE93E023C086E080937D0C86E2DE
:10B2B00099E790937F0C80937E0C80ED97E017C008
:10B2C00087E080937D0C8AE299E790937F0C8093CE
:10B2D0007E0C88EB9BE00BC088E080937D0C8EE2B7
:10B2E00099E790937F0C80937E0C88E893E190938C
:10B2F0007C0C80937B0C10927A0C1092790C10923B
:10B30000860C8FE08093770C8093780C822F90E0EE
:10B31000019766E070E00E94C579FC01E958F34F9F
:10B3200080917D0C818708950F93CF93DF93482FF1
:10B3300050E087E290E0489FD001499FB00D589FB0
:10B34000B00D1124AB5CB24F1A96ED91FC911B9796
:10B350008181882309F067C018968C91189780FF27
:10B3600062C014963C91149712962C911297230F59
:10B3700012962C93129715968C91159713969C9173
:10B380001397890F13968C9313978091450C87FD23
:10B390000DC03F3F21F4263348F483EC05C0313023
:10B3A00029F4233C18F085E312968C9387E290E011
:10B3B000489FE001499FD00D589FD00D1124CB5CD0
:10B3C000D24FEC85FD8585818F5F8583EC85FD857A
:10B3D0006A8164504B8144508985218102810E9499
:10B3E00078548A81482F50E0CA0104978770907082
:10B3F000892BC9F48B81282F30E0C901049787700D
:10B400009070892B81F44053504073E055954795D7
:10B410007A95E1F748832851304063E035952795C8
:10B420006A95E1F72983DF91CF910F9108950F93EA
:10B4300080910B0D982F82FF08C0E0910F0DF091C5
:10B44000100D85818F5F858364C0E0910D0DF091B3
:10B450000E0D8181882309F05CC090FF5AC02091B5
:10B46000070D9091050D920F9093050D4091080DD9
:10B470008091060D480F4093060D8091450C87FD85
:10B4800011C08091440C882369F42F3F21F4963336
:10B4900048F483EC05C0213029F4933C18F085E38F
:10B4A0008093050DE0910F0DF091100D85818F5F58
:10B4B00085836091050D6450445080910C0D21816D
:10B4C00002810E9478548091050D482F50E0CA01F6
:10B4D000049787709070892BE1F48091060D282FD6
:10B4E00030E0C901049787709070892B91F4405324
:10B4F0005040F3E055954795FA95E1F74093030DD9
:10B5000028513040E3E035952795EA95E1F72093FF
:10B51000040D0F9108958091040D8A30BCF483E0EE
:10B5200069E04EE65EE50E941E548AE168E04AE763
:10B530005EE50E941E5483E06CE046E85EE50E94F2
:10B540001E548BE16CE042E95EE52FC08E30BCF406
:10B5500083E069E046E55EE50E941E548AE168E00A
:10B560004CE55EE50E941E5483E06CE042E65EE539
:10B570000E941E548BE16CE048E65EE516C083E055
:10B5800069E044E75EE50E941E548AE168E040E815
:10B590005EE50E941E5483E06CE04CE85EE50E948C
:10B5A0001E548BE16CE048E95EE50E941E5408954C
:10B5B000FF920F931F936091440C611161E016E1BB
:10B5C000A6E1FA2E062F075E1BC040914C0C863078
:10B5D00060F066E00E94A5799F01290F311DC90125
:10B5E00066E070E00E94C579FC01E958F34F81855F
:10B5F00050E0480F511D812F602F0E9413451150BC
:10B600008F2D811BE82FF0E08091880C863018F098
:10B6100026E030E002C0282F30E0E217F307ACF25A
:10B620001F910F91FF9008950F931F9310E0012F2A
:10B63000085F802F69E140E050E00E94134580914F
:10B640001F0D181730F4802F69E14CE850E00E947C
:10B6500013451F5F153059F71F910F910895809181
:10B66000440C82FF20C08091E50C86FD03C040E0C1
:10B6700050E004C080918101482F50E086E063E1F2
:10B680000E941345409181018CE066E150E00E94E8
:10B69000134580918101882311F485E801C080E081
:10B6A000809381010895882309F045C08091A40CFE
:10B6B00084FD03C040E050E004C080918201482F27
:10B6C00050E087E066E00E9413458091A80C84FD5D
:10B6D00003C040E050E004C080918201482F50E058
:10B6E00087E166E00E9413458091E50C84FD03C06C
:10B6F00040E050E004C080918201482F50E087E094
:10B7000063E10E9413458091E90C84FD03C040E091
:10B7100050E004C080918201482F50E087E163E14E
:10B720000E94134580918201882311F489E101C0B0
:10B7300080E0809382010895EF92FF920F931F9310
:10B74000CF93DF93E62EF22E8A01EC018EEEF80EF7
:10B75000F8018491882351F1803259F02F2D482F20
:10B7600050E0622F70E0FB01E35FFE4F8081882391
:10B7700031F440914C0C8C2F6E2D50E00FC0992766
:10B7800087FD90954817590779F440914C0C50E08B
:10B790004E5E5F4F460F571F8C2F6E2D0E94134534
:10B7A0000F5F1F4F2196D4CF2F5FDBCFDF91CF915B
:10B7B0001F910F91FF90EF9008958091A40B882323
:10B7C00099F087E061E040E050E00E94134588E096
:10B7D00061E040E050E00E94134589E061E040E014
:10B7E00050E00E94134509C087E090E061E070E0FE
:10B7F0004AEF53E822E10E949C5B8091A40B91E008
:10B8000089278093A40B0895BF92CF92DF92EF9285
:10B81000FF920F931F93CF93DF93B62E69017A01A6
:10B82000EC0110E030C0C701B6012AE030E040E092
:10B8300050E00E94D879662339F4112329F0C1140D
:10B84000D104E104F10451F040914C0C50E04E5E03
:10B850005F4F460F511D8C2F6B2D05C040914C0C36
:10B860008C2F6B2D50E00E9413451F5FC701B6015E
:10B870002AE030E040E050E00E94D879C901DA01C6
:10B880006C017D012197101738F4112361F2C11466
:10B89000D104E104F10439F6DF91CF911F910F91AA
:10B8A000FF90EF90DF90CF90BF9008950F930AE044
:10B8B0000E94045C0F9108950F93242F30E040E024
:10B8C00050E003E00E94045C0F910895DF92EF9234
:10B8D000FF920F931F93CF93DF93D62E79018A01A6
:10B8E000C82FD0E0CE0170E00E94565CE114F10454
:10B8F0000105110539F4CE0101976D2D70E040E08E
:10B900000E945C5CDF91CF911F910F91FF90EF90AF
:10B91000DF9008959C0140E050E080914F0C9091A1
:10B92000500CA091510CB091520C280F391F4A1F96
:10B930005B1F20934F0C3093500C4093510C50934D
:10B94000520C8AE062E00E94665C20914F0C3091BC
:10B95000500C4091510C5091520C8091300D9091AF
:10B96000310DA091320DB091330D82179307A407CA
:10B97000B50760F42093300D3093310D4093320DB4
:10B980005093330D85E162E00E94665C20918A0C41
:10B9900030918B0C40918C0C50918D0C80914F0C00
:10B9A0009091500CA091510CB091520C821B930BB2
:10B9B000A40BB50B80519742A040B04030F160918C
:10B9C0001F0D862F90E0049714F085E002C0862FAB
:10B9D0008F5F80931F0D205F384D4F4F5F4F209337
:10B9E0008A0C30938B0C40938C0C50938D0C0E94DE
:10B9F000145B8091D30D9091D40D80689093D40DF9
:10BA00008093D30D81E88093200D08950F931F93A9
:10BA1000CF93DF93182F092FEB01E881F0E0EB566D
:10BA2000F34F208130E0898190E0019702C0359585
:10BA300027958A95E2F720FFE9C08091440C88237E
:10BA400091F48091D30D87FD0EC08091A30B8F5F81
:10BA50008093A30B80FF02C080E001C081E060E31F
:10BA600041E00E9441538091440C9091890C8823BD
:10BA700011F0892F02C0892F81508093890C9091F9
:10BA8000880C953010F084EB01C080EF80934D0C52
:10BA900080918E0C882309F440C08F5F80938E0CB8
:10BAA000853059F41092700D90912F0D923091F0D5
:10BAB0008091970D882371F05BC08C3079F41092DF
:10BAC000970D90912F0D913029F08091700D882362
:10BAD00009F046C0933009F04FC055C0843109F0D9
:10BAE00052C08091B20D87FF4EC01092BE0D909152
:10BAF0002F0D913031F08091700D882311F081E08D
:10BB000007C0923039F08091970D882319F082E0B8
:10BB100080932F0D10928E0C36C09330A0F540917B
:10BB20002F0D242F30E087E290E0289FF001299F1D
:10BB3000F00D389FF00D1124EB5CF24F92899923A0
:10BB400011F184898823F9F0892F8150828B882311
:10BB5000D1F4148A413031F08091700D882311F0B6
:10BB600081E00FC0423031F08091970D882311F0B1
:10BB700082E007C0433039F08091BE0D882319F070
:10BB800083E080932F0DE881F0E0EB56F34F29819D
:10BB900030E02150304081E090E002C0880F991FD2
:10BBA0002A95E2F78095208182238083602F6D5F44
:10BBB000812F8A5F40E050E00E9413450E940556A5
:10BBC000812F902F0E94DB55882321F081E0809304
:10BBD000460C04C08AE090E00E948A5C9091890C37
:10BBE0009D3211F09D3619F481E08093480C992321
:10BBF00069F410922B0D10922C0D10922D0D1092B5
:10BC00002E0D8091450C80618093450CDF91CF9182
:10BC10001F910F910895DF92EF92FF920F931F9360
:10BC2000DF93CF9300D00F92CDB7DEB780910B0D8D
:10BC3000282F30E0C9018E709070892B09F0E3C184
:10BC400025FFACC08091050D90E00497877090703F
:10BC5000892B09F0A3C08091060D90E004978770AE
:10BC60009070892B09F09AC08091040D3091030DDA
:10BC70001B8225E08202C0011124432F4595459582
:10BC8000480F3370330F27E0231BE42FF0E0EB560F
:10BC9000F34F808190E0022E02C0959587950A941B
:10BCA000E2F780FD02C081E08B832A834983809183
:10BCB000030D9091040DBE016F5F7F4F0E94065DE2
:10BCC0008091480C8230D9F42091030D332727FD51
:10BCD00030958091770C90E006972817390779F412
:10BCE0002091040D332727FD30958091780C90E04A
:10BCF00003972817390719F484E08093480C609162
:10BD0000050D7091060D4091070D5091080D809121
:10BD1000030D9091040D0E949D58882309F43EC0A4
:10BD20008091210D90E083709070009749F490917C
:10BD3000350D8091360D292F281B891B982F24C083
:10BD40008130910559F42091360D80915C0D280FBA
:10BD500090915D0D8091350D981B16C0029751F49E
:10BD60002091830D80915D0D281B90915C0D809139
:10BD7000840D09C02091840D8091AA0D280F909107
:10BD8000830D8091AB0D980F6091030D7091040DA0
:10BD9000822F47E05DE00E94DD572DC18091060DA6
:10BDA0002091050D1091040D0091030DE091110DEE
:10BDB000E23021F0D090120DEE2E04C0D090080D8C
:10BDC000E090070D30E0482F50E0CA01049724505E
:10BDD0003040822B932B2C5F3F4F87709070892BC4
:10BDE00009F446C0A091070D8A2F992787FD9095E9
:10BDF000280F391F2450304027703070232B09F052
:10BE0000FAC0F091080D6F2F772767FD7095460FE8
:10BE1000571F4450504047705070452B09F0EBC0FD
:10BE20009C0197FF03C0309521953F4F8E2F992796
:10BE300087FD909597FF03C0909581959F4F281798
:10BE4000390709F4D8C09B0177FF03C030952195CD
:10BE50003F4F8091120D992787FD909597FF03C062
:10BE6000909581959F4F2817390709F0C7C0C3C027
:10BE7000FF241B8285E01802C0011124302F359564
:10BE80003595380F802F8370880F27E0281BE32F0C
:10BE9000F0E0EB56F34F808190E0022E02C09595C2
:10BEA00087950A94E2F780FD02C081E08B832A83A4
:10BEB0003983C801BE016F5F7F4F0E94065D80918C
:10BEC000480C8230D9F42091030D332727FD30959B
:10BED0008091770C90E006972817390779F4209124
:10BEE000040D332727FD30958091780C90E003975F
:10BEF0002817390719F484E08093480C302F3E0D41
:10BF00001B821D0D85E01802C0011124E32FE59569
:10BF1000E595E80FE9833370330F27E0231B2A836D
:10BF2000F0E0EB56F34F808190E002C09595879545
:10BF30002A95E2F780FD02C081E08B8340910B0DD2
:10BF400040FF59C08B818823A9F1FF2009F053C01D
:10BF50008091110D823039F13091070D8091030DE0
:10BF6000380F8091080D2091040D820F1B8225E06F
:10BF70008202C0011124E32FE595E595E80FE983DE
:10BF80003370330F27E0231B2A83F0E0EB56F34F87
:10BF9000808190E002C0959587952A95E2F780FD13
:10BFA00002C081E08B838B81882329F14E7F4093EF
:10BFB0000B0D1EC0FF20C1F02091070D8091050DD3
:10BFC000820F8093050D9091080D8091060D890FC9
:10BFD0008093060D8091030D820F8093030D809155
:10BFE000040D890F8093040DD092080DE092070D87
:10BFF00082E08093110D0E94BE5605C00A0F1F0FEC
:10C00000FF24F39436CF0F900F900F90CF91DF91D4
:10C010001F910F91FF90EF90DF9008950F93882369
:10C0200009F4BCC080910B0D8E7F80930B0DE091C5
:10C030000F0DF091100D80910C0D60EF40EE2181FD
:10C0400002810E94785480913D0D8A7F80933D0D3E
:10C05000E091410DF091420D80913E0D60EF40EE78
:10C06000218102810E9478548091640D8A7F80939F
:10C07000640DE091680DF091690D8091650D60EFA0
:10C0800040EE218102810E94785480918B0D8A7F3D
:10C0900080938B0DE0918F0DF091900D80918C0D20
:10C0A00060EF40EE218102810E9478548091B20DB0
:10C0B0008A7F8093B20DE091B60DF091B70D80911B
:10C0C000B30D60EF40EE218102810E9478540E94FE
:10C0D000D74487E090E061E070E04AEF53E822E166
:10C0E0000E949C5B8EE090E061E070E04EEF53E8D0
:10C0F00022E10E949C5B2091300D3091310D4091E6
:10C10000320D5091330D85E162E00E94665C209112
:10C110004F0C3091500C4091510C5091520C8AE0D0
:10C1200062E00E94665C87E090E06AE070E049E0CF
:10C1300054E823E60E949C5B89E090E06EE070E0AA
:10C140004BE154E821E50E949C5B82E090E062E1D3
:10C1500070E049E254E825E70E949C5B85E090E0AE
:10C1600066E170E045E454E82AE30E949C5B82E0CB
:10C1700090E06AE170E04CE554E822E10E949C5BAB
:10C180008BE090E06AE170E04091870C0E945C5C7B
:10C190008CE291E090939E0B80939D0B80919D0B80
:10C1A00090919E0B009719F420E030E003C09C01B1
:10C1B0002150304030939E0B20939D0BC9010F916D
:10C1C00008951F938091440C882321F480910B0DD6
:10C1D00085FFDDC080913E0C90913F0C90FF3BC0ED
:10C1E00080919C0B8823C9F581E080939C0B809102
:10C1F000870C8F3F09F08F5F8093870C82E090E07F
:10C200006AE170E04CE554E822E10E949C5B8BE01F
:10C2100090E06AE170E04091870C0E945C5C2091A4
:10C22000450C23FF06C081E090E09093430C80937F
:10C23000420C2D782093450C10920B0D81E39AE36C
:10C240000E94394510924C0C82E08093440C81E0AE
:10C250000E940E6002C010929C0B80913E0C83FFE6
:10C260004BC080919B0B882309F048C081E08093EC
:10C270009B0B8091870C8823C1F090910B0D95FD4D
:10C2800014C081508093870C88E08093440C9F7D7C
:10C2900090930B0D8091450C83FF30C081E090E0BE
:10C2A0009093430C8093420C29C080910B0D85FF25
:10C2B0001CC02091450C23FF06C081E090E09093C4
:10C2C000430C8093420C2D782093450C10920B0D5B
:10C2D00081E39AE30E94394510924C0C82E08093EE
:10C2E000440C81E00E940E6009C088E790E09093C2
:10C2F000410C8093400C02C010929B0B8091400C2B
:10C300009091410C009709F442C08C33910569F17A
:10C310008D33910530F48130910551F04E9771F5D0
:10C3200019C08A359105B1F08837910539F51DC0DE
:10C3300082E090E06AE170E04CE554E822E10E947E
:10C340009C5B8BE090E06AE170E04091870C0E947A
:10C350005C5C14C012E0812F6AE140E050E00E9472
:10C3600013451F5F1D30B9F709C082E090E06AE114
:10C3700070E048E654E822E10E949C5B8091400C0A
:10C380009091410C01979093410C8093400C1F9128
:10C3900008950F931F93CF93DF93282F362F61308B
:10C3A00051F0613030F0623051F0633031F080E0B4
:10C3B0000BC090E007C090E004C09AE001C090E09C
:10C3C000965F945F892F8A5F280FC32FD0E087E2A2
:10C3D00090E0C89FF001C99FF00DD89FF00D112487
:10C3E000EB5CF24F808582FD2A5F69E0369F800119
:10C3F00011240D5A134F269FB00111246155764820
:10C40000C80149E050E00E94804D87E290E0C89F5B
:10C41000F001C99FF00DD89FF00D1124EB5CF24F95
:10C4200015870487DF91CF911F910F9108950F9386
:10C430001F93CF93DF93682F082F10E087E290E0DF
:10C44000089FF001099FF00D189FF00D1124EB5C7F
:10C45000F24F24818681281729F4958187819817C6
:10C4600009F44EC087E290E0089FF001099FF00DAB
:10C47000189FF00D1124EB5CF24F808581FD40C0C8
:10C4800083FD3EC08581222331F4813011F080E0AC
:10C4900009C082E007C0213011F483E003C02F3FC0
:10C4A00079F581E00E94C96187E290E0089FF00180
:10C4B000099FF00D189FF00D1124EB5CF24FA4853D
:10C4C000B58514968C9114972C91280F90E0EF016C
:10C4D000299614C01796ED91FC911897E80FF11D5D
:10C4E0003491E881F0E0E90FF11DEE0FFF1FEE0F30
:10C4F000FF1FEC5EF34F30838F5F9F5F821750F317
:10C5000087E290E0089FD001099FB00D189FB00D01
:10C510001124AB5CB24F1C96ED91FC911D97958157
:10C520008681981709F046C015821C96ED91FC9102
:10C530001D9784819081890F84831C96ED91FC91D5
:10C540001D9794818381981749F4148253968C9196
:10C550005397882319F0815053968C9387E290E08B
:10C56000089FF001099FF00D189FF00D1124EB5C5E
:10C57000F24FA485B58514968C9114972C91280FB1
:10C5800090E0EF01299614C01796ED91FC91189751
:10C59000E80FF11D3491E881F0E0E90FF11DEE0F95
:10C5A000FF1FEE0FFF1FEC5EF34F30838F5F9F5F27
:10C5B000821750F387E290E0089FF001099FF00D89
:10C5C000189FF00D1124EB5CF24F948185818783D5
:10C5D0009683DF91CF911F910F910895DF92EF9293
:10C5E000FF920F931F93CF93DF93D82EE82EFF2453
:10C5F00087E290E0E89ED001E99EB00DF89EB00D74
:10C600001124AB5CB24F1A96ED91FC911B9781817E
:10C61000882309F02FC218962C91189727FF5DC028
:10C6200054968C915497882391F412968C9112977A
:10C6300090E0049787709070892B49F413968C9141
:10C64000139790E0049787709070892B61F187E2CF
:10C6500090E0E89EF001E99EF00DF89EF00D1124A7
:10C66000EB5CF24F8381482F50E08189282F3327DC
:10C6700027FD3095C901039673E0880F991F7A95BD
:10C68000E1F74817590709F44DC02C5F3F4F63E0AD
:10C69000220F331F6A95E1F74217530709F0EAC1E9
:10C6A0008FEF8583E7C12F77206218962C93189718
:10C6B00081E08D1538F014961C9214978FEF159623
:10C6C0008C930BC082E0D81611F481E001C08FEF8B
:10C6D00014968C93149715961C9287E290E0E89E2E
:10C6E000F001E99EF00DF89EF00D1124EB5CF24F85
:10C6F000828190E0049787709070892B09F0BAC10D
:10C70000838190E0049787709070892B09F0B2C103
:10C71000208522FF9FC03081393031F481818830FB
:10C7200019F4148281E0BDCF87E290E0E89EF00129
:10C73000E99EF00DF89EF00D1124EB5CF24F80891C
:10C74000381709F097C091818189981709F092C034
:10C750002B7F208724E030E00E2C02C0220F331FF5
:10C760000A94E2F7209530958091D30D9091D40DE5
:10C77000822393239093D40D8093D30D958184814C
:10C78000882321F4913059F482E009C0813011F4FA
:10C7900083E005C08F3F11F08FEF01C081E06D2D68
:10C7A0000E94C961DD2091F080918E0C882311F5E3
:10C7B00087E290E0E89EF001E99EF00DF89EF00D12
:10C7C0001124EB5CF24F82898823A1F487E290E088
:10C7D000E89EF001E99EF00DF89EF00D1124EB5C4F
:10C7E000F24F8085806280878481819584838581F2
:10C7F000819557CF27E230E0E29EF001E39EF00DF5
:10C80000F29EF00D1124EB5CF24F808580688087EA
:10C8100081E0848B40912F0D842F90E0829FF00166
:10C82000839FF00D929FF00D1124EB5CF24F8085F9
:10C8300087FF02C0D41610F4D0922F0D87E290E04B
:10C84000E89EF001E99EF00DF89EF00D1124EB5CDE
:10C85000F24F0EC025FF0EC08081893059F48181CE
:10C86000883021F42F7D2064208704C08A3011F4A1
:10C87000148216CF07E210E0E09EE001E19ED00DA9
:10C88000F09ED00D1124CB5CD24F6A817B814C810C
:10C890005D81888199810E949D58882309F4EAC0AE
:10C8A000888590E082FD13C08A709070892B91F486
:10C8B0008D818130A1F18881883011F08A3079F53D
:10C8C0008981883009F4D6C0803149F5D3C02989DF
:10C8D000A889BCC080918F0C9091900C9C01237012
:10C8E0003070209FF001219FF00D309FF00D11243A
:10C8F000EB5CF24FA08101969C0123703070209F69
:10C90000F001219FF00D309FF00D1124EB5CF24FF0
:10C91000208101969093900C80938F0C97C080910A
:10C92000470C8230A9F4DD2029F480913C0C8670FC
:10C9300009F085C087E290E0E89EF001E99EF00DE5
:10C94000F89EF00D1124EB5CF24F2785A6857EC082
:10C9500081E0D81661F0D81608F471C082E0D816CC
:10C96000E1F083E0D816A9F120E0A0E06FC030919B
:10C97000030DE091070D9091080D292F220F220F32
:10C980008091040D280F9F3F29F0AE2FAA0FAA0F08
:10C99000A30F5CC0A32FA45059C02091030D909108
:10C9A000070D990FE091040D8091080D8F3F19F04C
:10C9B000892F820F02C0822F8250A82FAA0F809148
:10C9C000350DA81B292F2E0F220F8091360D281B05
:10C9D0003DC087E290E0E89EE001E99ED00DF89E20
:10C9E000D00D1124CB5CD24F4881552747FD50957F
:10C9F0008091030D992787FD9095481B590B29813C
:10CA0000332727FD30958091040D992787FD909558
:10CA1000281B390B229FC001239F900D329F900D40
:10CA20001124449F9001459F300D549F300D1124D7
:10CA3000820F931F62E00E949C55089728F0209176
:10CA4000040DA091030D02C02F85AE8587E290E012
:10CA5000E89EA001E99E500DF89E500D1124FA01A8
:10CA6000EB5CF24F60817181475C524F8A2F922FAD
:10CA70000E94DD57DF91CF911F910F91FF90EF90B2
:10CA8000DF9008950F931F9302E21DE099E0899FC4
:10CA9000B001112461557648C80149E050E00E9478
:10CAA000804D1093100D00930F0D1F910F9108955D
:10CAB0000F93CF93DF932091070D8091090D2817D5
:10CAC00031F49091080D80910A0D981779F18091B9
:10CAD000080D222331F4813011F080E009C082E09A
:10CAE00007C0213011F483E003C02F3FF9F481E047
:10CAF0000E944265C0910F0DD091100D9C8128813C
:10CB0000290F80910C0DA82FB0E0AA0FBB1FAA0F10
:10CB1000BB1FAC5EB34F08C0EF81F885E90FF11D74
:10CB2000E491EC939F5F14969217B0F380910B0DF4
:10CB3000857019F5C0910F0DD091100D8C81813049
:10CB4000E1F01D8281E08C8398819F5F80910C0DC4
:10CB5000A82FB0E0AA0FBB1FAA0FBB1FAC5EB34F3C
:10CB600081E008C0EF81F885E80FF11DE491EC93B6
:10CB70008F5F14968917B0F33DC0E0910F0DF091CF
:10CB8000100D958186819817A9F515828081948171
:10CB9000890F84839381891789F4148280910B0D06
:10CBA00082FF0CC08B7F886080930B0D80910C0DF1
:10CBB00060EF40EE218102810E947854C0910F0DF8
:10CBC000D091100D9C812881290F80910C0DA82FE8
:10CBD000B0E0AA0FBB1FAA0FBB1FAC5EB34F08C0CB
:10CBE000EF81F885E90FF11DE491EC939F5F1496B6
:10CBF0009217B0F39091070D8091080D80930A0D64
:10CC00009093090DDF91CF910F910895BF92CF922C
:10CC1000DF92EF92FF920F931F93282F882349F5FD
:10CC200080913C0CE82FF0E0CF0186709070892B4A
:10CC300001F1F695E7958E2F809581709091880C83
:10CC4000913029F0953010F48E5F01C08C5FE82F91
:10CC5000F0E0EF57FC47E49166E0E69FB001112455
:10CC60006B5E7C478AE49DE046E050E00E94804D88
:10CC700069C08091450C87FF02C0ECE015C080912F
:10CC8000440C882311F0EFE00FC08091880C8130B4
:10CC900011F4E0E009C0853010F4E3E005C085310F
:10CCA00010F0E9E001C0E6E04E2F4F5FF0E0E159FF
:10CCB000FC475491842F90E081599C47FC01B4902B
:10CCC0004F5F842F90E081599C47FC01149130E024
:10CCD00087E290E0289F7001299FF00C389FF00CAC
:10CCE00011248AE4C82E8DE0D82ECE0CDF1C06E07D
:10CCF000509FB00111246B5E7C47C60146E050E0B6
:10CD00000E94804D109FB00111246B5E7C47C701CB
:10CD10008A5A924F46E050E00E94804DB09E8001BA
:10CD200011240B5E1C47C701805B924FB80146E09F
:10CD300050E00E94804D85E39DE0E80EF91EF7016A
:10CD4000D386C2861F910F91FF90EF90DF90CF9016
:10CD5000BF9008951F93CF93DF93182FC82FD0E073
:10CD600087E290E0C89FA001C99F500DD89F500D49
:10CD70001124FA01EB5CF24F8085282F30E082FD10
:10CD80004AC0828190E0049787709070892B09F0E7
:10CD900042C0838190E0049787709070892BD9F509
:10CDA0008081833039F481818A30A9F584818F3F75
:10CDB00091F518C0843071F481818A3061F58481E5
:10CDC000813049F52A703070232B11F0CA011BC045
:10CDD000CA011DC08F3051F481818A30E1F4848111
:10CDE0008130C9F4CA018A5A924F13C08E3099F427
:10CDF00081818A3081F484818F3F69F42A70307098
:10CE0000232B21F0CA01805B924F03C0CA01865BCD
:10CE1000924F9387828787E290E0C89FF001C99F75
:10CE2000F00DD89FF00D1124EB5CF24F80858A70D5
:10CE300011F00E94BE5687E290E0C89FF001C99FA2
:10CE4000F00DD89FF00D1124EB5CF24F808586FF2A
:10CE500011C08F7B8087133069F480913C0C83FF75
:10CE600003C0877F816004C084FF04C08F7E83601D
:10CE700080933C0C87E290E0C89FF001C99FF00DC1
:10CE8000D89FF00D1124EB5CF24F908593FF5FC0AB
:10CE90008389882309F05BC0977F9087958184817F
:10CEA000882321F4913059F482E009C0813011F4D3
:10CEB00083E005C08F3F11F08FEF01C081E0612F4B
:10CEC0000E94C96187E290E0C89FA001C99F500DF0
:10CED000D89F500D1124FA01EB5CF24F9A012A5AA7
:10CEE000324F828593858217930729F0CA01865BAA
:10CEF000924F9387828787E290E0C89FF001C99F95
:10CF0000F00DD89FF00D1124EB5CF24FA485B58590
:10CF100014968C9114972C91280F90E0EF0129968C
:10CF200014C01796ED91FC911897E80FF11D3491FC
:10CF3000E881F0E0E90FF11DEE0FFF1FEE0FFF1F7C
:10CF4000EC5EF34F30838F5F9F5F821750F31123A6
:10CF5000D1F480913C0C80FF16C0982F9E7F91FFEA
:10CF600009C08C7F846080933C0C80E00E94066640
:10CF700086E007C0926090933C0C80E00E940666B9
:10CF800085E08093340DDF91CF911F910895EF924A
:10CF9000FF920F931F938091450C87FF02C088E09A
:10CFA00015C08091440C882311F08AE00FC0809155
:10CFB000880C813011F480E009C0853010F482E0E3
:10CFC00005C0853110F086E001C084E0E82FF0E074
:10CFD000ED59FC4724918F5F90E08D599C47FC01EF
:10CFE000149153E1E52E5DE0F52E06E0209FB0019F
:10CFF00011246B5E7C47C70146E050E00E94804DE3
:10D00000109F800111240B5E1C47C7010696B801D2
:10D0100046E050E00E94804DF0920E0DE0920D0D22
:10D020001F910F91FF90EF900895DF92EF92FF9282
:10D030000F931F93CF93DF930E94D74478EEE72E90
:10D04000E092050D1CE61093060DDD24DA94D092D3
:10D05000070D1092080DE0910F0DF091100D8091C9
:10D060000C0D68EE48E6218102810E947854FF246D
:10D07000F394F0920B0D0E94C76781E00E94426515
:10D08000E092370D1093380D10923B0D10923C0D2D
:10D09000D092390D10923A0DE091410DF091420D70
:10D0A00080913E0D68EE48E6218102810E9478540D
:10D0B000F0923D0D80E00E94066680913D0D8E7FCE
:10D0C00080933D0D85E06FE479E70E944A5485E046
:10D0D00060EE48E622E002E00E94785489E890E899
:10D0E0000E94A74FFF24C0E0D0E0DD24D39467E086
:10D0F000E62E0E943E458823E1F30E94414580913F
:10D10000050D883C49F48091070D8F3F29F48091EB
:10D110003D0D816080933D0D8091370D883D59F420
:10D120008091390D8F3F39F485E060E043E622E0DD
:10D1300002E00E9478548091050D843089F4E091DA
:10D140000F0DF091100D80910C0D60EF40EE2181DC
:10D1500002810E94785480910B0D8E7F80930B0D7D
:10D16000F1FC2EC08091370D883751F582E0F82A06
:10D17000E0913F0DF091400D1082E0913F0DF09154
:10D18000400D1182E0913F0DF091400DD282E0916F
:10D190003F0DF091400D1382E0913F0DF091400D55
:10D1A000E482E0913F0DF091400D158281E060E056
:10D1B0000E94C9618FE06DE041ED50E00E9413458F
:10D1C0001F2DF1FE0AC08091370D843731F48EE0B7
:10D1D0006DE040ED50E00E94134512FD2CC080919F
:10D1E000370D8C3641F584E0F82AE091410DF0913D
:10D1F000420D80913E0D60EF40EE218102810E9440
:10D2000078548FE06DE040E050E00E9413458EE0DE
:10D210006DE040E050E00E9413458FE06DE042ED8C
:10D2200050E00E9413458DE06DE04EEC50E00E940E
:10D230001345C4EBD0E01F2DF0FC0AC080910D0D0A
:10D2400090910E0D0E94F9560E94175A0E9458653F
:10D2500012FD0DC080913F0D9091400D0E94F95636
:10D2600080E00E94945980E00E9417620FC02097CE
:10D2700099F02197CC33D10539F48DE06DE04FEC76
:10D2800050E00E94134502C0209731F08091210D9B
:10D290008F5F8093210D2DCFDF91CF911F910F9143
:10D2A000FF90EF90DF900895FF920F931F93CF931D
:10D2B000DF93F82E882311F00E94D7448091480C08
:10D2C00081FF10C08D7F8093480C10927A0C1092D1
:10D2D000790C8091770C6091780C40E050E00E94CE
:10D2E000134514C083FF12C0877F8093480C1092AF
:10D2F000860CE0917E0CF0917F0C24913196E491A4
:10D3000080E060EF40EE0E2F0E947854FF20F9F08D
:10D310008DE98093890C10923C0C1092900C109225
:10D320008F0C9091880C913011F482E005C09230FE
:10D3300011F081E001C083E080932F0D10928E0CDC
:10D34000953010F084EB01C080EF80934D0C8091FC
:10D350000B0D85FD02C01092210D1092940C1092BD
:10D36000930C88EC90E09093920C8093910C82E067
:10D3700099E790934A0C8093490C85E060EF40EE6A
:10D3800022E002E00E947854CBE3DDE010E01A8254
:10D3900018821982EE81FF818B8160EF40EE21813E
:10D3A00002810E947854112319F08A8180688A834F
:10D3B0001F5FA796143059F71093340D81E090E069
:10D3C0009093D40D8093D30D1092200DFF2071F017
:10D3D00082E063E041EB5BE50E941E5485E99CE03E
:10D3E00067E873E84EE650E00E94804D87E090E0E9
:10D3F00061E070E04AEF53E822E10E949C5B8EE01E
:10D4000090E061E070E04EEF53E822E10E949C5B07
:10D410002091300D3091310D4091320D5091330DEE
:10D4200085E162E00E94665C20914F0C3091500CC7
:10D430004091510C5091520C8AE062E00E94665C6F
:10D440000E94145B0E9402590E94D85A80910B0DD1
:10D4500085FF05C08CE06FE048EA5EE510C0FF2064
:10D4600051F08091880C813031F48CE06BE041EB1D
:10D470005EE50E941E548DE06FE041EA5EE50E9489
:10D480001E5489E08093030D80E18093040D8CE7A6
:10D490008093050D8CE98093060D8FEF8093070D27
:10D4A0001092080D82E08093110D1092120D1092CF
:10D4B000090D10920A0D80930C0D0E94C767809190
:10D4C0000B0D816080930B0D81E00E944265C0913D
:10D4D0000F0DD091100D1C82288180910C0DA82F6A
:10D4E000B0E0AA0FBB1FAA0FBB1FAC5EB34F90E00A
:10D4F00008C0EF81F885E90FF11DE491EC939F5F7F
:10D5000014969217B0F36091050D64504091060D8A
:10D51000445029810A810E94785409E00093350D16
:10D5200088E08093360D80E18093430D1092440D86
:10D530008AE78093370D8CE58093380D0093450D75
:10D540001AE01093460D8FEF8093390D10923A0D2B
:10D5500083E080933E0D81E060E00E94C96180918C
:10D560003D0D816080933D0D80E00E940666109223
:10D57000490D00935C0D10935D0D82E080936A0D60
:10D5800010926B0D8CE780935E0D8CE680935F0D9F
:10D5900000936C0D10936D0D1092600D81E08093DF
:10D5A000610D84E08093650D82E061E00E94C961B5
:10D5B0008091640D81608093640D81E00E94066615
:10D5C000FF2021F010926E0D1092700D28E0209334
:10D5D000830D9AE09093840D80E18093910D85E115
:10D5E0008093920D84E78093850D8DE68093860D60
:10D5F0002093930D9093940D1092870D8FEF80934D
:10D60000880D85E080938C0D80E062E00E94C96106
:10D6100080918B0D816080938B0D82E00E94066665
:10D62000FF2079F09091880C913011F080E001C0DA
:10D6300083E18093950D1092970D913011F49093A2
:10D64000970D9AE09093AA0D9093AB0D82E0809392
:10D65000B80D85E18093B90D84E88093AC0D8BE61D
:10D660008093AD0D9093BA0D9093BB0D1092AE0DBB
:10D670008FEF8093AF0D86E08093B30D80E063E081
:10D680000E94C9618091B20D81608093B20D83E0E8
:10D690000E940666FF20A1F09091880C913011F451
:10D6A00087E205C0923011F080E001C080E28093F3
:10D6B000BC0D1092BE0D933018F481E08093BE0D26
:10D6C000DF91CF911F910F91FF900895EF92FF92FC
:10D6D0000F931F93CF93DF93882309F460C00E94B8
:10D6E000D74485E99CE067E873E84EE650E00E9485
:10D6F000804D85EE9CE065EF73E845E050E00E94C8
:10D70000804D87E090E061E070E04AEF53E822E16D
:10D710000E949C5B8EE090E061E070E04EEF53E889
:10D7200022E10E949C5B2091300D3091310D40919F
:10D73000320D5091330D85E162E00E94665C2091CC
:10D740004F0C3091500C4091510C5091520C8AE08A
:10D7500062E00E94665C86E090E065E070E044E78D
:10D7600054E822E10E949C5B82E090E06AE170E074
:10D770004CE554E822E10E949C5B8BE090E06AE17A
:10D7800070E04091870C0E945C5C0E9402590E94EC
:10D79000D85A85E992E09093A00B80939F0B8091DB
:10D7A0009F0B9091A00B009709F4F3C00197909301
:10D7B000A00B80939F0B009709F4EBC022E0883503
:10D7C000920769F485E068E04EE050E00E9413455E
:10D7D00088E090E068E070E049E854E80AC0A2E020
:10D7E0008C319A0759F482E190E068E070E04DEAEC
:10D7F00054E82CE20E949C5B04E021C1B1E0803E31
:10D800009B0769F485E06BE04FE050E00E94134510
:10D8100088E090E06BE070E041E954E80AC0E1E0A4
:10D82000843A9E0741F482E190E06BE070E046EBC1
:10D8300054E82AE3DFCFF1E088369F0769F485E0FA
:10D840006EE040E150E00E94134588E090E06EE019
:10D8500070E049E954E80AC021E08C32920741F4B3
:10D8600082E190E06EE070E04EEB54E821E5C2CF3B
:10D87000803F910569F485E061E141E150E00E945B
:10D88000134588E090E061E170E042EA54E809C0A5
:10D89000843B910541F482E190E061E170E045EC68
:10D8A00054E823E6A7CF8837910559F58CE065E168
:10D8B00044E850E00E9413458FE090E065E170E09D
:10D8C0004AE00E945C5C81E190E065E170E049EA39
:10D8D00054E822E10E949C5B8CE066E145E850E060
:10D8E0000E9413458FE090E066E170E042E30E9401
:10D8F0005C5C81E190E066E170E049EA54E822E195
:10D9000079CF8C33910539F486E090E068E170E0DE
:10D9100045E454E88ECF019709F06ECF84E18093FF
:10D92000030D80E18093040D84ED8093050D8CE957
:10D930008093060D8FEF8093070D1092080D82E003
:10D940008093110D1092120D1092090D10920A0D74
:10D95000E0910F0DF091100D80910C0D64ED48E9F0
:10D96000218102810E94785481E080930B0D0E94F6
:10D97000C76787E06CE479E70E944A544091060D3E
:10D98000445087E06091050D21E001E00E94785449
:10D9900033CF82E08093110D1092120D0E940B5E26
:10D9A00080910D0D90910E0D0E94F9560E94175A0C
:10D9B0000E9458658091210D90E08F709070892BA6
:10D9C00011F40E942F5B8091030D813161F082314F
:10D9D0001CF4803161F409C0823119F0833139F4CB
:10D9E00036C011E035C012E033C013E031C0CDE3E2
:10D9F000DDE010E004E0888182FD0AC08A819B811D
:10DA00000E94F956812F0E949459812F0E9417621B
:10DA1000888182FD01501F5FA796143061F78091C5
:10DA2000030D882339F48091070D8F3F19F481E0AD
:10DA30008093070D8091210D8F5F8093210D802FA2
:10DA4000DF91CF911F910F91FF90EF90089510E01B
:10DA5000212F30E087E290E0289F7001299FF00C91
:10DA6000389FF00C112485E39DE0E80EF91E84E157
:10DA7000D7018C9380E111968C93119784ED1296C7
:10DA80008C9312978CE913968C9313978FEF1496BF
:10DA90008C93149715961C92159716961C921697B0
:10DAA00017961C9217971C96ED91FC911D9719964D
:10DAB0008C9164ED48E9218102810E94785481E0D3
:10DAC000F7018087812F0E94066691CF80E00E9437
:10DAD0002846282F8093A10B9093A20B40910B0D09
:10DAE00045FD2DC086FF02C08FEF03C087FF06C033
:10DAF00081E08093110D1092120D0DC084FF04C0BF
:10DB00001092110D8FEF05C085FF05C01092110D09
:10DB100081E08093120D20FF0FC080918001882347
:10DB200071F01092800130E080914B0C882309F451
:10DB300031E030934B0C03C081E080938001822F51
:10DB4000807F19F0416040930B0D822F08958F92D2
:10DB50009F92AF92BF92DF92EF92FF920F931F932B
:10DB6000CF93DF93D82E0E94D74468EEE62EE09242
:10DB7000050D5CE6F52EF092060D1FEF1093070DD4
:10DB80001092080DE0910F0DF091100D80910C0D89
:10DB900068EE48E6218102810E94785481E08093FA
:10DBA0000B0D0E94C76781E00E944265E092370D2D
:10DBB000F092380D1093390D10923A0D10933B0DE1
:10DBC00010923C0DE091410DF091420D80913E0D7F
:10DBD00068EE48E6218102810E94785410923D0D42
:10DBE00080E00E94066685E06FE479E70E944A546F
:10DBF00085E060EE48E622E002E00E947854109250
:10DC0000210D89E890E80E94A74F81E0D8128AE0B0
:10DC100060E00E94C961E0910F0DF091100D8481C8
:10DC20002081280F90E018C0E0910F0DF091100DA9
:10DC30000780F085E02DE80FF11D3491E0910C0D87
:10DC4000F0E0E90FF11DEE0FFF1FEE0FFF1FEC5E7E
:10DC5000F34F30838F5F9F5F821730F3C091410D88
:10DC6000D091420D9C812881290F80913E0DA82FD3
:10DC7000B0E0AA0FBB1FAA0FBB1FAC5EB34F08C01A
:10DC8000EF81F885E90FF11DE491EC939F5F149605
:10DC90009217B0F3FF24F39499E1A92E9DE0B92ED9
:10DCA00080E5882E8DE0982EEE24E3940E943E4578
:10DCB0008823E1F30E944145FF2031F489E890E890
:10DCC0000E94A74FFF24F3948091050D883C49F4EE
:10DCD0008091070D8F3F29F480913D0D81608093E5
:10DCE0003D0D8091370D883D59F48091390D8F3F5E
:10DCF00039F485E060E043E622E002E00E947854D7
:10DD00008091050D8430A9F48091070D8F3F89F42F
:10DD1000E0910F0DF091100D80910C0D60EF40EE31
:10DD2000218102810E94785480910B0D8E7F809317
:10DD30000B0D1091370D143009F06CC08091390D26
:10DD40008F3F09F067C00E94CE4F81E0D816C9F519
:10DD500080910B0D8E7F80930B0DD092390D109218
:10DD60003A0DD0923B0D10923C0D10933E0D83E086
:10DD700060E00E94C961C091410DD091420D9C812B
:10DD80002881290F80913E0DA82FB0E0AA0FBB1F5C
:10DD9000AA0FBB1FAC5EB34F08C0EF81F885E90F37
:10DDA000F11DE491EC939F5F14969217B0F34091AC
:10DDB000380D445064E029810A810E947854FF2480
:10DDC0002DC0E092390D10923A0DE0923B0D109269
:10DDD0003C0D8BE060E00E94C961C091410DD09183
:10DDE000420D9C812881290F80913E0DA82FB0E023
:10DDF000AA0FBB1FAA0FBB1FAC5EB34F08C0EF81B9
:10DE0000F885E90FF11DE491EC939F5F149692174A
:10DE1000B0F367C081E0D81609F064C08091370D77
:10DE20008032E9F48091390D813009F068C0809327
:10DE3000070D1092080D8093090D10920A0D809124
:10DE40000B0D816080930B0D8091060D82508093A5
:10DE5000060D85E00E94426510920C0D4DC0813286
:10DE600009F04DC08091390D813009F048C0E09132
:10DE70000F0DF091100D84812081280F90E018C0C3
:10DE8000E0910F0DF091100D0780F085E02DE80F67
:10DE9000F11D3491E0910C0DF0E0E90FF11DEE0F52
:10DEA000FF1FEE0FFF1FEC5EF34F30838F5F9F5F0E
:10DEB000821730F3E0910F0DF091100D80910C0D51
:10DEC0006091050D4091060D218102810E947854D8
:10DED000B0920E0DA0920D0D9092400D80923F0DCC
:10DEE0000EC0FF2483E0D81639F48091370D8031BD
:10DEF000A9F48091390D09C081E0D81679F4809198
:10DF0000050D803159F48091070D813039F485E099
:10DF100060EE44E622E002E00E9478540E945865D8
:10DF200080910D0D90910E0D0E94F9560E94175A86
:10DF300080E00E94176280913F0D9091400D0E94F9
:10DF4000F95680E00E9494598091370D843EB9F4CF
:10DF50008091390D813099F4D81689F5E091410D01
:10DF6000F091420D80913E0D60EF40EE21810281E3
:10DF70000E94785480913D0D8E7F80933D0D80915D
:10DF8000050D883EB1F48091070D813091F4E09148
:10DF90000F0DF091100D80910C0D60EF40EE21817E
:10DFA00002810E94785482E080930C0D10923E0D05
:10DFB00006C08091210D8F5F8093210D77CEDF9178
:10DFC000CF911F910F91FF90EF90DF90BF90AF9096
:10DFD0009F908F9008958091880C823021F481E089
:10DFE0000E94A76D0895853019F40E941568089560
:10DFF000893021F08D3011F0813119F483E00E94D5
:10E00000A76D089580E090E06AE50E94474681E0B0
:10E0100090E065E50E94474680E490E06FEF0E9443
:10E02000474681E490E06FEF0E9447460895DF93F2
:10E03000CF93CDB7DEB7A0970FB6F894DEBF0FBE73
:10E04000CDBF8DE090E09A8389830E94894D88231B
:10E0500011F40E9402704091300D5091310D609189
:10E06000320D7091330DFE01339628E130E0DB0173
:10E07000CA01022E04C0B695A795979587950A9474
:10E08000D2F78193285030408FEF283F380779F737
:10E09000CE0101960E94FA4DA0960FB6F894DEBF0D
:10E0A0000FBECDBFCF91DF910895EF92FF920F93F6
:10E0B0001F93CF93DF938091450C82FF95C08B7F98
:10E0C0008093450C8091440C8823C1F424E030E017
:10E0D00000904E0C02C0220F331F0A94E2F7809189
:10E0E000D30D9091D40D822B932B9093D40D8093CC
:10E0F000D30D88E06CE741E00E94415380919A0B78
:10E100008111815080939A0B8091450C88608F7BA0
:10E110008093450C80914E0C90E027E230E0829F86
:10E12000A001839F500D929F500D1124FA01EB5CCA
:10E13000F24F90859D7F906190878091440C882359
:10E1400069F4CA01865B924F93878287138A809114
:10E15000910C9091920C0E948A5C02C09E7F9087E5
:10E160008CE390E09093430C8093420C80914E0C92
:10E1700090E027E230E0829FF001839FF00D929FB4
:10E18000F00D1124EB5CF24FA485B585818560EF1D
:10E1900040EE11962C91119712960C910E94785492
:10E1A000E0910F0DF091100D80910C0D60EF40EE9D
:10E1B000218102810E9478546091490C70914A0C2F
:10E1C00087E00E944A54E091490CF0914A0C249156
:10E1D0003196E4916091050D68504091060D4450D0
:10E1E00087E00E2F0E9478542091450C23FFCEC06B
:10E1F0008091420C9091430C009709F4A8C00197BC
:10E200009093430C8093420C892B09F0A0C0277F88
:10E210002093450C80914E0C90E0C7E2D0E08C9F9B
:10E22000F0018D9FF00D9C9FF00D1124EB5CF24FDF
:10E2300080858F7E84608087E091490CF0914A0C44
:10E2400024913196E49187E060EF40EE0E2F0E941A
:10E2500078540E948D568091440C882309F096C012
:10E2600060914E0C862F90E09C012C9FC0012D9F49
:10E27000900D3C9F900D1124FC01EB5CF24F865BEE
:10E28000924F9387828795818481882321F49130EE
:10E2900059F482E009C0813011F483E005C08F3F5A
:10E2A00011F08FEF01C081E00E94C96180914E0C96
:10E2B00090E027E230E0829FF001839FF00D929F73
:10E2C000F00D1124EB5CF24FA485B58514968C916A
:10E2D0001497AC91A80F90E0AF01445F5F4FBF016E
:10E2E000675F7F4F17C0EA0128813981E901EF811B
:10E2F000F885E80FF11D2491EB01E881F0E0E90FCA
:10E30000F11DEE0FFF1FEE0FFF1FEC5EF34F20839A
:10E310008F5F9F5F8A1738F30E94BE56882309F0EB
:10E3200070C68091450C80648093450CE0910F0D80
:10E33000F091100D6091050D64504091060D445010
:10E3400080910C0D218102810E9478541FC0809120
:10E35000420C9091430C8F709070892BA1F40E9415
:10E360002F5B8091440C882371F480910B0D85FD07
:10E370000AC08091420C9091430C8F719070892B50
:10E3800011F40E94DD5B0E94E1603BC68091440C69
:10E39000882321F480910B0D85FF02C00E94E1606B
:10E3A0008091440C882309F481C081E39AE30E94A0
:10E3B000394510924C0C8091440C80FF0DC08E7F2B
:10E3C00084608093440C10923C0C8DE98093890CFE
:10E3D00081E00E94666B6AC082FF15C080E00E94E7
:10E3E000666B882309F062C09091440C9B7F8091FA
:10E3F0000B0D8E7F80930B0D92609093440C81E007
:10E400000E940E60FEC581FF18C080E00E940E6071
:10E41000892B09F04BC08091440C8D7F1092410CE8
:10E420001092400C10923C0C88608093440C8091B8
:10E430000B0D806280930B0D39C083FF37C0877F3F
:10E440008093440C81EF98E00E94394585EC8093DD
:10E450004C0C8091450C82608093450C90913D0C52
:10E460008091210D890F8093210D9F5F90933D0C2A
:10E470001092440C81E08093880C10924F0C109203
:10E48000500C1092510C1092520C10928A0C109257
:10E490008B0C10928C0C10928D0C80910B0D85FDC5
:10E4A00002C083E001C081E080931F0D2091450CE4
:10E4B00024FFD8C060912B0D70912C0D80912D0DF3
:10E4C00090912E0D611571058105910509F042C0ED
:10E4D0002F7B2093450C1092460C10929A0B1092B1
:10E4E000D40D1092D30D10923C0C8CE291E0A0E080
:10E4F000B0E080932B0D90932C0DA0932D0DB09335
:10E500002E0DE0910F0DF091100D1482E0910F0D82
:10E51000F091100D84812081280F90E018C0E091C7
:10E520000F0DF091100D0780F085E02DE80FF11D23
:10E530003491E0910C0DF0E0E90FF11DEE0FFF1F9B
:10E54000EE0FFF1FEC5EF34F30838F5F9F5F8217EC
:10E5500030F371C07B018C010894E108F1080109D6
:10E560001109E0922B0DF0922C0D00932D0D1093BC
:10E570002E0DE1EFEE16F1040105110591F4CDE346
:10E58000DDE01882EC81FD81898160EF40EE218120
:10E5900002810E947854A796FDE0C93DDF0789F704
:10E5A0004AC0E114F10401051105D1F480E880931B
:10E5B000450C80E060EF40EE29E001E00E947854D5
:10E5C0000E94EB6F82E08093450C80911F0D8F5F5E
:10E5D00080931F0D8091880C8F5F8093880C2BC0D7
:10E5E00021EFE216F1040105110528F5C801B70174
:10E5F0002CE330E040E050E00E94D87961157105CD
:10E600008105910529F486E063E04EE550E611C0EE
:10E61000C801B7012EE130E040E050E00E94D87917
:10E62000611571058105910531F486E063E04AEBDF
:10E630005EE50E941E5480912B0D90912C0DA091AF
:10E640002D0DB0912E0D0097A105B10509F4D9C487
:10E650008F719070A070B0700097A105B10509F09E
:10E66000D0C47DC121FF34C02D7F20622093450C92
:10E67000EDE3FDE0808181608083B7963DE0E93D78
:10E68000F307C1F78091880C813029F087E990E089
:10E69000A0E0B0E004C08CE291E0A0E0B0E08093A4
:10E6A0002B0D90932C0DA0932D0DB0932E0D81E08A
:10E6B0000E94546980910B0D85FDA3C48091880C44
:10E6C000813009F09EC48FE19FE70E94A74F99C453
:10E6D00025FF48C180912B0D90912C0DA0912D0DFF
:10E6E000B0912E0D0197A109B10980932B0D909344
:10E6F0002C0DA0932D0DB0932E0D86399105A105FB
:10E70000B10509F0DFC080910B0D85FD0EC0809131
:10E71000880C813051F41CE0812F6BE040E050E028
:10E720000E9413451F5F1331B9F7E091410DF0913D
:10E73000420D84812081280F90E018C0E091410DA6
:10E74000F091420D0780F085E02DE80FF11D349126
:10E75000E0913E0DF0E0E90FF11DEE0FFF1FEE0F0F
:10E76000FF1FEC5EF34F30838F5F9F5F821730F3A4
:10E77000E091410DF091420D6091370D6450409150
:10E78000380D445080913E0D218102810E947854C1
:10E79000E091680DF091690D84812081280F90E04F
:10E7A00018C0E091680DF091690D0780F085E02DAB
:10E7B000E80FF11D3491E091650DF0E0E90FF11DD6
:10E7C000EE0FFF1FEE0FFF1FEC5EF34F30838F5FE6
:10E7D0009F5F821730F3E091680DF091690D6091B1
:10E7E0005E0D645040915F0D44508091650D218114
:10E7F00002810E947854E0918F0DF091900D8481F8
:10E800002081280F90E018C0E0918F0DF091900DBD
:10E810000780F085E02DE80FF11D3491E0918C0D1B
:10E82000F0E0E90FF11DEE0FFF1FEE0FFF1FEC5E92
:10E83000F34F30838F5F9F5F821730F3E0918F0D2E
:10E84000F091900D6091850D64504091860D44507B
:10E8500080918C0D218102810E947854E091B60D47
:10E86000F091B70D84812081280F90E018C0E091CD
:10E87000B60DF091B70D0780F085E02DE80FF11D82
:10E880003491E091B30DF0E0E90FF11DEE0FFF1FA1
:10E89000EE0FFF1FEC5EF34F30838F5F9F5F821799
:10E8A00030F3E091B60DF091B70D6091AC0D64506E
:10E8B0004091AD0D44508091B30D218102810E94A1
:10E8C000785438C00097A105B105A1F52F7D2064CB
:10E8D0002093450C1092460C82E08093470C1092D6
:10E8E000480C80911F0D815080931F0D0E94145B76
:10E8F00080910B0D85FD1EC08DE06FE040E050E083
:10E900000E9413458EE06FE040E050E00E94134506
:10E910008FE06FE040E050E00E94134580E16FE03F
:10E9200040E050E00E94134581E16FE040E050E09C
:10E930000E94134580912B0D90912C0DA0912D0DCF
:10E94000B0912E0D8F719070A070B0700097A105DE
:10E95000B10509F056C380910B0D85FD52C30E948D
:10E96000DD5B4FC330910B0D31FF6BC03D7F3093AA
:10E970000B0D20642093450CE0910F0DF091100DCC
:10E980006091050D64504091060D445080910C0D2E
:10E99000218102810E94785480910B0D84608E7FCA
:10E9A00080930B0DCDE3DDE011E0EC81FD818981E9
:10E9B00060EF40EE218102810E94785488818E7F31
:10E9C00088831C87A7968DE0C93DD80771F784E03E
:10E9D0000E944265E0910F0DF091100D1482E091BC
:10E9E0000F0DF091100D84812081280F90E018C048
:10E9F000E0910F0DF091100D0780F085E02DE80FEC
:10EA0000F11D3491E0910C0DF0E0E90FF11DEE0FD6
:10EA1000FF1FEE0FFF1FEC5EF34F30838F5F9F5F92
:10EA2000821730F38091D30D9091D40D9160909323
:10EA3000D40D8093D30D83E066EA41E00E944153F8
:10EA4000E0C232FDDEC233FF88C0377F30930B0D4A
:10EA50008091770C6091780C40E050E00E94134563
:10EA6000E0917E0CF0917F0C24913196E49180E04E
:10EA700060EF40EE0E2F0E9478541092480C1092D6
:10EA8000460C80911F0D9091450C882399F19F7B36
:10EA900090629093450C8091D30D9091D40D817428
:10EAA0009E7F9093D40D8093D30D84E08093340D9A
:10EAB00080913C0C81FF03C08D7F886004C082FF81
:10EAC00004C08B7F806180933C0C81E080938E0C2E
:10EAD00080932F0D80E00E94546987E990E0A0E0C8
:10EAE000B0E080932B0D90932C0DA0932D0DB0933F
:10EAF0002E0D4AC080910B0D80619F7B9093450C39
:10EB000080930B0D20914F0C3091500C4091510C83
:10EB10005091520C8091300D9091310DA091320D99
:10EB2000B091330D281739074A075B0711F40E948B
:10EB3000177080910B0D85FD03C084EB90E002C03F
:10EB400081E090E09093D20D8093D10D8CE06FE046
:10EB500048EA5EE50E941E5417C034FF15C080913C
:10EB6000D10D9091D20D009779F001979093D20D2D
:10EB70008093D10D892B41F43F7D30930B0D809113
:10EB8000440C81608093440C8091460C80FFA1C0AE
:10EB90008E7F8093460C8091440C882351F582E34C
:10EBA00090E00E948A5C0E9436568091930C90916E
:10EBB000940C892BF1F082E08093460C8091D30D68
:10EBC0009091D40D82609093D40D8093D30DEDE39A
:10EBD000FDE0808190919A0B82FD03C0892F8F5FA9
:10EBE00001C0892F80939A0BB7962DE0E93DF2077B
:10EBF00081F789E19DE090930E0D80930D0D88ECD7
:10EC000090E09093920C8093910C82E099E790931E
:10EC10004A0C8093490CC9E3DDE000E010E057E2C4
:10EC2000E52EF12C602F8C81847A31F488818195D6
:10EC300088838981819589838091440C882331F46C
:10EC40008091930C9091940C892BD9F18C8182FD49
:10EC500038C0877F82608C8384E00E94C961E88528
:10EC6000F98584812081280F90E015C0E885F98519
:10EC70000780F085E02DE80FF11D3491ED81F0E083
:10EC8000E90FF11DEE0FFF1FEE0FFF1FEC5EF34FBC
:10EC900030838F5F9F5F821748F30E9DA0010F9D09
:10ECA000500D1E9D500D11249A012A5A324F8E810B
:10ECB0009F818217930729F0CA01805B924F9F833F
:10ECC0008E830F5F1F4FA7960430110509F0AACF5E
:10ECD000D5C0823019F0843009F0BDC080919A0B04
:10ECE000882391F08091210D90E087709070892B9E
:10ECF00059F48091D30D9091D40D049728F487E0B6
:10ED000066EA41E00E9441538091460C823009F04E
:10ED100046C08091930C9091940C009709F4AEC07A
:10ED200001979093940C8093930C892B09F0A6C0C3
:10ED300084E08093460C0E947356082FCDE3DDE0FB
:10ED400010E0888181FF26C08D7F886088830B87D3
:10ED500085E0612F0E94C961EC81FD818481208161
:10ED6000280F90E015C0EC81FD810780F085E02D33
:10ED7000E80FF11D3491E981F0E0E90FF11DEE0F8C
:10ED8000FF1FEE0FFF1FEC5EF34F30838F5F9F5F1F
:10ED9000821748F31F5FA796143099F66FC084302E
:10EDA00009F06CC08091480D882309F067C08091FC
:10EDB0006F0D882309F062C08091960D882309F0B9
:10EDC0005DC08091BD0D882309F058C08091D30D9E
:10EDD0009091D40D8D7F9093D40D8093D30D10928C
:10EDE0009A0B1092460C83E19DE090930E0D809358
:10EDF0000D0DC9E3DDE000E010E0A7E2EA2EF12C02
:10EE0000602F8C8183FF20C0877F8C830E9DC00183
:10EE10000F9D900D1E9D900D1124865B924F9F8338
:10EE20008E8399818881882321F4913059F482E07E
:10EE300009C0813011F483E005C08F3F11F08FEFDE
:10EE400001C081E00E94C9610F5F1F4FA796043087
:10EE50001105B1F613C080912B0D90912C0DA0914E
:10EE60002D0DB0912E0D0196A11DB11D80932B0D7E
:10EE700090932C0DA0932D0DB0932E0D8091470CE7
:10EE8000813019F08430B1F402C082E001C088E022
:10EE90008093470CE9E3FDE08481847A31F480813A
:10EEA00081958083818181958183B7963DE0E53DA1
:10EEB000F30791F78091480C8130B9F482E0809398
:10EEC000480C80914C0C40917D0C50E0480F511D36
:10EED0008091770C6091780C0E94134588E592E050
:10EEE00090937A0C8093790C8CC0823029F58091B4
:10EEF000790C90917A0C009709F483C00197909354
:10EF00007A0C8093790C892B09F07BC01092480C05
:10EF100080910B0D85FF07C08CE06FE048EA5EE54D
:10EF20000E941E546EC08091770C6091780C40E076
:10EF300050E00E94134565C0843009F049C082E06A
:10EF400060ED41E00E94415388E08093480C80913D
:10EF50007B0C90917C0C0E948A5C80910B0D85FF4C
:10EF600007C08CE06FE048EA5EE50E941E5408C0CE
:10EF70008091770C6091780C40E050E00E9413453E
:10EF800060917E0C70917F0C80E00E944A54E09169
:10EF90007E0CF0917F0C24913196E4916091770C76
:10EFA00070E0F3E0660F771FFA95E1F76450704068
:10EFB0004091780C50E073E0440F551F7A95E1F7CB
:10EFC00080E00E2F0E94785480EF8093860C19C049
:10EFD0008830B9F48091860C882399F08150809311
:10EFE000860C882371F41092480CE0917E0CF0910D
:10EFF0007F0C24913196E49160EF40EE0E2F0E9439
:10F000007854DF91CF911F910F91FF90EF90089569
:10F01000CF92DF92EF92FF920F931F93DF93CF93E4
:10F02000CDB7DEB7A0970FB6F894DEBF0FBECDBF49
:10F030008DE090E09A8389830E94894D882311F4A2
:10F040000E9402708DE090E0BE016F5F7F4F0E94D2
:10F050009F4D8823A1F58E010D5F1F4F40E050E0CA
:10F0600060E070E0E0E0F0E088E1E82EF12CD8010B
:10F070008D918D0190E0A0E0B0E09F01220F331F41
:10F08000220F331F220F331F6701C21AD30A0C2C21
:10F0900004C0880F991FAA1FBB1F0A94D2F7482BE0
:10F0A000592B6A2B7B2B3196E430F10501F7409305
:10F0B000300D5093310D6093320D7093330DA09647
:10F0C0000FB6F894DEBF0FBECDBFCF91DF911F9179
:10F0D0000F91FF90EF90DF90CF900895EF92FF9205
:10F0E0001F93CF93DF9388E99EE70E948C4F80EBBC
:10F0F0000E94115081EF98E00E94394582E092E62B
:10F100000E94344581E00E941B5485EC80934C0C96
:10F110008091440C81608093440C0E94087882E0C6
:10F1200080930C0D83E080933E0D84E08093650D09
:10F1300085E080938C0D86E08093B30D81E0809311
:10F140004B0C97E2E92EF12C0E943E458823E1F317
:10F150000E9441450E9455700E94666D90933F0C3D
:10F1600080933E0C8091450C982F86FD21C08091A4
:10F17000440C882349F793FFE7CFCDE3DDE010E0AF
:10F18000888182FF10C08A819B810E94F956812F5D
:10F190000E94EE62812F0E949459812F0E94176273
:10F1A000812F0E94AA661F5FA796143049F7CCCF23
:10F1B0002091D30D3091D40DC9018C739070892B9F
:10F1C00079F02038310560F48091210D90E08F7046
:10F1D0009070892B29F489E066EA41E00E9441534E
:10F1E0008091210D90E08F709070892BF9F40E942E
:10F1F0002F5B8091210D90E08F719070892BB1F47D
:10F2000080910B0D85FD12C00E94DD5B80914B0C3F
:10F21000882361F08091D30D9091D40D019731F442
:10F220008091340D66EA41E00E94415380914D0C7B
:10F230008823A9F1815080934D0C882381F580911A
:10F24000880C853010F084EB01C080EF80934D0C6A
:10F2500020912F0D822F90E08E9DF0018F9DF00D5B
:10F260009E9DF00D1124EB5CF24F148A213031F099
:10F270008091700D882311F081E00FC0223031F0B1
:10F280008091970D882311F082E007C0233039F078
:10F290008091BE0D882319F083E080932F0D0E948A
:10F2A0000B5E0E948B5A80910B0D80FF06C08091EF
:10F2B0000D0D90910E0D0E94F9560E94175A0E9452
:10F2C0005865CFE3DDE010E0888199810E94F9560E
:10F2D000812F0E94EE62812F0E949459812F0E94FB
:10F2E000AA66812F0E9417621F5FA796143061F7EC
:10F2F0000E941A572091200D222309F18091D30DED
:10F300009091D40D90FD1BC0822F81508093200DD1
:10F3100090E08F709070892B91F48AE066EA41E06A
:10F320000E9441538091200D882349F48091D30D90
:10F330009091D40D8F779093D40D8093D30D8091BD
:10F34000210D8F5F8093210DFFCE991B79E004C0C2
:10F35000991F961708F0961B881F7A95C9F7809514
:10F360000895AA1BBB1B51E107C0AA1FBB1FA6170C
:10F37000B70710F0A61BB70B881F991F5A95A9F75E
:10F3800080959095BC01CD01089597FB092E072625
:10F390000AD077FD04D0E5DF06D000201AF470957E
:10F3A00061957F4F0895F6F7909581959F4F089549
:10F3B000A1E21A2EAA1BBB1BFD010DC0AA1FBB1F79
:10F3C000EE1FFF1FA217B307E407F50720F0A21BEB
:10F3D000B30BE40BF50B661F771F881F991F1A9458
:10F3E00069F760957095809590959B01AC01BD0182
:08F3F000CF010895F894FFCF4E
:10F3F8000100408891D2E4ADB5B6BEBFFF303132CE
:10F408003334353637383943454748494F505253D6
:10F418005541444B4D4E54222D41424448494B4C92
:10F428004E4F535759222D2E5C30313839414344C1
:10F43800454647494B4D4E4F50535759222D314160
:10F4480042454648494B4C4E4F5052535559222D30
:10F458004142434445484B4C4E4F505253545559E2
:10F468002D3031414243464D4E4F50525354550072
:04F4780001851900F1
:00000001FF
